:1000000000800020BD010000F1D10000A9D1000056
:10001000A9D10000A9D10000A9D10000A9D10000F8
:10002000A9D10000A9D10000A9D10000F1D10000A0
:10003000F1D10000A9D10000F1EE0000F5EF0000C1
:10004000F1D10000F1D10000F1D10000F1D10000A8
:10005000F1D10000F1D10000F1D10000F1D1000098
:10006000F1D10000F1D10000F1D10000F1D1000088
:10007000F1D10000F1D10000F1D10000F1D1000078
:10008000F1D10000F1D10000F1D10000F1D1000068
:10009000F1D10000F1D10000F1D10000F1D1000058
:1000A000C5B20000D1B20000F1D10000F1D10000D2
:1000B000F1D10000F1D10000F1D10000F1D1000038
:1000C000F1D10000F1D10000F1D10000F1D1000028
:1000D000F1D10000F1D10000F1D10000F1D1000018
:1000E000F1D10000F1D10000F1D10000F1D1000008
:1000F000F1D10000D1F10000F1D10000FDF20000CB
:10010000F1D1000035DE0000F1D10000F1D1000096
:10011000F1D10000F1D10000F1D10000F1D10000D7
:10012000F1D10000F1D10000F1D10000F1D10000C7
:10013000F1D10000F1D10000F1D10000F1D10000B7
:10014000F1D10000F1D10000F1D10000F1D10000A7
:10015000F1D10000F1D10000F1D10000F1D1000097
:10016000F1D100000DE10000F1D10000F1D100005B
:10017000F1D10000F1D10000F1D10000F1D1000077
:10018000F1D10000F1D10000F1D10000F1D1000067
:10019000F1D10000F1D10000F1D10000F1D1000057
:1001A000F1D10000F1D10000F1D10000F1D1000047
:1001B000F1D10000F1D10000F1D10000564B4CF21A
:1001C000205210B51A804DF628121A8000BF00BFC9
:1001D0000DF012F8514B4FF010621A60504A9A60BD
:1001E000504ADA60504A136813F4807304D14F49BF
:1001F0000B604FF4A85313604D4B1A78110703D5C9
:100200001A7842F008021A704A4B4B492A221A7097
:100210004A4A4B4B8B4204D252F8040F43F8040B6A
:10022000F8E7484B484900228B4202D243F8042B9E
:10023000FAE74649464A002352F8230041F82300D2
:1002400001336F2BF8D1434B434A802103F8011B44
:100250009342FBD1414B3D4A1A60414B8A221A70AE
:10026000A3F5805324225A70A0221A709A7992071B
:10027000FCD59A79D406FCD43A4A937903F00C035E
:10028000082B384BF9D103221A7140225A719A79FE
:100290009006FCD5334A9179324B4906FBD5324A58
:1002A000324911600221516020221A709A7902F0BD
:1002B0000C020C2AFAD12E4B2E4A1A602E4B2F4AD2
:1002C0001A6000225A60072243F8042C2C4AC3F813
:1002D0000C2D62B60DF076FC144B1B68DA0705D5C1
:1002E00028480DF0C5FA284B284A1A60284B1B787D
:1002F0005B0609D5244C254B22689A4204D121483B
:100300000DF0B6FA0023236010F000FB0CF07AFF2A
:100310000EF0E4FEFEE700BF0E20054030800440F2
:10032000823F04000100002B10D0034014D0034092
:1003300002D0074000E007403C9DFF1F0040010045
:100340004088FF1F3C9DFF1F34A2FF1F0082FF1F3C
:100350000000000000E400E05FE400E008ED00E0E1
:100360000050064000400640448004400000030165
:1003700004800440C010050014E000E0FF76010096
:1003800000002020F453935C1CE00340A5C3945A62
:1003900000F00740FFFFFFFFFFFFFFFFFFFFFFFF32
:1003A000FFFFFFFFFFFFFFFFFFFFFFFFFFFFFFFF5D
:1003B000FFFFFFFFFFFFFFFFFFFFFFFFFFFFFFFF4D
:1003C000FFFFFFFFFFFFFFFFFFFFFFFFFFFFFFFF3D
:1003D000FFFFFFFFFFFFFFFFFFFFFFFFFFFFFFFF2D
:1003E000FFFFFFFFFFFFFFFFFFFFFFFFFFFFFFFF1D
:1003F000FFFFFFFFFFFFFFFFFFFFFFFFFFFFFFFF0D
:10040000FFFFFFFFFFFFFFFFFFFFFFFFDEF9FFFF23
:1004100010B5054C237833B9044B13B10448AFF33E
:1004200000800123237010BD3C9DFF1F00000000D1
:1004300004400100084B10B51BB108490848AFF350
:1004400000800848036803B910BD074B002BFBD0A0
:10045000BDE81040184700BF00000000409DFF1F8E
:10046000044001003C9DFF1F0000000070B44C6878
:10047000A04220D901230133DBB21CB2A60051F8FF
:10048000244084421D46F6D3A04211D005F1804598
:10049000013D965951F8251052F82530401AF21AAC
:1004A00000FB02F0641AB0FBF4F4E01870BC704773
:1004B000905970BC704704260125E5E700280CDA46
:1004C000064A434282FB0320DA17C2EB600000EBCE
:1004D0004000A3EB8000C0F10C007047ABAAAA2A31
:1004E000684B1B880C2B12D8DFE803F01E29333D24
:1004F0001148525C66707A12070063490B68984293
:1005000078D90B6C9842C0F0A580604B186C70478E
:100510005D490B68984240F28E800B6C9842C0F0A7
:1005200096805B4B186C704757490B6898427FD98F
:100530000B6C9842C0F08880564B186C704752493B
:100540000B68984271D90B6C98427AD3524B186C55
:1005500070474D490B68984264D90B6C98426DD333
:100560004E4B186C704748490B68984257D90B6C32
:100570009842C0F084804A4B186C704742490B681F
:10058000984249D90B6C984276D3464B186C704709
:100590003D490B6898423CD90B6C984269D3424B59
:1005A000186C704738490B6898422FD90B6C9842E9
:1005B0005CD33E4B186C704733490B68984222D984
:1005C0000B6C98424FD33A4B186C70472E490B680E
:1005D000984215D90B6C984242D3364B186C704731
:1005E00029490B68984208D90B6C984235D3324B95
:1005F000186C7047254B186870472F4B1868704768
:100600002C4B186870472A4B18687047274B18689E
:100610007047254B18687047224B18687047204B6D
:10062000186870471D4B186870471B4B1868704757
:10063000184B18687047164B18687047174AFFF731
:1006400015BF154AFFF712BF124AFFF70FBF104A36
:10065000FFF70CBF0D4AFFF709BF174AFFF706BFA8
:10066000144AFFF703BF124AFFF700BF0F4AFFF714
:10067000FDBE0D4AFFF7FABE0A4AFFF7F7BE084A69
:10068000FFF7F4BEAA9DFF1F988AFF1F848BFF1FF0
:10069000408BFF1F488DFF1F3889FF1F048DFF1FF0
:1006A000C08CFF1FA08DFF1F7C89FF1FC089FF1F0B
:1006B000048AFF1F648CFF1FFC8BFF1F38B5284A7C
:1006C000284B14881D68AC4247DA274A274B10682C
:1006D0001B88421F191BAB42A8BF2B469142A3EBBC
:1006E0000403C3BF043843430131534393FBF1F187
:1006F00005310A200DF0CEF81D4A1E4B14881B68E8
:10070000A34205DC00210920BDE838400DF0C2B845
:1007100019491A4A0D881068AB42A5EB0401A0F1F3
:100720000502A8BF2B4691420CDD1B1B043800FBC1
:1007300003F30131092093FBF1F1BDE838400531A5
:100740000DF0A8B81B1B02FB03F3092093FBF1F18A
:10075000BDE8384005310DF09DB80021C9E700BF64
:100760001E9EFF1FD89EFF1FF88DFF1FEC9EFF1FD0
:10077000EC9DFF1F6C9DFF1FCC9EFF1F8C8DFF1FEC
:100780002DE9F04F8FB002AD0024E1B26E480AF0BF
:100790000DFE01340C2C45F8040BF6D16B4B6C4C60
:1007A000B3F800E00A9B00227345227014DB089B1B
:1007B0009E4500F3B480069B664A9E4503DD137890
:1007C000002B40F0BC80049B9E4540F3AE804FF070
:1007D000020C84F800C009E0069B5E4A9E45CCBF2F
:1007E0004FF0060C4FF0050C84F800C00C9F039EE0
:1007F0000598079982F800C0BE45D4BF002701279D
:10080000B645D4BF002601268645099ADFF87081D7
:100810000B9B0D9DDFF86CA1DFF86C918AF80060EE
:10082000D4BF002001208E45D4BF0021012188F8CB
:10083000001096454849DFF854B1484E89F8000049
:10084000D4BF002201229E45D4BF002301230A7099
:10085000AE45434A8BF80070D4BF00250125012026
:10086000137035700DF052FB3E4B3F4A1D681188E6
:100870003E4BA842D4BF002201220B291A7001D995
:100880000C2901D0A84246DC00230193384B9AF88A
:1008900000E01F7899F800C098F800209BF800301D
:1008A0002D49DFF8ECA091F800902D49367891F8A9
:1008B00000802478A7EB4E07CCEB070CA2EB82025A
:1008C000C3EB83776244C3EB8703134403EB490311
:1008D000BAF80020274FDFF8BCE0B7F800C0264F79
:1008E000434403EB8606033A0C2313FB046602EB36
:1008F000420206EB8202019BCEF800606244A842ED
:10090000A2F10C021A44C8BF1C4B3A60C8BF1E704B
:100910000FB0BDE8F08FA1F10C030193B6E74FF0E3
:10092000040C84F800C00B4A60E7029B9E45C6BFDA
:100930004FF0010C84F800C04FF0000C56E74FF068
:10094000030C84F800C051E7189EFF1FF49EFF1FA0
:10095000449EFF1F509EFF1FD59EFF1F319FFF1F0C
:10096000309FFF1F548CFF1FCE9EFF1F9C9DFF1FBB
:10097000BC8CFF1FAC9DFF1FF89EFF1FF69EFF1F44
:100980002D9FFF1FC49EFF1F2C9FFF1F2E9FFF1F29
:10099000B49EFF1FF89DFF1F30B50E4C85B001239C
:1009A00020463C2202210BF02FFF20460BF0BCFE1C
:1009B00001250022402180232046019100930295C9
:1009C0001146054B0BF0BCF9204605B0BDE83040A0
:1009D0000CF04CB8049FFF1F0032010010B500EB73
:1009E000C000821DD2B293B284B09C1E981C3D23DD
:1009F00003918DE81900392102480BF005F904B084
:100A000010BD00BF049FFF1F70B50E4C84B01225AF
:100A10000422012306460390029320468DE8240019
:100A2000142310210BF0F0F80622092302930396F9
:100A3000019520460092142310210BF0E5F804B034
:100A400070BD00BF049FFF1F10B50C4C81B2204643
:100A50000BF0BCFB204602210BF0B2FB204621220A
:100A60005A210BF0A9FB064B204619880EF02EFBED
:100A70002046BDE810400EF0D9BA00BF049FFF1F0A
:100A8000B88CFF1F10B50C4C81B220460BF09EFBBA
:100A9000204602210BF094FB204621225A210BF024
:100AA0008BFB064B204619880EF010FB2046BDE854
:100AB00010400EF0BBBA00BF049FFF1F948AFF1FB7
:100AC00010B50C4C81B220460BF080FB2046022171
:100AD0000BF076FB2046212253210BF06DFB064BD9
:100AE000204619880EF0F2FA2046BDE810400EF0BC
:100AF0009DBA00BF049FFF1FBA8CFF1F38B50C467C
:100B00000546C9B20CF028FB210A681CBDE8384034
:100B10000CF022BB38B505460CF004FB4FF0000486
:100B200060F30704681C0CF0FDFA60F30F24A0B218
:100B300038BD00BF38B50F4D2B78013B01381B0283
:100B4000C4B203F47063200443F4404343F00C0345
:100B500000F4FE0018430DF087FF2868013860F0AC
:100B60003F00C0B20DF040F92046BDE838400DF01E
:100B70003BB900BF049EFF1F38B5104D2B78013BD9
:100B80001B0203F47063044643F41043000443F073
:100B9000090300F4FE0018430DF066FF28680138D1
:100BA00060F06F00C0B20DF01FF920460DF01CF987
:100BB0000020BDE838400DF017B900BF049EFF1FAC
:100BC00038B50E4D2B78013B1B0203F470630446CD
:100BD00043F45043000443F00D0300F4FE001843B7
:100BE0000DF042FF2868013860F02F00C0B20DF010
:100BF000FBF82046BDE838400DF0F6B8049EFF1F14
:100C000010B504464FF440600DF09EF80DF0F6F874
:100C10002CB1102C044BA8BF10241C6010BD024B3B
:100C200001241C6010BD00BF049EFF1F10B50446C8
:100C300041F0E0000DF0D8F804F07F000DF0D4F89A
:100C4000C4F3C610BDE810400DF0CEB838B5114D54
:100C50002B78A0F50052013B1B0202F30D0202F5B6
:100C6000005203F47063044643F46043100443F0FD
:100C70000E0300F4FE005204184302F0FE4210433B
:100C80000DF0F2FE296801392046C9B2BDE83840AE
:100C9000FFF7CCBF049EFF1F2DE9F04F172087B050
:100CA0000DF034F9DFF86093C9F8000016200DF05C
:100CB0002DF9B84BB84A1B8810600C2B00F04F82FE
:100CC0000023B64C0F2023700DF020F9B44A23788E
:100CD000128801921146B34A054652F821404BB1A1
:100CE00020460FF057FB4FF07C510FF0A7FB0FF0A1
:100CF00081FD0446AC4BDFF814831B88D8F800A0B4
:100D0000AA4A013B554552F823B050DAA84BA94EE8
:100D10001B88012B00F0D581A74BA84A30680093AF
:100D20001F4604920FF036FB4FF07C510FF086FB0C
:100D3000A34902900988039120460FF02BFB049AE7
:100D400003993F6852F821100FF078FB014600200C
:100D50000FF06AFA0FF04EFDCBEB070BAB45CAEB79
:100D60000B015A46B8BF2A46CAEB02028842BABFF4
:100D700000FB02220131424392FBF1F0DFF890A226
:100D80000FF008FB4FF07C510FF058FB02990FF069
:100D90004DFA0FF02FFD30608A4A1288013A032A7B
:100DA0006AD8DFE812F0EB00D3005300DF00DFF871
:100DB00060A2DAF80020954238DD7D4B05921B8851
:100DC0007C4E012B00F0AC817B4B00931F463068BA
:100DD0007A4B04930FF0DEFA4FF07C510FF02EFBAC
:100DE000774902900988039120460FF0D3FA0399BE
:100DF000049B3F6853F821100FF020FB0FF0FAFC22
:100E0000059ABB44C2EB0B01AB45A8BFAB46884279
:100E1000C2EB0B0B80F2AD8100FB0BBB01319BFBE6
:100E2000F1F00FF0B7FA4FF07C51ADE7614E624B35
:100E3000306800931F460FF0ADFA4FF07C510FF071
:100E4000FDFA0FF0D7FC3F683060A5E738460FF099
:100E5000A1FA5D490FF0F2FA834628460FF09AFA9C
:100E60005A490FF0EBFA014658460FF0DFF90FF040
:100E7000C1FC009B074618605549564A08881288ED
:100E8000D9F80010544DC0EB070EC3199142C8F8B1
:100E900000E0CAF80030B5F800E080F2DC80002500
:100EA000C2EB0E0C3C4B64451F6880F2C880631C8B
:100EB000974205FB03F50CF1010C95FBFCF5C0F224
:100EC0006681BE45A8BFBE46C2EB0E0E03FB0EF404
:100ED00094FBFCF4914200F39D80BA42C0F29A80E8
:100EE0003E4C20680FF056FA3D490FF0A7FA3D49F5
:100EF0000FF09CF90FF07EFCA0F5FF531C3B082B74
:100F000098BF4FF400503368184400282060C0F2A6
:100F10009480B0F5804F80F2A580334B1B781BB1D5
:100F2000B0F5005F40F0A680304D2B78002B40F0EC
:100F3000A9802F4D20682B68284C984203D0FFF7DA
:100F400085FE23682B6007B0BDE8F08F38460FF0B0
:100F500021FA28490FF072FA834628460FF01AFA50
:100F600025497EE738460FF015FA1D490FF066FA5D
:100F7000834628460FF00EFA204972E738460FF0F4
:100F800009FA1F490FF05AFA834628460FF002FA71
:100F90001C4966E7CE9EFF1F009FFF1F659DFF1F38
:100FA000D49DFF1F088BFF1FB88CFF1FC88BFF1F2E
:100FB000FE9DFF1F8C9DFF1FC09EFF1F6C8AFF1FA1
:100FC000C09DFF1F948AFF1FCDCC4C3FCDCC4C3E23
:100FD000BA8CFF1F349EFF1FBC9DFF1F988DFF1F03
:100FE0009A99193FCDCC4C45E09EFF1F199EFF1FDB
:100FF0003489FF1F6666663FCDCCCC3DCDCCCC3E60
:101000003333733FCDCC4C3DD09DFF1FE89DFF1F78
:101010003C9EFF1F019B002B3FF462AF2B1B002B5C
:10102000B8BF5B42092B34DC33685A4C4FF4005094
:10103000184400282060BFF66CAF002214E09742ED
:1010400005FB04F5B8BF002395FBFCF580F2968004
:1010500093FBFCF43EE77145D4BFC2EB0105C2EB44
:101060000E051DE743F6FF724B4B22601B78002BE9
:101070003FF45AAF00210D200CF01AFD474B01221E
:101080001A7056E701210D200CF012FD00232B7081
:101090004FE705F500500130001B0FF07BF9404988
:1010A0003C4C0FF0CBF9054620680FF073F93D4931
:1010B0000FF0C4F9014628460FF0B8F80FF09AFB7C
:1010C00021E7394B00931F463068384B04930FF0EB
:1010D00061F94FF07C510FF0B1F9354A0290128856
:1010E000039220460FF056F9039A049B3F6853F889
:1010F00022100FF0A3F90FF07DFBCBEB070BAB45F4
:10110000CAEB0B02B8BFAB46CAEB0B0B8242C6BFA1
:1011100000FB0BBB013200FB0BFB9BFBF2F02DE64F
:10112000224B0493204B306800931F460FF032F996
:101130004FF07C510FF082F91D490290098803910C
:1011400020460FF027F9049B03993F6853F82110BC
:101150000FF074F9014600200FF066F84EE601200A
:101160000CF0D4FE134B1B689842D4BF002301231C
:10117000A7E500FB0BFB9BFBF1F052E67745D4BFE4
:10118000C2EB0703C2EB0E0304FB03F360E79646D2
:101190009AE600BF988DFF1FE09EFF1F199EFF1F5C
:1011A000CDCCCC3E9A99193FC09EFF1F6C8AFF1F81
:1011B000C09DFF1F548CFF1F38B5054642F0B0009C
:1011C0000C460CF011FE28460CF00EFEE0B2BDE815
:1011D00038400CF009BE00BF70B50F4D2B78013BB5
:1011E0001B0203F47063044643F4304308062204F0
:1011F00000F0FE4043F00B03034302F4FE001843EB
:101200000E460DF031FC2A68013A3146E0B2D2B206
:10121000BDE87040FFF7D0BF049EFF1F10B50C4C17
:10122000236843B90B4B1B88022B0CD00A4A0023BE
:101230001370236010BD00210520FFF7CDFF054B83
:101240001B88022BF2D100214120FFF7C5FFEDE7FB
:10125000E89EFF1F289EFF1FEE9DFF1F08B564211B
:101260000720FFF7B9FF7F210B20BDE80840FFF7FB
:10127000B3BF00BF10B500217B20FFF7ADFF0024F6
:10128000E0B2FFF779FC013402200CF04DFC802C19
:10129000F6D110BD30B58DB06D460024E1B23448B2
:1012A0000AF084F801340C2C45F8040BF6D1314BCC
:1012B0000A9A1B889A4216DA009A934213DD029A20
:1012C000934210DD049A93420DDD2B4A2B4B11887B
:1012D0001B882B4A0B4412685B10934238DB294A67
:1012E0001268934201DB0DB030BD274B00241C7007
:1012F000FFF7C0FF21460D200CF0DAFB32200CF086
:1013000013FC01210D200CF0D3FB32200CF00CFC5F
:1013100021460D200CF0CCFB32200CF005FC012105
:101320000D200CF0C5FB32200CF0FEFB21460D20F9
:101330000CF0BEFB32200CF0F7FB0D2001210CF06D
:10134000B7FB4FF42F700DB0BDE830400CF0ECBB94
:101350000D4B002101240D201C700CF0A9FB322044
:101360000CF0E2FB0D2021460CF0A2FB3220EAE754
:10137000189EFF1FF49EFF1FBC9DFF1F349EFF1F82
:10138000D09DFF1F009FFF1FA89DFF1F294A2A4BCA
:1013900010881B68294A2A491288834270B52DDBC0
:1013A0009342A8BF134698420B60C8BF002327DDB5
:1013B000101AB0F5804FAABF9B03C3EB83330130F3
:1013C00093FBF0F0FFF78CF81E4E3368C0F3C615A0
:1013D0009D42044606D01C4B1B882BBB1B4B1B8815
:1013E000F3B935601A4D2B689C4206D0164B1B880A
:1013F0005A1F032A0BD92C6070BD70BD03460860CC
:101400009A42D4BFC0EB0203C0EB0303D0E7114AFA
:10141000D05C04F07F012030FFF7DEFE2C6070BD51
:101420002846FFF7CDFBDCE70A4A2946D05CFFF7E8
:10143000D3FED3E71E9EFF1FB09EFF1FEC9EFF1F33
:10144000D89EFF1FDC9DFF1F989EFF1F1A9EFF1F47
:10145000A49DFF1FA88CFF1F2DE9F0417B4C7C4D04
:1014600020680EF097FF7B490EF0E8FF064610203B
:101470000CF04CFD0EF08EFF77490EF0DFFF314689
:101480000EF0D4FE0FF0B6F92B882060002B3FD071
:10149000724F3A8890423BDB01467148067836B974
:1014A0004FF0010E042B80F800E000F0B380012B18
:1014B0006AD0022B00F0BC80032B36D1694B1B880D
:1014C000092B32D023683C88674AA342128853DB39
:1014D0009342D4BFC4EB0303C4EB0203141B7E2C62
:1014E000DFF88881D5BFC3EB8313C3EBC3135B0065
:1014F000013493FBF4F4D8F800300134A34203D054
:1015000021464A20FFF768FEC8F80040BDE8F08198
:10151000534A117849B10024012B147016D0022BC4
:101520001FD0032B03D0042B28D0BDE8F0814D4BF6
:101530001B88092BF9D04D4D2B68002BF5D0214687
:101540004A20FFF749FE2C60BDE8F081474D2A682C
:10155000002AEAD018462146FFF73EFE2C60BDE87F
:10156000F081424D2B68002BDFD021460420FFF78D
:1015700033FE2C60BDE8F0810023AFE72146402018
:10158000BDE8F041FFF728BE374B1B888B42D4BF24
:10159000C2EB0306C2EB01069A1ADFF8D0807E2A5E
:1015A000D8BFC6EB8616D8F80030C6BFC6EBC61645
:1015B0000132760096FBF2F60136B34203D0314693
:1015C0000120FFF709FE2B88C8F80060022B7FF48A
:1015D00073AF23683E88244AB34212882CDA002372
:1015E000961B7E2EDFF88480D5BFC3EB8313C3EB3D
:1015F000C3135B00013693FBF6F6D8F800300136D2
:10160000B34220D031460420FFF7E6FD2B88C8F80E
:10161000006051E77F214020FFF7DEFD2B88012B82
:10162000D4D121683A88104B91421B88B4DBADE7D6
:101630000D4A236812883E889A42D4BFC6EB020343
:10164000C6EB0303CCE70223E1E700BFC49DFF1F05
:10165000CC9DFF1F9A99193FCDCCCC3E969DFF1F84
:10166000DC9EFF1F989EFF1F4E9EFF1F309EFF1F98
:1016700038B5114A114B14881B68114AA3421288CD
:1016800013DA0023141B0F4D7F2CCABFDB01C3EB01
:10169000C313013493FBF4F42B68A34203D0214617
:1016A0000520FFF799FD2C6038BD9342D4BFC4EBF1
:1016B0000303C4EB0203E5E7EC9DFF1F6C9DFF1FD6
:1016C000CC9EFF1FE89EFF1F10B50B200CF0F6F913
:1016D000D8B111200CF01AFC134B1860134A128871
:1016E0007AB113491B68098899420ADC114C2378A6
:1016F0001BB9022A13D001232370BDE81040FFF765
:10170000B7BF0C4B1B7833B910BD15200BF026FC6E
:10171000054B1860E2E7BDE81040FFF77FBD7F2171
:101720004120FFF759FDE6E76C9DFF1F289EFF1F34
:10173000EC9DFF1FEE9DFF1F38B5054642F090005F
:101740000C460CF051FB28460CF04EFBE0B2BDE815
:1017500038400CF049BB00BF70B50F4D2B78013BF2
:101760001B0203F47063044643F4104300040A06AA
:1017700000F4FE0043F00903034302F0FE40184367
:101780000E460DF071F92A68013A31462046D2B270
:10179000BDE87040FFF7D0BF049EFF1F08B50BF0F7
:1017A00079FC084809F09AFD002301214FF07E5290
:1017B000054809F08BFF04210448BDE808400AF001
:1017C0009BBF00BF189EFF1F709EFF1F049FFF1F3F
:1017D00000B5244B1A7883B00121052302B30022FF
:1017E00001910093114620480AF022F91F4B1A7804
:1017F00002B3052301220192009300220A211A4814
:101800000AF016F91A4B1A7802BB0523012101913F
:101810000093142114480AF08DF903B05DF804FB1D
:1018200001910093114610480AF084F90F4B1A7881
:10183000002ADED105230121019100930A210A48E3
:101840000AF078F90A4B1A78002ADED00523012223
:10185000019200930022142103480AF0E9F803B032
:101860005DF804FBD59EFF1F049FFF1F309FFF1FE5
:10187000319FFF1F2DE9F04FC54D2B78A3F10A02D0
:10188000022A83B040F22281C24EA3F11402022A3E
:101890003CD8DFF83083C04AD8F800E01268BF496E
:1018A0009645D1F8009080F20E82C2EB090CBCF193
:1018B0005A0F4FF00004BA4F40F31282D7F800A03D
:1018C0005B2052450CF1010100FB04F494FBF1F4A0
:1018D00004F11C0440F3E882002292FBF1F11C3178
:1018E000A14200F0158209B200232622AD480AF079
:1018F00095FE21B201232622AA480AF08FFEA948AC
:101900000BF0B4F8D8F800202B783A60A3F11E024F
:10191000022A00F28B80A44FDFF8ACA23968DAF813
:101920000030DFF8A8929942D9F8002080F25A815D
:10193000D01A5A284FF00004DFF8948240F35E81F9
:10194000D8F800104FF05B0E8B420EFB04F400F150
:10195000010E94FBFEF404F11C0400F3B9829142E1
:10196000A8BF1146C3EB010C5B2101FB0CF191FBFD
:10197000FEF11C31A14200F0548109B2002326225D
:1019800088480AF04BFE21B20123262285480AF03E
:1019900045FEDAF80030DFF83CA2D9F80020DAF88A
:1019A000001099424FF0010CA2EB0300C0F24481F9
:1019B0009142D4BFC3EB0104C3EB02045A28DFF801
:1019C000189240F34081D9F800B000F1010E5B4558
:1019D0004FF05B0000FB04F494FBFEF404F11C04E4
:1019E00000F378825A45A8BF5A46D21A5B2000FB02
:1019F00002F090FBFEF01C30A04200F0398101B2F1
:101A00000023262267480AF009FE21B2012326227C
:101A100064480AF003FE63480BF028F8DAF8001077
:101A20003A682B78C8F80020C9F80010A3F1280202
:101A3000022A42D8DFF8A4815C4AD8F800E0126894
:101A40005B499645D1F800C080F21A81C2EB0C01C7
:101A50005A294FF00004574F40F31E8138684FF069
:101A60005B09824201F1010109FB04F494FBF1F4EA
:101A700004F11C0400F316828445A8BF8446C2EB1F
:101A80000C0C5B2000FB0CF090FBF1F11C31A1422F
:101A900000F0158109B20023262242480AF0BEFD5B
:101AA00021B2012326223F480AF0B8FD3D480AF042
:101AB000DDFFD8F800202B783A603C3B012B40F248
:101AC0003A810023337003B0BDE8F08F3A4ADFF863
:101AD00010811668D8F800E0384AB645126834DA42
:101AE000911B5A294FF00004354F38DD38684FF00C
:101AF0005B0C864201F101010CFB04F494FBF1F450
:101B000004F11C0400F3E8819042A8BF1046861B34
:101B10005B2000FB06F090FBF1F11C31A14230D0BC
:101B200009B2002326221F481A4E0AF077FD21B27F
:101B3000012326221B480AF071FD1A480AF096FF7D
:101B4000D8F800202B783A609FE6911B9645D4BFC9
:101B5000C6EB0E04C6EB02045A29194FC6DCD7F8AF
:101B600000C05A20664500FB04F494FBF1F404F134
:101B70001C0440F3BC81002292FBF1F11C31A14214
:101B8000CED1044E3278002A40F0D3807246DAE794
:101B9000149EFF1F749DFF1F688AFF1FE48DFF1FA7
:101BA0005C9EFF1F049FFF1FD09DFF1FFC8DFF1F2A
:101BB0005C8AFF1F889DFF1F389EFF1F588AFF1FEA
:101BC000D09EFF1F6C9DFF1FE88DFF1F3C8BFF1FEA
:101BD000D89DFF1F009FFF1F349FFF1FC49DFF1F45
:101BE000B09EFF1FD01A9142D4BFC3EB0104C3EBD8
:101BF00002045A28DFF824833FF7A2AED8F800E0A9
:101C00005A21734501FB04F494FBF0F404F11C0425
:101C100040F36481002191FBF0F11C31A1427FF47B
:101C2000ACAE3478002C77D1DFF8F4A2DAF80010EB
:101C30009942A446BFF6BCAE5A284FF00004DFF824
:101C4000E4923FF7C0AED9F800E04FF05A0B73456D
:101C50000BFB04F494FBF0F404F11C0440F3198131
:101C60004FF0000B9BFBF0F01C30A0427FF4C7AE9E
:101C70003378002B56D1BCF1000F3FF4D1AECAE649
:101C8000C2EB0C01E645D4BFC2EB0E04C2EB0C0460
:101C90005A299B4F3FF7E2AED7F800905A204A45A9
:101CA00000FB04F494FBF1F404F11C0440F30781FD
:101CB000002292FBF1F11C31A1427FF4EBAE3278AD
:101CC00072BB7246F8E6C2EB090CCE45D4BFC2EB3C
:101CD0000E04C2EB0904BCF15A0F8A4F3FF7EEAD78
:101CE00039685A208A4200FB04F494FBFCF404F1A6
:101CF0001C0400F3E2804945A8BF4946891A5A20CE
:101D000000FB01F090FBFCF11C31A1427FF4EBAD34
:101D100032781AB97246F8E509B235E609B2E9E552
:101D200009B2BEE601B20123262277480AF076FC0A
:101D300071E609B2FCE6262200248DE81400762321
:101D40001C217148714D724F09F0A4FE1DE08242C2
:101D5000D4BFC3EB0201C3EB0001D31A4FF05A0EFC
:101D600073454FF05B00CABF41430EFB01F10133E5
:101D700091FBF3F303F11C0101231C44262209B259
:101D800061480AF04BFC0C2C09D0E1B2614809F023
:101D90000DFB2B683A688342D9DD0021DDE7DFF8CF
:101DA00088815D4C01200CF0B1F8D8F800C02368A0
:101DB0003A682968CCEB030E8B1A9E45CCEB0000E9
:101DC0005BDD03FB00000EF1010390FBF3F3134412
:101DD00099424EDC9A42D4BFC1EB0203C1EB03032C
:101DE000521A5A2ACABF5B215A21013201FB03F35E
:101DF00093FBF2F202F11C0109B2012326224248B0
:101E00000AF00CFC00200CF081F8D8F800E03A68E9
:101E1000296824688B1ACEEB04049C42CEEB0000A8
:101E200031DD03FB0000631C90FBF3F31344994284
:101E300021DC9A42D4BFC1EB0203C1EB0303521A67
:101E40005A2ACABF5B215A21013201FB03F393FBDB
:101E5000F2F202F11C0109B2012326222A480AF0FB
:101E6000DDFB29480AF002FE0023337003B0BDE811
:101E7000F08F0023B4E70023E1E703FB00F393FBBB
:101E8000FEF31344A4E703FB00F393FBF4F31344C2
:101E9000CDE77245D4BFC3EB0203C3EB0E030BFBCC
:101EA00003FBDFE69446EAE5D145D4BFC2EB090265
:101EB000C2EB0A0200FB02F20FE511461EE7CC4519
:101EC000D4BFC2EB0C02C2EB090200FB02F2F0E647
:101ED000194647E51A4688E5304618E67245D4BFEC
:101EE000C3EB020EC3EB0E0E01FB0EF193E662454F
:101EF000D4BFC6EB0202C6EB0C0200FB02F23BE6CB
:101F0000889DFF1F5C9EFF1F049FFF1FF48DFF1F16
:101F1000408CFF1F189EFF1F5C8CFF1FD89DFF1F6A
:101F2000009FFF1F349FFF1F608AFF1F08B581B20B
:101F300017480AF04BF9022115480AF041F921220D
:101F40005A2113480AF038F9124B114819880DF03C
:101F5000BDF80F480DF06AF80F4B197891B90C488D
:101F60000AF034F901210A480AF02AF933227421CF
:101F700007480AF021F9012208490548BDE8084050
:101F80000DF040B8012102480AF020F9EAE700BF4D
:101F9000049FFF1F609EFF1FE29EFF1F542F010042
:101FA00010B5104C012120460AF010F920460121FD
:101FB0000AF006F92046342255210AF0FDF82046A1
:101FC000022209490DF01EF82046052207490DF0AE
:101FD00019F820460DF02AF82046BDE810400AF016
:101FE00045BD00BF049FFF1F402F0100442F01008B
:101FF0002DE9F84F0C200AF07DFF0C200BF048FD76
:10200000022103200BF068FD022104200BF064FD87
:10201000022105200BF060FD022106200BF05CFD83
:1020200001210A200BF058FD012109200BF054FD7D
:1020300001210D200BF050FD02210B200BF04CFD77
:1020400001210C200BF048FD00210C200BF030FD8D
:102050000020FEF75FFD172840F28A8204200BF073
:102060002DFD002800F07E820020FEF753FD1F2882
:1020700000F0BA821F210020FEF740FD0C210E2047
:10208000FEF73CFD01211020FEF738FD0221122051
:10209000FEF734FD00211420FEF730FD002116204C
:1020A000FEF72CFD02211820FEF728FD01211A2041
:1020B000FEF724FD02211C20FEF720FD04211E2036
:1020C000FEF71CFD14212020FEF718FD012126201B
:1020D000FEF714FD03212820FEF710FD04212C201B
:1020E000FEF70CFD14212E20FEF708FD0021302004
:1020F000FEF704FD0C213220FEF700FD0021342004
:10210000FEF7FCFC00213620FEF7F8FC0021382009
:10211000FEF7F4FC00213A20FEF7F0FC00213C2001
:10212000FEF7ECFC00213E20FEF7E8FC00214020F9
:10213000FEF7E4FC00214220FEF7E0FC1F214420D2
:10214000FEF7DCFC13214620FEF7D8FC0E214820C8
:10215000FEF7D4FC11214A20FEF7D0FC0A214C20C6
:10216000FEF7CCFC00214E20FEF7C8FC06215020D3
:10217000FEF7C4FC02215220FEF7C0FC0F215420C0
:10218000FEF7BCFC00215620FEF7B8FC0220FEF74B
:10219000C1FCBA4BBA4C18800420FEF7BBFCB94B0B
:1021A000DFF89C8318800620FEF7B4FCB64BDFF8FE
:1021B00094A318800820FEF7ADFCB44BB44E1880F1
:1021C0000A20FEF7A7FCB34BB34D18800C20FEF796
:1021D000A1FCB24B18800E20FEF79CFCB04B18807F
:1021E0001020FEF797FC20801220FEF793FCAD4BE9
:1021F00018801420FEF78EFCAB4B18801620FEF7DB
:1022000089FCAA4B18801820FEF784FCA84B188084
:102210001A20FEF77FFCA74B18801C20FEF77AFCE3
:10222000A54B18801E20FEF775FCA44B18802020BB
:10223000FEF770FCA24B18802220FEF76BFCA14B2E
:1022400018802420FEF766FC9F4B18802620FEF79E
:1022500061FC9E4B81462820A3F80090FEF75AFCB3
:102260009B4B18802A20FEF755FC9A4B07462C20E2
:102270001F80FEF74FFC984B18802E20FEF74AFC7B
:10228000964B18803020FEF745FC954B1880322085
:10229000FEF740FC934B18803420FEF73BFCA8F877
:1022A00000003620FEF736FCA8F802003820FEF7C2
:1022B00031FCA8F804003A20FEF72CFCA8F8060030
:1022C0003C20FEF727FCA8F808003E20FEF722FC81
:1022D000A8F80A004020FEF71DFCA8F80C004220D8
:1022E000FEF718FC804B80464420A3F80080FEF7E0
:1022F00011FC7E4BA0F1180246201A60FEF70AFC82
:10230000A0F118034820CAF80030FEF703FCA0F142
:1023100018034A20CAF80430FEF7FCFBA0F11803AA
:102320004C20CAF80830FEF7F5FBA0F118034E2048
:10233000CAF80C30FEF7EEFB6D4B18805020FEF70C
:10234000E9FB6C4B18805220FEF7E4FB6A4B1880C7
:102350005420FEF7DFFB30805620FEF7DBFB674A98
:10236000DFF8E4E16649D2F800A0664B664ADEF881
:1023700000B0D1F800C0D3F800E01168634A644BA4
:1023800085F80090CCEB0B0CCEEB0A0E82FB0CBA5E
:10239000D3F800905F4BE2444FEAEC7CCCEBAA1CF4
:1023A000DFF8A8A118805C4BCAF800C082FB0EAC15
:1023B00018685A4BF4444FEAEE7ECEEBAC1EDFF8C1
:1023C00090C11B68CCF800E0C1EB090982FB09CE83
:1023D000C01ACE44DFF87CC1514B52491B680968D2
:1023E0004FEAE979C9EBAE1ECCF800E082FB00ECC5
:1023F0008444C017C1EB030EC0EBAC10DFF858C12A
:1024000082FB0E92CCF8000072444748DFF84CC1C2
:102410004FEAEE7E5FFA88F8CEEBA212026008F077
:102420000209424A8CF8009008F0040C82F800C0BF
:10243000DFF82CE13E483F4A08F008088EF800809B
:1024400000681268C91A121A9142A7EB03030FDD44
:1024500002FB0333013193FBF1F30344364A37485F
:1024600013605A2108F0DEFF002840F0CA80FEE722
:1024700002FB03F292FBF1F30344EFE71E9EFF1F02
:10248000609EFF1FEC9EFF1FEC9DFF1FCC9EFF1F59
:10249000BA8CFF1F349EFF1FF69DFF1FBC9DFF1FC0
:1024A000AC9DFF1F989EFF1F1A9EFF1F5C9DFF1F84
:1024B000289EFF1FD49DFF1FCC9DFF1FC09DFF1FA7
:1024C000DE9EFF1F969DFF1F4E9EFF1F6C9EFF1FEF
:1024D000B49EFF1FF49EFF1FAA9DFF1FBC9EFF1FFF
:1024E000689DFF1FCE9EFF1FEE9EFF1F048BFF1FE8
:1024F000CA9DFF1FB88CFF1F948AFF1FE48DFF1F2A
:10250000389EFF1F688AFF1FE88DFF1FC94216B261
:102510003C8BFF1FFE9DFF1F5C8AFF1FFC8DFF1F72
:10252000408CFF1FF48DFF1FE09DFF1F1C9EFF1FAF
:10253000608AFF1F5C8CFF1F548CFF1F189EFF1FBB
:10254000789DFF1F448CFF1F588AFF1FA09EFF1F0E
:10255000B89EFF1FA49EFF1F549EFF1FC29DFF1F1A
:10256000E29EFF1F06200BF0A9FA00287FF47CAD45
:102570001F210020FEF7C2FA4FF4AF610220FEF7E0
:10258000BDFA04204FF47A61FEF7B8FA0B200BF085
:1025900095FA002800F0A88040F628210620FEF7D2
:1025A000ADFA40F6E4410820FEF7A8FA4FF4AF6117
:1025B0000A20FEF7A3FA40F6FC010C20FEF79EFA73
:1025C0004FF496612220FEF799FA4FF41661242009
:1025D000FEF794FA7D212A20FEF790FA0020FEF7FC
:1025E00099FA1F287FF446AD04200BF067FA002803
:1025F0007FF4CCAD06200BF061FA00283FF43AAD31
:10260000C4E53F4A3F481268DFF800813E4F00238F
:10261000012109F079F8FEF7BFF90023C8F800306E
:102620003B604FF001090F200BF070FC3B68DFF8B6
:10263000D8A003440E203B600AF090FCD8F800308C
:1026400009F0010103440D20C8F8003009F1010927
:102650000BF02EFAFA200BF067FAB9F1050FE2D170
:10266000DAF80030D8F8002031882848284E002BAE
:10267000B8BF0333002AB8BF03329B103B609210EF
:10268000244F02605A1A0D200B44002133603A6037
:102690000BF00EFAFA200BF047FA01210D200BF097
:1026A00007FAFA200BF040FA00210D200BF000FA97
:1026B000FFF776FC40F2DC500BF036FA164B0126A1
:1026C00004201E600BF0FAF910B9144B28701E702C
:1026D0002378134A18461370FEF792FA01210D2051
:1026E000BDE8F84F0BF0E4B94FF496610620FEF711
:1026F00005FA4FF4FA610820FEF700FA56E700BF2A
:102700004C8AFF1F709EFF1FC09EFF1F709DFF1F02
:102710003C9EFF1FE89DFF1FC89EFF1F9D9DFF1F42
:10272000379EFF1F70B5194C82B034260023012557
:1027300020460193009640230B223F2109F078F9AF
:1027400040230B222046009601953F2109F0F2F923
:102750002946204609F03AFD2946204609F030FD79
:1027600020460F22442109F027FD0922084920466E
:102770000CF048FC20460CF059FC064B20461D701E
:1027800002B0BDE870400AF071B900BF049FFF1F9E
:102790004C2F0100FC9EFF1F70B5194C82B03426EF
:1027A0000023012520460193009640230B223F2160
:1027B00009F03EF940230B222046009601953F2167
:1027C00009F0B8F92946204609F000FD29462046BF
:1027D00009F0F6FC20460F22512109F0EDFC0522FC
:1027E000084920460CF00EFC20460CF01FFC284641
:1027F000FEF72AF9204602B0BDE870400AF036B96B
:10280000049FFF1F582F010070B5194C82B0342669
:102810000023012520460193009640230B223F21EF
:1028200009F006F940230B222046009601953F212E
:1028300009F080F92946204609F0C8FC29462046BF
:1028400009F0BEFC20460F22512109F0B5FC0522FB
:10285000084920460CF0D6FB20460CF0E7FB284642
:10286000FEF72EF9204602B0BDE870400AF0FEB82F
:10287000049FFF1F582F010070B5194C82B03426F9
:102880000023012520460193009640230B223F217F
:1028900009F0CEF840230B222046009601953F21F7
:1028A00009F048F92946204609F090FC29462046BF
:1028B00009F086FC20460F22512109F07DFC0522FB
:1028C000084920460CF09EFB20460CF0AFFB284642
:1028D000FEF7D8F8204602B0BDE870400AF0C6B84E
:1028E000049FFF1F582F010070B5194C82B0342689
:1028F0000023012520460193009640230B223F210F
:1029000009F096F840230B222046009601953F21BE
:1029100009F010F92946204609F058FC29462046BE
:1029200009F04EFC20460F22442109F045FC092203
:10293000084920460CF066FB20460CF077FB284641
:10294000FFF7F4FA204602B0BDE870400AF08EB8F6
:10295000049FFF1F602F010008B581B2104809F0E5
:1029600035FC02210E4809F02BFC4F2121220C4896
:1029700009F022FC0B4B198849B903220A4908487F
:102980000CF040FB0648BDE808400CF04FBB044883
:102990000CF09CFB0248BDE808400CF047BB00BFB0
:1029A000049FFF1F5C9DFF1F6C2F010070B5194C29
:1029B00082B034260023012520460193009640234F
:1029C0000B223F2109F034F840230B2220460096C9
:1029D00001953F2109F0AEF82946204609F0F6FBA3
:1029E0002946204609F0ECFB20460F22472109F03A
:1029F000E3FB0822084920460CF004FB20460CF0BB
:102A000015FB2846FFF7A8FF204602B0BDE870403E
:102A10000AF02CB8049FFF1F702F010010B581B27F
:102A2000124C134809F0D2FB0221114809F0C8FBEF
:102A3000238821226BB94F210D4809F0BDFB0322E9
:102A40000C490B480CF0DEFA0948BDE810400CF0C8
:102A5000EDBA5A21064809F0AFFB218804480CF072
:102A600035FB0348BDE810400CF0E0BAC09DFF1FE5
:102A7000049FFF1F7C2F010070B5194C82B03426D3
:102A80000023012520460193009640230B223F217D
:102A900008F0CEFF40230B222046009601953F21EF
:102AA00009F048F82946204609F090FB29462046BF
:102AB00009F086FB20460F22512109F07DFB0522FB
:102AC000084920460CF09EFA20460CF0AFFA284642
:102AD000FFF7A4FF204602B0BDE8704009F0C6BF72
:102AE000049FFF1F582F010010B581B21748184CE2
:102AF00009F06CFB0221154809F062FB21224C21F0
:102B0000124809F059FB23884BB9032211490F4899
:102B10000CF078FA0D48BDE810400CF087BA02229C
:102B20000D490A480CF06EFA08480CF07FFA212291
:102B30006521064809F040FB218804480CF0C6FADC
:102B40000248BDE810400CF071BA00BF049FFF1F9F
:102B5000D49DFF1F7C2F0100802F010070B5194C00
:102B600082B034260023012520460193009640239D
:102B70000B223F2108F05CFF40230B2220460096E9
:102B800001953F2108F0D6FF2946204609F01EFB9B
:102B90002946204609F014FB20460F22442109F063
:102BA0000BFB0922084920460CF02CFA20460CF0B9
:102BB0003DFA2846FFF798FF204602B0BDE8704076
:102BC00009F054BF049FFF1F842F010010B581B28C
:102BD000124C134809F0FAFA0221114809F0F0FAF0
:102BE000238821226BB94F210D4809F0E5FA032211
:102BF0000C490B480CF006FA0948BDE810400CF0EF
:102C000015BA5A21064809F0D7FA218804480CF071
:102C10005DFA0348BDE810400CF008BA689DFF1F3C
:102C2000049FFF1F7C2F010070B5194C82B0342621
:102C30000023012520460193009640230B223F21CB
:102C400008F0F6FE40230B222046009601953F2116
:102C500008F070FF2946204609F0B8FA29462046B8
:102C600009F0AEFA20460F22482109F0A5FA082201
:102C7000084920460CF0C6F920460CF0D7F9284642
:102C8000FFF7A4FF204602B0BDE8704009F0EEBE99
:102C9000049FFF1F902F010010B50C4681B2194808
:102CA00009F094FA0221174809F08AFA21225021EA
:102CB000144809F081FA002C4FF0010214DB12498C
:102CC00010480CF09FF90F480CF0B0F95D2121225B
:102CD0000C4809F071FA21460A480CF0F7F9094846
:102CE000BDE810400CF0A2B9084906480CF08AF97A
:102CF00004480CF09BF95D212122024809F05CFA9E
:102D00006142E9E7049FFF1F9C2F0100A02F0100F3
:102D10000CB42DE9F04184B00AAC0646294814F8F9
:102D2000045B884609F000FD0121264809F048FAB5
:102D30000121244809F04AFA00221146214809F0ED
:102D40003BFA30460EF09CFB314602461D480CF023
:102D500059F91C480CF06AF9092201238DE80C008E
:102D600000217F23174808F095FE0394EDB16F1EF4
:102D7000FFB2013704EB87070C25043454F8046CC8
:102D8000104803942AB2002109F016FA30460EF0DA
:102D900077FB314602460B480CF034F909480CF039
:102DA00045F90935BC42ADB2E7D140460121FDF7F6
:102DB00015FE044809F05AFE04B0BDE8F04102B027
:102DC000704700BF049FFF1F30B52B4D0FCD8DB056
:102DD00006AC0FC495E8030044F8040B23202180BF
:102DE0000AF0BCF840F6B833984212DC234B40F6A8
:102DF000F50219889B78ADF8251090428DF82730A0
:102E00000EDC1F4B1A889B78ADF829208DF82B30EB
:102E10001EE01C4B1A889B78ADF825208DF82730D2
:102E2000194A00EB400000EB001382FB0320DB1784
:102E3000C3EB60200DF0AEFA14490DF0FFFA0DF16E
:102E40002903012203210AF03BFA56238DF82C3086
:102E50000F4B10481978104D104C114A114B04902B
:102E60000192009306A8039502940F4B0622FFF7E8
:102E70004FFF0DB030BD00BFF02F0100A42F0100A7
:102E8000A82F0100EC2F0100976A3E2BCDCCCC3D42
:102E90003289FF1FBC2F0100C82F0100D42F010071
:102EA000DC2F0100E42F0100B02F010030B50A4BE8
:102EB0000A4D19780A4C0B480B4A0C4B87B002900C
:102EC0000192009304950394094B0A480622FFF7E8
:102ED0001FFF07B030BD00BF948DFF1F24300100DD
:102EE000303001003C300100483001005430010016
:102EF000083001001430010010B586B0084C0948B4
:102F000009490A4A0A4B03900291019200930494E2
:102F1000084B09480622FF21FFF7FAFE06B010BD54
:102F2000902F01007C30010088300100702F0100DB
:102F300090300100603001006C30010010B586B0A7
:102F4000084C094809490A4A0A4B03900291019228
:102F500000930494084B09480622FF21FFF7D8FE8E
:102F600006B010BDB4300100C0300100CC3001000B
:102F7000D4300100842F01009C300100A8300100F2
:102F800000B585B008480949094A0A4B03900291E7
:102F9000019200930848094B0522FF21FFF7B8FE74
:102FA00005B05DF804FB00BFE8300100F43001001B
:102FB000FC30010004310100CC300100E0300100A0
:102FC00010B581B22048214C09F000F902211E48B9
:102FD00009F0F6F8212250211B4809F0EDF823886A
:102FE0000B2B4FF0010218DC194917480CF00AF8B6
:102FF00015480CF01BF821225D21134809F0DCF87C
:10300000218811480C390029B8BF49420CF05EF8FC
:103010000D48BDE810400CF009B80E490A480BF005
:10302000F1FF09480CF002F821225D21064809F061
:10303000C3F8218804480C390CF048F80248BDE870
:1030400010400BF0F3BF00BF049FFF1FAC9DFF1F9C
:10305000A02F01009C2F010070B5194C82B03426BE
:103060000023012520460193009640230B223F2197
:1030700008F0DEFC40230B222046009601953F21FC
:1030800008F058FD2946204609F0A0F829462046B8
:1030900009F096F820460F22442109F08DF8092204
:1030A000084920460BF0AEFF20460BF0BFFF284634
:1030B000FFF786FF204602B0BDE8704009F0D6BC9D
:1030C000049FFF1FB02F010010B581B22048214C92
:1030D00009F07CF802211E4809F072F821225021E3
:1030E0001B4809F069F82388022B4FF0010218DC15
:1030F000194917480BF086FF15480BF097FF21225E
:103100005D21134809F058F8218811480339002936
:10311000B8BF49420BF0DAFF0D48BDE810400BF094
:1031200085BF0E490A480BF06DFF09480BF07EFF82
:1031300021225D21064809F03FF82188044803391F
:103140000BF0C4FF0248BDE810400BF06FBF00BF9A
:10315000049FFF1FB49EFF1FA02F01009C2F0100A2
:1031600070B5194C82B03426002301252046019306
:10317000009640230B223F2108F05AFC40230B22EB
:103180002046009601953F2108F0D4FC29462046B0
:1031900009F01CF82946204609F012F820460F22B3
:1031A0004D2109F009F80622084920460BF02AFFB4
:1031B00020460BF03BFF2846FFF786FF204602B073
:1031C000BDE8704009F052BC049FFF1FE42F0100CE
:1031D00000B5324B1B78013B85B0052B0AD8DFE8E0
:1031E00003F00C21364B54032D492E4B5A2001225B
:1031F00008701A7005B05DF804FB01232A4A1946CD
:1032000018461370FDF7EAFB284809F02FFC284AFE
:10321000284B12680192019A1A60FFF71DFF05B052
:103220005DF804FB0123244A194602201370FDF7C0
:10323000D5FB1E4809F01AFC1D4A1E4B126802926B
:10324000029A1A60FFF78CFF05B05DF804FB0123BA
:103250001A4A194603201370FDF7C0FB134809F002
:1032600005FC134A134B12680392039A1A60FFF786
:103270003BFB05B05DF804FB09490A4B0A2001221B
:1032800008701A7005B05DF804FB0549054B502025
:10329000012208701A7005B05DF804FB3289FF1F27
:1032A000149EFF1F588CFF1FAA9EFF1F049FFF1F25
:1032B000409FFF1F409EFF1FB49DFF1FF59DFF1FF6
:1032C00008B581B20D4808F081FF02210B4808F0D3
:1032D00077FF21224F21094808F06EFF084B1B8819
:1032E0004BB90849032205480BF08CFE0348BDE8A2
:1032F00008400BF09BBE02220349F4E7049FFF1F26
:103300001A9EFF1F7C2F01000C31010070B5194C73
:1033100082B03426002301252046019300964023E5
:103320000B223F2108F084FB40230B22204600960D
:1033300001953F2108F0FEFB2946204608F046FF94
:103340002946204608F03CFF20460F22442108F081
:1033500033FF0922084920460BF054FE20460BF0AB
:1033600065FE2846FFF7ACFF204602B0BDE870407E
:1033700009F07CBB049FFF1F9030010008B581B2AB
:103380000D4808F023FF02210B4808F019FF212205
:103390004F21094808F010FF084B1B88032243B156
:1033A000074905480BF02EFE0348BDE808400BF026
:1033B0003DBE0449F5E700BF049FFF1FFE9DFF1FB0
:1033C000143101001031010070B5194C82B034265F
:1033D0000023012520460193009640230B223F2124
:1033E00008F026FB40230B222046009601953F2142
:1033F00008F0A0FB2946204608F0E8FE29462046B2
:1034000008F0DEFE20460F22442108F0D5FE0922F6
:10341000084920460BF0F6FD20460BF007FE284633
:10342000FFF7ACFF204602B0BDE8704009F01EBBBC
:10343000049FFF1FE830010000B53A4B1B78013BA9
:1034400087B0042B16D8DFE803F0182D425703008D
:103450000123354A194605201370FDF7BFFA33489A
:1034600009F004FB324A334B12680592059A1A6040
:10347000FFF7AAFF07B05DF804FB01232E4A1946A7
:1034800018461370FDF7AAFA284809F0EFFA284AFF
:10349000284B12680192019A1A60FFF7EDFA07B003
:1034A0005DF804FB0123254A194602201370FDF73D
:1034B00095FA1E4809F0DAFA1D4A1E4B126802926C
:1034C000029A1A60FFF768F907B05DF804FB012360
:1034D0001B4A194603201370FDF780FA134809F0C0
:1034E000C5FA134A134B12680392039A1A60FFF746
:1034F000C3F907B05DF804FB0123124A1946042002
:103500001370FDF76BFA094809F0B0FA084A094B45
:1035100012680492049A1A60FFF776F907B05DF812
:1035200004FB00BF488AFF1FE19EFF1F049FFF1F8F
:10353000409FFF1F409EFF1F369EFF1F089EFF1FDC
:10354000E49DFF1FE09EFF1F08B581B20D4808F003
:103550003DFE02210B4808F033FE21224F2109488D
:1035600008F02AFE084B1B88032243B90749054887
:103570000BF048FD0348BDE808400BF057BD044977
:10358000F5E700BF049FFF1FCA9DFF1F1C3101000C
:103590001831010070B5194C82B034260023012582
:1035A00020460193009640230B223F2108F040FA69
:1035B00040230B222046009601953F2108F0BAFADD
:1035C0002946204608F002FE2946204608F0F8FD6C
:1035D00020460F22442108F0EFFD09220849204629
:1035E0000BF010FD20460BF021FD2846FFF7ACFF45
:1035F000204602B0BDE8704009F038BA049FFF1FB2
:103600002031010000B5444B1B78013B87B0052BEE
:1036100016D8DFE803F0182D42576C0301233F4A08
:10362000194606201370FDF7D9F93D4809F01EFA36
:103630003C4A3D4B12680592059A1A60FFF7AAFFB3
:1036400007B05DF804FB0123384A19461846137089
:10365000FDF7C4F9324809F009FA324A324B1268D0
:103660000092009A1A60FFF75DF807B05DF804FB5E
:1036700001232F4A194602201370FDF7AFF928489D
:1036800009F0F4F9274A284B12680192019A1A604E
:10369000FFF748F807B05DF804FB254B0222012133
:1036A00003201A70FDF79AF91D4809F0DFF91D4A49
:1036B0001D4B12680292029A1A60FFF733F807B0A6
:1036C0005DF804FB1A4B0322012104201A70FDF758
:1036D00085F9134809F0CAF9124A134B126803928C
:1036E000039A1A60FFF71EF807B05DF804FB104B51
:1036F0000422012105201A70FDF770F9084809F02D
:10370000B5F9084A084B12680492049A1A60FFF748
:1037100009F807B05DF804FB948DFF1F589EFF1F4A
:10372000049FFF1F409FFF1F409EFF1F459EFF1FDE
:10373000E49EFF1F08B581B2154808F047FD02213D
:10374000134808F03DFD4F212122114808F034FDB7
:10375000104B198849B9104903220D480BF052FC4F
:103760000B48BDE808400BF061BC09480BF0AEFC0B
:1037700007480BF05BFC28226921054808F01CFD76
:103780000121034808F01CFD02220449E5E700BFBF
:10379000049FFF1FBC9EFF1F7C2F01002C310100E6
:1037A00070B5194C82B034260023012520460193C0
:1037B000009640230B223F2108F03AF940230B22C8
:1037C0002046009601953F2108F0B4F9294620468D
:1037D00008F0FCFC2946204608F0F2FC20460F22A7
:1037E000452108F0E9FC0922084920460BF00AFCB3
:1037F00020460BF01BFC2846FFF79CFF204602B03A
:10380000BDE8704009F032B9049FFF1F7C30010011
:1038100008B581B2154808F0D9FC0221134808F018
:10382000CFFC4F212122114808F0C6FC104B19880B
:1038300049B9104903220D480BF0E4FB0B48BDE8E1
:1038400008400BF0F3BB09480BF040FC07480BF0B5
:10385000EDFB28226921054808F0AEFC0121034850
:1038600008F0AEFC02220449E5E700BF049FFF1FF9
:10387000DE9EFF1F7C2F01002C31010070B5194C1A
:1038800082B0342600230125204601930096402370
:103890000B223F2108F0CCF840230B222046009653
:1038A00001953F2108F046F92946204608F08EFC94
:1038B0002946204608F084FC20460F22472108F0C4
:1038C0007BFC0822084920460BF09CFB20460BF0AD
:1038D000ADFB2846FFF79CFF204602B0BDE87040D4
:1038E00009F0C4B8049FFF1FC030010030B5544830
:1038F00083B008F019FF0121514808F061FC012153
:103900004F4808F063FC022219214D4808F054FC8E
:103910000B224C494A480BF075FB49480BF086FBDB
:1039200014220021464808F047FC03224649444837
:103930000BF068FB424801240BF078FB11228DE864
:103940001400782319213E4808F0A4F81325192300
:103950001946009512223A48019408F09BF8782302
:103960001946009512223648019408F093F81D225A
:103970008DE8140078231921314808F08BF81C25B4
:103980001923194600951B222D48019408F082F84E
:103990007823194600951B222948019408F07AF8EB
:1039A00023220021264808F007FC03222749244847
:1039B0000BF028FB22480BF039FB28251923194668
:1039C00024221F480194009508F064F878231946D2
:1039D0002422019400951A4808F05CF81C4A1D4BFB
:1039E00011681B681C4A5B1A5C2B12881DDC511A7B
:1039F0005C2202FB01F292FBF3F31B33174A1048DF
:103A0000136001241BB21A2219468DE814001422F7
:103A100008F040F8124B20461C70FCF7F5FF0848F0
:103A200003B0BDE8304009F021B8521A02EB42025F
:103A3000C2EB4212234492FBF3F31B33DEE700BFD9
:103A4000049FFF1F303101003C3101004031010073
:103A5000F48DFF1F408CFF1FF49EFF1F609DFF1F12
:103A6000909EFF1FF0B58548854E864D83B008F0C7
:103A70005BFE0121814808F0A3FB01217F4808F08B
:103A8000A5FB022219217D4808F096FB0A227E49F7
:103A90007A480BF0B7FA79480BF0C8FA14220021E3
:103AA000764808F089FB0322784974480BF0AAFA9B
:103AB000724801240BF0BAFA11228DE81400782321
:103AC00019216E4807F0E6FF1327192319460097BE
:103AD00012226A48019407F0DDFF78231946009707
:103AE00012226648019407F0D5FF1D228DE81400CC
:103AF00078231921614807F0CDFF1C2719231946A7
:103B000000971B225D48019407F0C4FF78231946F3
:103B100000971B225948019407F0BCFF2322002183
:103B2000564808F049FB0322594954480BF06AFAF9
:103B300052480BF07BFA28271923194600972422B4
:103B40004E48019407F0A6FF7823194600972422D7
:103B50004A48019407F09EFF32220021474808F0AE
:103B60002BFB03224B4945480BF04CFA43480BF022
:103B70005DFA2F228DE81400782319213F4807F0C1
:103B800089FF312719231946009730223B480194B9
:103B900007F080FF782319460097302237480194B8
:103BA00007F078FF3C228DE8140078231921334870
:103BB00007F070FF3B27192319463A222F4801943A
:103BC000009707F067FF782319463A22019400977F
:103BD0002A4807F05FFF31682B682F4A5B1A5C2B7D
:103BE000128839DD521A02EB4202C2EB4212234420
:103BF00092FBF3F31B33294A2048136001241BB2C4
:103C00001A2219468DE81400142207F043FF316888
:103C10002B682348234A04705B1A5C2B128823DC30
:103C2000511A5C2202FB01F292FBF3F31B331E4A92
:103C30001248136001241BB2392219468DE8140082
:103C4000322207F027FF2046FCF7DEFE0B4803B0C8
:103C5000BDE8F04008F00ABF511A5C2202FB01F2F5
:103C600092FBF3F31B33C6E7521A02EB4202C2EB9C
:103C70004212234492FBF3F31B33D8E7049FFF1F48
:103C8000E88DFF1F3C8BFF1F443101003C310100D8
:103C90004031010050310100349EFF1F609DFF1F25
:103CA000909EFF1FBC9DFF1FAC9EFF1FF0B5854877
:103CB000854E864D83B008F037FD0121814808F01C
:103CC0007FFA01217F4808F081FA022219217D48FC
:103CD00008F072FA0A227E497A480BF093F9794883
:103CE0000BF0A4F914220021764808F065FA0322AB
:103CF000784974480BF086F9724801240BF096F964
:103D000011228DE81400782319216E4807F0C2FEB5
:103D1000132719231946009712226A48019407F0C5
:103D2000B9FE78231946009712226648019407F0DD
:103D3000B1FE1D228DE8140078231921614807F097
:103D4000A9FE1C271923194600971B225D480194E0
:103D500007F0A0FE7823194600971B2259480194CA
:103D600007F098FE23220021564808F025FA032286
:103D7000594954480BF046F952480BF057F9282797
:103D800019231946009724224E48019407F082FE19
:103D900078231946009724224A48019407F07AFEB6
:103DA00032220021474808F007FA03224B494548D0
:103DB0000BF028F943480BF039F92F228DE8140055
:103DC000782319213F4807F065FE3127192319464A
:103DD000009730223B48019407F05CFE7823194697
:103DE000009730223748019407F054FE3C228DE8BA
:103DF000140078231921334807F04CFE3B27192380
:103E000019463A222F480194009707F043FE782381
:103E100019463A22019400972A4807F03BFE316880
:103E20002B682F4A5B1A5C2B128839DD521A02EB81
:103E30004202C2EB4212234492FBF3F31B33294AA2
:103E40002048136001241BB21A2219468DE8140081
:103E5000142207F01FFE31682B682348234A0470A0
:103E60005B1A5C2B128823DC511A5C2202FB01F2E4
:103E700092FBF3F31B331E4A1248136001241BB25A
:103E8000392219468DE81400322207F003FE20463D
:103E9000FCF7BAFD0B4803B0BDE8F04008F0E6BD02
:103EA000511A5C2202FB01F292FBF3F31B33C6E7CB
:103EB000521A02EB4202C2EB4212234492FBF3F38A
:103EC0001B33D8E7049FFF1F688AFF1FE48DFF1F85
:103ED000543101003C3101004031010050310100FA
:103EE000EC9DFF1F609DFF1F909EFF1FCC9EFF1F3C
:103EF000AC9EFF1FF0B58548854E864D83B008F017
:103F000013FC0121814808F05BF901217F4808F08A
:103F10005DF9022219217D4808F04EF910227E49F0
:103F20007A480BF06FF879480BF080F814220021E2
:103F3000764808F041F90322784974480BF062F89A
:103F4000724801240BF072F811228DE814007823D6
:103F500019216E4807F09EFD132719231946009773
:103F600012226A48019407F095FD782319460097BC
:103F700012226648019407F08DFD1D228DE8140081
:103F800078231921614807F085FD1C27192319465C
:103F900000971B225D48019407F07CFD78231946A9
:103FA00000971B225948019407F074FD2322002139
:103FB000564808F001F90322594954480BF022F8F9
:103FC00052480BF033F8282719231946009724226A
:103FD0004E48019407F05EFD78231946009724228D
:103FE0004A48019407F056FD32220021474808F064
:103FF000E3F803224B4945480BF004F843480BF023
:1040000015F82F228DE81400782319213F4807F076
:1040100041FD312719231946009730223B4801946E
:1040200007F038FD7823194600973022374801946D
:1040300007F030FD3C228DE8140078231921334825
:1040400007F028FD3B27192319463A222F480194EF
:10405000009707F01FFD782319463A220194009734
:104060002A4807F017FD31682B682F4A5B1A5C2B32
:10407000128839DD521A02EB4202C2EB421223448B
:1040800092FBF3F31B33294A2048136001241BB22F
:104090001A2219468DE81400142207F0FBFC31683F
:1040A0002B682348234A04705B1A5C2B128823DC9C
:1040B000511A5C2202FB01F292FBF3F31B331E4AFE
:1040C0001248136001241BB2392219468DE81400EE
:1040D000322207F0DFFC2046FCF796FC0B4803B0C9
:1040E000BDE8F04008F0C2BC511A5C2202FB01F2AC
:1040F00092FBF3F31B33C6E7521A02EB4202C2EB08
:104100004212234492FBF3F31B33D8E7049FFF1FB3
:10411000FC8DFF1F5C8AFF1F603101003C310100F4
:104120004031010050310100969DFF1F609DFF1F2F
:10413000909EFF1F4E9EFF1FAC9EFF1FF0B585484F
:10414000854E864D83B008F0EFFA0121814808F0D2
:1041500037F801217F4808F039F8022219217D48FB
:1041600008F02AF806227E497A480AF04BFF79487F
:104170000AF05CFF14220021764808F01DF80322A3
:10418000784974480AF03EFF724801240AF04EFF55
:1041900011228DE81400782319216E4807F07AFC6B
:1041A000132719231946009712226A48019407F031
:1041B00071FC78231946009712226648019407F093
:1041C00069FC1D228DE8140078231921614807F04D
:1041D00061FC1C271923194600971B225D48019496
:1041E00007F058FC7823194600971B225948019480
:1041F00007F050FC23220021564807F0DDFF032280
:10420000594954480AF0FEFE52480AF00FFF282789
:1042100019231946009724224E48019407F03AFCCE
:1042200078231946009724224A48019407F032FC6B
:1042300032220021474807F0BFFF03224B4945487F
:104240000AF0E0FE43480AF0F1FE2F228DE8140048
:10425000782319213F4807F01DFC312719231946FF
:10426000009730223B48019407F014FC782319464C
:10427000009730223748019407F00CFC3C228DE86F
:10428000140078231921334807F004FC3B27192335
:1042900019463A222F480194009707F0FBFB782338
:1042A00019463A22019400972A4807F0F3FB316837
:1042B0002B682F4A5B1A5C2B128839DD521A02EBED
:1042C0004202C2EB4212234492FBF3F31B33294A0E
:1042D0002048136001241BB21A2219468DE81400ED
:1042E000142207F0D7FB31682B682348234A047057
:1042F0005B1A5C2B128823DC511A5C2202FB01F250
:1043000092FBF3F31B331E4A1248136001241BB2C5
:10431000392219468DE81400322207F0BBFB2046F3
:10432000FCF772FB0B4803B0BDE8F04008F09EBB01
:10433000511A5C2202FB01F292FBF3F31B33C6E736
:10434000521A02EB4202C2EB4212234492FBF3F3F5
:104350001B33D8E7049FFF1F389EFF1F588AFF1F9B
:10436000743101003C310100403101005031010045
:104370001E9EFF1F609DFF1F909EFF1FEC9EFF1F54
:10438000AC9EFF1F10B581B219481A4C07F01EFFF2
:104390000221174807F014FF4F212122144807F08B
:1043A0000BFF21880B2910D90C2917D001221249A3
:1043B0000F480AF027FE21880D480C390AF086FEC6
:1043C0000B48BDE810400AF031BE0C3908480AF02D
:1043D0007DFE0748BDE810400AF028BE03220749C9
:1043E00003480AF00FFE0248BDE810400AF01EBE66
:1043F000049FFF1FCE9EFF1F9C2F01007C310100F8
:1044000070B5194C82B03426002301252046019353
:10441000009640230B223F2107F00AFB40230B228A
:104420002046009601953F2107F084FB294620464F
:1044300007F0CCFE2946204607F0C2FE20460F2298
:10444000442107F0B9FE0922084920460AF0DAFDA6
:1044500020460AF0EBFD2846FFF794FF204602B005
:10446000BDE8704008F002BB049FFF1FB43001009C
:1044700008B581B20F4807F0A9FE02210D4807F0E8
:104480009FFE21224F210B4807F096FE0A4B1A8807
:10449000012A0CD0022A0EBF084909490322054807
:1044A0000AF0B0FD0348BDE808400AF0BFBD022293
:1044B0000449F4E7049FFF1F289EFF1F803101007D
:1044C0007C2F01000C31010070B5194C82B03426EC
:1044D0000023012520460193009640230B223F2113
:1044E00007F0A6FA40230B222046009601953F21B3
:1044F00007F020FB2946204607F068FE29462046A3
:1045000007F05EFE20460F22472107F055FE0822E5
:10451000084920460AF076FD20460AF087FD284625
:10452000FFF7A6FF204602B0BDE8704008F09EBA33
:10453000049FFF1F9C30010008B581B2224807F09C
:1045400045FE0221204807F03BFE21224F211E4854
:1045500007F032FE1D4B1B88042B33D8DFE803F035
:10456000121A222A030021225321174807F024FEA1
:104570001749022214480AF045FD1348BDE80840D7
:104580000AF054BD21224F210F4807F015FE0322E7
:104590001049EFE7212253210B4807F00DFE0222BC
:1045A0000D49E7E721225321074807F005FE0222C3
:1045B0000A49DFE721225321034807F0FDFD0222CB
:1045C0000749D7E708BD00BF049FFF1FCC9DFF1F11
:1045D000903101007C2F01008431010088310100FD
:1045E0008C31010070B5194C82B0342600230125AE
:1045F00020460193009640230B223F2107F018FA32
:1046000040230B222046009601953F2107F092FAA5
:104610002946204607F0DAFD2946204607F0D0FD5E
:1046200020460F22442107F0C7FD092208492046F1
:104630000AF0E8FC20460AF0F9FC2846FFF77CFF68
:10464000204602B0BDE8704008F010BA049FFF1F7A
:10465000D430010000B53E4B1B78013B87B0052BE1
:1046600016D8DFE803F0182D425760030123394ABA
:10467000194606201370FCF7B1F9374808F0F6F92F
:10468000364A374B12680592059A1A60FFF7B8FE52
:1046900007B05DF804FB0123324A1946184613702F
:1046A000FCF79CF92C4808F0E1F92C4A2C4B1268D5
:1046B0000192019A1A60FFF707FF07B05DF804FB4B
:1046C0000123294A194602201370FCF787F9224872
:1046D00008F0CCF9214A224B12680292029A1A6021
:1046E000FEF73CFA07B05DF804FB01231F4A1946A8
:1046F00003201370FCF772F9174808F0B7F9174A4E
:10470000174B12680392039A1A60FFF76BFF07B00A
:104710005DF804FB1649174B6E20012208701A70D1
:1047200007B05DF804FB0123134A194605201370F6
:10473000FCF754F9084808F099F9084A084B126840
:104740000492049A1A60FFF799F807B05DF804FB29
:10475000548AFF1F9E9DFF1F049FFF1F409FFF1F46
:10476000409EFF1F4C9EFF1F589DFF1F649DFF1F13
:10477000149EFF1F588CFF1FC99DFF1F10B5334C9F
:10478000334807F0D1FF237803BB01213048314C77
:1047900007F01CFD06212E4807F012FD2388092B87
:1047A0004ED9632B4FF00A0294BF1F2111462848AF
:1047B00007F002FD218826480AF088FC24480AF008
:1047C00035FC2348BDE8104008F050B9FDF700F86B
:1047D0002378012BD9D9022B4FF001011C4817D0A7
:1047E00007F0F4FC06211A4807F0EAFC0A221146F9
:1047F000174807F0E1FC0322174915480AF002FCAC
:1048000013480AF013FC1248BDE8104008F02EB916
:1048100007F0DCFC06210E4807F0D2FC0A22114604
:104820000B4807F0C9FC03220C4909480AF0EAFBCF
:1048300007480AF0FBFB0648BDE8104008F016B92F
:104840000A223021024807F0B7FCB3E7669DFF1F3C
:10485000049FFF1F6C9EFF1F9831010094310100DF
:1048600008B581B2394807F0B1FC0221374807F09A
:10487000A7FC374B1B884BB1013B092B65D8DFE800
:1048800003F01C242C343C444C545C1421224F2152
:104890002E4807F091FC2F4903222C480AF0B2FB66
:1048A0002A48BDE808400AF0C1BB2122532127480D
:1048B00007F082FC02222849EFE7212253212348F6
:1048C00007F07AFC02222549E7E7212253211F48FD
:1048D00007F072FC02222249DFE7212253211B4804
:1048E00007F06AFC02221F49D7E72122532117480B
:1048F00007F062FC02221C49CFE721224F21134816
:1049000007F05AFC03221949C7E721224F210F481B
:1049100007F052FC03221649BFE721224F210B4822
:1049200007F04AFC03221349B7E721224F21074829
:1049300007F042FC03221049AFE72122532103482C
:1049400007F03AFC02220D49A7E708BD049FFF1FAC
:10495000989EFF1F7C2F0100B831010084310100B7
:104960009C310100A0310100A4310100A8310100F7
:10497000AC310100B0310100B43101008C310100D3
:1049800070B5194C82B034260023012520460193CE
:10499000009640230B223F2107F04AF840230B22C8
:1049A0002046009601953F2107F0C4F8294620468D
:1049B00007F00CFC2946204607F002FC20460F2297
:1049C000442107F0F9FB0922084920460AF01AFBA6
:1049D00020460AF02BFB2846FFF742FF204602B094
:1049E000BDE8704008F042B8049FFF1F603001002E
:1049F00008B581B2414807F0E9FB02213F4807F0C2
:104A0000DFFB3F4B1B880C2B77D8DFE803F0161E2B
:104A1000262E363E464E565E666E070021225321F4
:104A2000364807F0C9FB3749022234480AF0EAFA4F
:104A30003248BDE808400AF0F9BA212253212F4834
:104A400007F0BAFB02223049EFE7212253212B481D
:104A500007F0B2FB02222D49E7E721225321274824
:104A600007F0AAFB02222A49DFE72122532123482B
:104A700007F0A2FB02222749D7E721224F211F4836
:104A800007F09AFB03222449CFE7212253211B4838
:104A900007F092FB02222149C7E721225321174840
:104AA00007F08AFB02221E49BFE721225321134847
:104AB00007F082FB02221B49B7E7212253210F484E
:104AC00007F07AFB02221849AFE7212253210B4855
:104AD00007F072FB02221549A7E72122532107485C
:104AE00007F06AFB022212499FE721225321034863
:104AF00007F062FB02220F4997E708BD049FFF1FE2
:104B0000AA9DFF1FEC310100BC310100C031010042
:104B1000C4310100C8310100CC310100D0310100A5
:104B2000D4310100D8310100DC310100E031010055
:104B3000E4310100E831010070B5194C82B034262F
:104B40000023012520460193009640230B223F219C
:104B500006F06EFF40230B222046009601953F2170
:104B600006F0E8FF2946204607F030FB294620469C
:104B700007F026FB20460F22502107F01DFB0522DF
:104B8000084920460AF03EFA20460AF04FFA284625
:104B9000FFF72EFF204602B0BDE8704007F066BF69
:104BA000049FFF1F8830010000B5444B1B78013B78
:104BB00087B0052B16D8DFE803F0182D42576C0399
:104BC00001233F4A194606201370FBF707FF3D48B3
:104BD00007F04CFF3C4A3D4B12680592059A1A605B
:104BE000FEF722F807B05DF804FB0123384A1946A6
:104BF00018461370FBF7F2FE324807F037FF324ACF
:104C0000324B12680092009A1A60FFF7B9FE07B0A3
:104C10005DF804FB01232F4A194602201370FBF7AD
:104C2000DDFE284807F022FF274A284B1268019230
:104C3000019A1A60FEF76AFB07B05DF804FB0123D6
:104C4000254A194603201370FBF7C8FE1D4807F0DC
:104C50000DFF1D4A1D4B12680292029A1A60FDF761
:104C6000A5FE07B05DF804FB01231C4A1946042089
:104C70001370FBF7B3FE134807F0F8FE124A134B0C
:104C800012680392039A1A60FFF756FF07B05DF8A7
:104C900004FB0123124A194605201370FBF79EFE00
:104CA000084807F0E3FE084A084B12680492049A89
:104CB0001A60FEF775FD07B05DF804FB648AFF1FFC
:104CC000F49DFF1F049FFF1F409FFF1F409EFF1F7B
:104CD0005A9DFF1FD49EFF1F949DFF1F2F9FFF1FF4
:104CE000BE9DFF1F2DE9F0430320ADF5257D08F0A3
:104CF000E5FEB0FA80F4042008F0E0FE002814BFBE
:104D000000210221640905200C4408F0D7FE002888
:104D100014BF0021042106200C4408F0CFFE9E4D54
:104D20009E4E2B68002814BF00210821214499427F
:104D3000316000F02D819A4C9A4B22680492049ABB
:104D40001A60236805939848059B0068944F9B1A46
:104D5000834220D9954B1A68914216D03A6807923F
:104D6000934ADDF81CE093481960C2F800E00AF0AD
:104D7000ADF990480AF05AF93B6806938E4A8F4B7A
:104D800006981060316801221A70012900F0E18054
:104D9000042900F0DE808A4F29603D78002D00F064
:104DA000CD80236882490B93864A0B9B0968126861
:104DB0007B485B1A93423FD9834E84488449854A95
:104DC000854D864CDFF864C2DFF864E2012333705E
:104DD000002303700B70137081488249824A2B7044
:104DE000237003700B701370804D814C8148824991
:104DF000824A2B70237003700B701370804D814CAE
:104E000081488249824A8CF800303B708EF800302D
:104E10002B70237003700B701370AE217D48674CAC
:104E200007F08AFC002333702378002B40F00481C4
:104E30000DF5257DBDE8F083022D00F03381012DB5
:104E400000F0E681642D00F089810A2D00F02A82AD
:104E50000B2D01F03B800C2D01F04781142D01F04A
:104E60005482152D00F0B883162D01F0B7841E2D45
:104E700001F0BE861F2D01F06487202D02F07480A2
:104E8000282D02F0D181292D02F078822A2D02F0FE
:104E900085833C2D02F073843D2D02F02185502D39
:104EA00002F08C865A2D02F0D3866E2DC0D1464E6C
:104EB0003378002B43F078804A4D2A78002A02F09C
:104EC00076872368DFF86C818E93534A8E9BD8F8DF
:104ED000001012685B1A934211D9504B1A78012ABC
:104EE0000CBF002201221A701878FDF797FD49487F
:104EF00007F0BCFD23688F938F9BC8F800302F4AC2
:104F00001378002B94D0294B1B680021013B1170B2
:104F1000072B8DD801A252F823F000BFF9940000AE
:104F2000CB940000314E000095940000314E0000FB
:104F3000314E0000314E000067940000224E33785D
:104F4000002B7FF46AAF1D4C2378002B3FF470AF29
:104F500072E023681848324A08930668089B106874
:104F60000F4A9B1B83427FF616AF13682D480993A7
:104F70002D4E099B07683668DB1BB3427FF60BAFEB
:104F800013680A930A9A0D4B026001221A7002E715
:104F9000044B034C1A68D4E62C9EFF1FF09EFF1FA3
:104FA000409FFF1F9C9EFF1F608CFF1F949EFF1F52
:104FB000989DFF1F1094FF1F109EFF1FFC9DFF1F59
:104FC000149EFF1FF08DFF1F588CFF1F5A9DFF1F5F
:104FD000D49EFF1F949DFF1F4C9EFF1F589DFF1FD7
:104FE000649DFF1F369EFF1FC99DFF1F9E9DFF1FD3
:104FF000BE9DFF1FF49DFF1F459EFF1FE49EFF1FE8
:10500000589EFF1F089EFF1FE49DFF1FE09EFF1F8D
:10501000E19EFF1F049FFF1F908DFF1F909EFF1FAB
:10502000508AFF1F909DFF1FB48CFF1FAA9EFF1F79
:10503000F59DFF1F409EFF1F00232370FBF7A0FB81
:10504000B94ABA4BBA49BB4812781B78096800784C
:1050500002EB43034A1E03EB80030E2A3FF6E8AE41
:1050600001A151F822F000BF135500002B5500009C
:10507000314E0000DB540000314E0000314E000084
:10508000314E0000A1540000314E0000314E0000AE
:10509000314E0000314E0000314E0000314E000014
:1050A0009D540000A44E3378002B40F00287A34D9E
:1050B0002A6823680D93A2490D9B09689B1A8B42AD
:1050C00011D9A048A04901220023027026200B70AC
:1050D0003B703270FBF71EFD9C4B1988884202D052
:1050E0002620FBF70BFD9A4B1A78002A3FF4A0AE5E
:1050F00000221A70FBF744FB8B4A8C4B8C498D487D
:1051000012781B780968007802EB43034A1E03EB10
:1051100080030E2A3FF68CAE01A151F822F000BFA9
:105120005957000029570000314E0000E356000097
:10513000314E0000314E0000314E0000BD560000DF
:10514000314E00009F570000314E0000314E0000EC
:10515000314E0000314E00009D540000764E3378F1
:10516000002B41F0CC807B4D2B78002B40F0508100
:10517000DFF8F89199F80050002D01F05D81236867
:10518000DFF8EC812493744AD8F80010249B12684D
:105190005B1A9342714A117800D8C1B1704B1878EC
:1051A000012802F0D78001201870002941F0D6862E
:1051B00018786C4B013D53F82510FDF76DFD6A48DA
:1051C00007F054FC23682593259BC8F80030604AFB
:1051D0001378002B3FF42CAE554B1B680021013B8C
:1051E0001170072B3FF624AE01A252F823F000BF46
:1051F000275C0000E75B0000314E00009D5B000073
:10520000314E0000314E0000314E00004F5B000077
:10521000494E3378002B40F06287DFF8589199F8B7
:105220000000002800F0A8802368DFF84481129372
:10523000494A129BD8F8001012685B1A934210D9A1
:10524000474B1A78012A0CBF002001201870FDF787
:10525000B7FE454807F00AFC23681393139BC8F870
:1052600000303B4A1378002B3FF4E2AD304B1B6813
:105270000021013B1170072B3FF6DAAD01A252F875
:1052800023F000BF3D5900000D590000314E0000D1
:10529000D7580000314E0000314E0000314E000062
:1052A000A7580000244E3378002B40F08D812368EE
:1052B000DFF8BC802E93284A2E9BD8F80010126885
:1052C0005B1A934210D9264B1A78012A0CBF002092
:1052D00001201870FBF798FB234807F0C7FB2368F1
:1052E0002F932F9BC8F80030194A1378002B3FF4F6
:1052F0009FAD0F4B1B680021013B1170072B3FF640
:1053000097AD01A252F823F07158000069580000CF
:10531000314E000033580000314E0000314E000085
:10532000314E0000FF570000D59EFF1F309FFF1F2A
:10533000949EFF1F319FFF1F588CFF1FB09DFF1FC2
:10534000EC8DFF1F9D9DFF1F669DFF1F6C9EFF1F25
:10535000FC9DFF1F459EFF1F908DFF1FFC9EFF1FA2
:10536000909EFF1F448CFF1F049FFF1FE49EFF1FA2
:10537000409EFF1FAA9EFF1FDFF8349399F800306C
:10538000002B40F0E580DFF82C9399F80020002AEC
:1053900001F050812268DFF820831A92B1491A9AED
:1053A000D8F800000968121A8A4211D9AE4A117859
:1053B00001290BBF1846012013701070FCF7B6FDD1
:1053C000AA4807F053FB23681B931B9BC8F80030C7
:1053D000A74A1378002B3FF42BADA64B1B68002186
:1053E000013B1170072B3FF623AD01A252F823F0C9
:1053F000475E00000B5E0000314E00007D5E000045
:10540000314E0000314E0000314E0000DB5D0000E7
:105410002368DFF8A4822093924AD8F80010209BDA
:1054200012685B1A9342944A117800D8B1B18E4B3E
:105430001878012801F08E8501201870002941F0AC
:10544000AB8318788D4B1968FDF726FC874807F069
:105450000DFB23682193219BC8F80030844A137800
:10546000002B3FF4E5AC834B1B680021013B11701E
:10547000072B3FF6DDAC01A252F823F0495A000099
:10548000155A0000314E0000DD590000314E000079
:10549000314E0000314E00007359000008F034FE18
:1054A000774B78491C78784B784A09881B881268B2
:1054B0000B44002C01F08C80B2EB630F81F28A86E2
:1054C000734B1B78002B01F03284AF21674807F043
:1054D00033F901233B703370AAE4002B01F0A6805E
:1054E000013B6C4A32F813304BB16B4D6B486C4941
:1054F0006C4A2B800123002505700B701370AF21BF
:105500005A4807F019F9012302223A7023703370C8
:105510008EE463B901232370AF21544807F00CF9DE
:10552000022201233A70337082E4002BF4D0013B55
:10553000584A32F81330002BEED0574C5748584990
:10554000584A23800123002404700B701370E3E792
:105550002368DFF864811693424A169BD8F800103E
:1055600012685B1A93420FD93F4B1A78012A18BF71
:1055700001201870FDF7A8FD3C4807F077FA236872
:105580001793179BC8F80030394A1378002B3FF463
:105590004FAC384B1B680021013B1170072B3FF6C5
:1055A00047AC01A252F823F0195B0000E95A000051
:1055B000314E0000B35A0000314E0000314E000061
:1055C000314E0000835A0000FEF7B8FD364A012133
:1055D0000023117033706AE62368DFF8DC803A93A9
:1055E000204A3A9BD8F8001012685B1A934219D9E6
:1055F0001D4A1E481378012B0CBF00230123137092
:105600002A4A0193B2F900301A2219460092142254
:1056100006F040FA154807F029FA23683B933B9BB4
:10562000C8F80030124A1378002B3FF401AC114B3C
:105630001B680021013B1170072B3FF6F9AB01A25B
:1056400052F823F05B5D0000355D0000314E000034
:10565000B55C0000314E0000314E0000314E0000BC
:10566000735C0000908DFF1F909EFF1F049FFF1F23
:10567000FC9DFF1F949EFF1FFC9EFF1F048BFF1FBE
:105680009C9DFF1F969DFF1F4E9EFF1FC49DFF1FE9
:10569000BF9DFF1F789DFF1F6C9EFF1FF69DFF1F84
:1056A0009D9DFF1F669DFF1F749DFF1F609DFF1F37
:1056B000B49DFF1FF59DFF1F409EFF1FBA4C23782E
:1056C000012B41F253862620FBF724FAB74B1988A9
:1056D000884202D02620FBF711FA00232370FFF73F
:1056E000A7BB002B01F04185013BB14A32F81360A2
:1056F00096B1AE4BAF48B049AB4A1E80002701239C
:10570000077026200B701370FBF704FA864203D053
:1057100031462620FBF7F2F9FFF730F823681093A3
:10572000109B2B60FFF784BB83B1013BA04A32F88A
:1057300013305BB19D4E9F489F499B4A33800123A4
:10574000002606700B701370FFF718F823680F938C
:105750000F9B2B60FFF76CBB002B01F0F484013B27
:10576000934A32F8136096B1904B924892498E4A10
:105770001E8000270123077026200B701370FBF793
:10578000C9F9864203D031462620FBF7B7F9FEF768
:10579000F5FF23680E930E9B2B60FFF749BBFBF7C9
:1057A00069FD864806F0C0FF0121844806F00EFD21
:1057B0000221824806F004FD0F2223217F4806F0D3
:1057C000FBFC05227E497D4809F01CFC7B4809F062
:1057D0002DFC1E222321794806F0EEFC0522794992
:1057E000764809F00FFC754809F020FC734807F073
:1057F0003DF923681193119B2B60FFF719BB01231F
:1058000002203B703370FBF785F96F4B1988884293
:1058100002D00220FBF772F90420FBF77BF96B4BF7
:10582000198888423FF404AB0420FBF767F9FFF7BF
:10583000FFBA01233C22022033703A70FBF76AF969
:10584000614B1988884202D00220FBF757F90420E7
:10585000FBF760F95D4B198888423FF4E9AA042000
:10586000FBF74CF9FFF7E4BA0B233B70FFF7E0BA04
:1058700001231422022033703A70FBF74BF9524B8C
:105880001988884202D00220FBF738F90420FBF780
:1058900041F94E4B198888423FF4CAAA0420FBF70D
:1058A0002DF9FFF7C5BA0120FDF78AFB484B4348A5
:1058B00000241C7007F0DAF80E2089F80040FBF78E
:1058C00029F9444B198888423FF4B2AA0E20FBF70D
:1058D00015F9FFF7ADBA3F4D2B88172B3FF6A8AA55
:1058E0000020FDF76DFB2B88012003442B80FDF782
:1058F00067FB374B314800221A7007F0B7F823686E
:105900001593159BC8F80030FFF792BA0120FDF7F8
:1059100057FB2F4B294800241C7007F0A7F80E20D6
:1059200089F80040FBF7F6F82A4B198888423FF4C3
:105930007FAA0E20FBF7E2F8FFF77ABA254D2B88F5
:10594000002B3FF475AA0020FDF73AFB2B880120BD
:10595000013B2B80FDF734FB1D4B184800221A70C9
:1059600007F084F823681493149BC8F80030FFF7FD
:105970005FBA194C01202168FDF78EF9144B0F48CE
:1059800000261E7007F072F844202E70FBF7C2F854
:105990002168183188423FF44BAA89B24420FBF7B2
:1059A000ADF8FFF745BA00BF669DFF1F6C9EFF1F55
:1059B000789DFF1FF69DFF1F9D9DFF1F049FFF1FEA
:1059C000F0310100F83101001E9EFF1FEC9EFF1F09
:1059D000909EFF1FAC9DFF1F048BFF1FAE4D2968DB
:1059E00017293FF725AA0020FDF756F92B68013348
:1059F000194601202B60FDF74FF9A84BA84800225B
:105A00001A7007F033F823682393239BC8F80030FB
:105A1000FFF70EBAA04C01202168FDF73DF99F4B1E
:105A20009F4800261E7007F021F844202E70FBF7D7
:105A300071F82168183188423FF4FAA989B24420EC
:105A4000FBF75CF8FFF7F4B9934D296811F1170FD4
:105A5000FFF6EEA90020FDF71FF92B68013B194660
:105A600001202B60FDF718F98C4B8D4800221A702D
:105A700006F0FCFF23682293229BC8F80030FFF752
:105A8000D7B90120FDF720FB844B854800241C700A
:105A900006F0ECFF282089F80040FBF73BF8814B2B
:105AA000198888423FF4C4A92820FBF727F8FFF79C
:105AB000BFB97C4D2B88052B3FF6BAA90020FDF716
:105AC00003FB2B88012003442B80FDF7FDFA734B69
:105AD000734800221A7006F0C9FF23681993199BB6
:105AE000C8F80030FFF7A4B90120FDF7EDFA6B4BC1
:105AF0006B4800241C7006F0B9FF282089F800408C
:105B0000FBF708F8674B198888423FF491A92820D1
:105B1000FAF7F4FFFFF78CB9624D2B88002B3FF4A6
:105B200087A90020FDF7D0FA2B880120013B2B80AC
:105B3000FDF7CAFA594B5A4800221A7006F096FF30
:105B400023681893189BC8F80030FFF771B999F8CB
:105B50000030554E013B012056F82310FDF79CF80C
:105B60004E4B4F4800221A7006F080FF99F8005003
:105B700005F122046400E4B2013D2046FAF7CAFFB1
:105B800056F825101831884203D089B22046FAF71A
:105B9000B5FF002389F80030FFF74AB999F80030C3
:105BA000414D424E013B55F8231017293FF740A9BC
:105BB0000020FDF771F83378013B012055F82320D0
:105BC0000244114645F82320FDF766F8334B34486C
:105BD00000221A7006F04AFF23682793279BC8F813
:105BE0000030FFF725B999F800302F4E013B012016
:105BF00056F82310FDF750F8284B294800221A7058
:105C000006F034FF99F8005005F122046400E4B274
:105C10002046013DFAF77EFF56F825309842B8D06D
:105C200003F11801B1E799F800301F4D1F4E013BF9
:105C300055F8231011F1170FFFF6FAA80020FDF711
:105C40002BF83378013B012055F82320013A114607
:105C500045F82320FDF720F8104B114800221A7058
:105C600006F004FF23682693269BC8F80030FFF750
:105C7000DFB80F4B0A48B3F90030142401221A256B
:105C800001920095194622463C7005F003FF044836
:105C900006F0ECFEFFF7CCB8048BFF1F909EFF1FB1
:105CA000049FFF1FB49EFF1F448CFF1FE49EFF1F35
:105CB000609DFF1FB24EB34BB34F32881B683968EB
:105CC0001A448A42BFF6B4A8B04D3280B5F900300C
:105CD000AF484FF0000E1A2219468DE804401422F6
:105CE00005F0D8FEAB4B3A6819683388521A5C2A23
:105CF00042F34280591A5D23561C03FB01F393FBC8
:105D0000F6F61B3633B201211A2201910092194690
:105D100014229F482E6005F0BDFE9D4806F0A6FEA9
:105D200023683D933D9A9C4BC8F8002000221A70CE
:105D3000FFF77EB8954B9648B3F9003001241A223C
:105D40008DE814001624194614223C7005F0A2FEBA
:105D50008F4806F08BFEFFF76BB8894E894A8D4F4E
:105D60003388126839689A1A8A427FF761A8874D8A
:105D70003280B5F9003086484FF0000E1A221946DD
:105D80008DE80440142205F085FE7F4B39681A68BF
:105D90003388521A5C2A41F3F887591A5D23561C3E
:105DA00003FB01F393FBF6F61B3633B201211A22F3
:105DB000019100921946142275482E6005F06AFE82
:105DC000734806F053FE23683C933C9A724BC8F824
:105DD000002000221A70FFF72BB80120FCF7A6F86C
:105DE0006D4B6B4800241C7006F040FE102089F8B3
:105DF0000040FAF78FFE694B198888423FF418A8D3
:105E00001020FAF77BFEFFF713B8FAF7B9FC644BE2
:105E10001C78002C41F0B8860120FCF787F85E4B17
:105E20005B481C7006F022FE102089F80040FAF74B
:105E300071FE5A4B198888423EF4FAAF1020FAF7E7
:105E40005DFEFEF7F5BF554D2B88012B7EF6F0AFBA
:105E50000020FCF76BF82B880120013B2B80FCF71E
:105E600065F84D4B4A4800221A7006F0FFFD236882
:105E70001C931C9BC8F80030FEF7DABF474D2B88F7
:105E80000F2B3EF6D5AF0020FCF750F82B880120F1
:105E900003442B80FCF74AF83F4B3D4800221A7020
:105EA00006F0E4FD23681D931D9BC8F80030FEF743
:105EB000BFBF0390FEF762FC03983A4D03680C9352
:105EC0000C9A2A6000233370FFF7F3B80368DFF8F9
:105ED000E4803093344A309BD8F8001012685B1A83
:105EE000934219D92C4A2A481378012B0CBF00235E
:105EF00001231370254A0193B2F900301A22194682
:105F00000092142205F0C6FD214806F0AFFD23687B
:105F10003193319BC8F80030244A1378002B3EF4AB
:105F200087AF234B1B680021013B1170072B3EF606
:105F30007FAF01A252F823F05F60000039600000DB
:105F4000314E0000B95F0000314E0000314E0000BC
:105F5000314E0000595F00000C4B0D48B3F9003082
:105F600001241A228DE814000A24194614223C70D8
:105F700005F090FD064806F079FDFEF759BF00BF19
:105F8000EC9DFF1FB89EFF1FE48DFF1F609DFF1F4C
:105F9000049FFF1F688AFF1F909EFF1F609EFF1FC8
:105FA0009C9DFF1FB09DFF1F908DFF1FFC9DFF1F3D
:105FB000949EFF1F409EFF1FA24EA34BA34F32880B
:105FC0001B6839681A448A42BEF632AFA04D32804F
:105FD000B5F900309F484FF0000E1A2219468DE89F
:105FE0000440142205F056FD9B4B3A68196833882B
:105FF000521A5C2A41F35A84591A5D23561C03FB3A
:1060000001F393FBF6F61B3633B201211A220191FC
:106010000092194614228F482E6005F03BFD8D48F2
:1060200006F024FD23683393339A8C4BC8F8002084
:1060300000221A70FEF7FCBE854B8648B3F900308B
:1060400001241A228DE814000C24194614223C70F5
:1060500005F020FD7F4806F009FDFEF7E9BE794E08
:10606000794A7D4F3388126839689A1A8A427EF7D6
:10607000DFAE774D3280B5F9003076484FF0000E34
:106080001A2219468DE80440142205F003FD6F4BD7
:1060900039681A683388521A5C2A41F31084591AF5
:1060A0005D23561C03FB01F393FBF6F61B3633B25C
:1060B00001211A22019100921946142265482E608E
:1060C00005F0E8FC634806F0D1FC23683293329A6D
:1060D000624BC8F8002000221A70FEF7A9BEFCF738
:1060E00073FE00233370FFF798B80368DFF88481EC
:1060F00034935B4A349BD8F8001012685B1A9342C1
:1061000019D9564B53481A78012A0CBF0022012294
:106110001A70544B0192B3F900303922194600929B
:10612000322205F0B7FC4B4806F0A0FC23683593FB
:10613000359BC8F800304C4A1378002B3EF478AEFB
:106140004A4B1B680021013B1170072B3EF670AED5
:1061500001A252F823F000BF796200001F62000024
:10616000314E00009F610000314E0000314E0000B2
:10617000314E0000796100003A4B3648B3F90030E7
:10618000012439228DE814000A24194632223C7079
:1061900005F080FC2F4806F069FCFEF749BE344E3E
:1061A000294B2A4F32881B6839681A448A42BEF646
:1061B0003FAE2C4D3280B5F9003026484FF0000E2E
:1061C000392219468DE80440322205F063FC224B47
:1061D0003A6819683388521A5C2A41F3A484591A20
:1061E0005D23561C03FB01F393FBF6F61B3633B21B
:1061F00001213922019100921946322215482E6060
:1062000005F048FC134806F031FC23683793379AB1
:10621000124BC8F8002000221A70FEF709BE114B7D
:106220000C48B3F90030012439228DE814000A2407
:10623000194632223C7005F02DFC064806F016FC8B
:10624000FEF7F6BD1E9EFF1FA09EFF1F588AFF1F70
:10625000609DFF1F049FFF1F389EFF1F909EFF1F22
:10626000908DFF1FAC9EFF1FFC9DFF1F949EFF1F84
:10627000EC9EFF1F409EFF1FC34FC44AC448C54940
:106280003B881268008809689A1A43189A427EF778
:10629000CFADC14D3A80B5F90030C0483922002653
:1062A00019468DE84400322205F0F4FBBC4ABD4B90
:1062B00011681A683B88521A5C2A41F33D84591AC6
:1062C0005D23561C03FB01F393FBF6F61B3633B23A
:1062D000012139220191009219463222AF482E60E5
:1062E00005F0D8FBAD4806F0C1FB23683693369A1B
:1062F000AD4BC8F8002000221A70FEF799BDFCF7DC
:10630000D5FD00233370FEF72EBFA84E3378002B47
:1063100040F004852368DFF8B0823893A44A389BA4
:10632000D8F8001012685B1A934210D99E4B1A7865
:10633000012A0CBF002001201870FAF765FB97486E
:1063400006F094FB23683993399BC8F80030994ACA
:106350001378002B3EF46CAD974B1B680021013B7A
:106360001170072B3EF664AD01A252F823F000BF76
:1063700003640000FB630000314E0000C5630000B1
:10638000314E0000314E0000314E0000916300009C
:10639000012306203B703370FAF7BCFB874B19884A
:1063A000884202D00620FAF7A9FB0820FAF7B2FBD0
:1063B000834B198888423EF43BAD0820FAF79EFBD8
:1063C000FEF736BD01230A22062033703A70FAF731
:1063D000A1FB7A4B1988884202D00620FAF78EFB7F
:1063E0000820FAF797FB764B198888423EF420ADD7
:1063F0000820FAF783FBFEF71BBD15233B70FEF761
:1064000017BD01231E22062033703A70FAF782FB73
:106410006A4B1988884202D00620FAF76FFB0820E1
:10642000FAF778FB664B198888423EF401AD0820E4
:10643000FAF764FBFEF7FCBCDFF89091236899F84B
:106440000010DFF88481002900F0D8822893584A90
:10645000289BD8F8001012685B1A934211D9524B4E
:106460001A78012A15BF0120284618701D70FDF703
:106470006BF84A4806F0FAFA23682993299BC8F872
:1064800000304C4A1378002B3EF4D2AC4A4B1B68C8
:106490000021013B1170072B3EF6CAAC01A252F855
:1064A00023F000BF5765000027650000314E000053
:1064B000F5640000314E0000314E0000314E000006
:1064C000C56400000120FDF73FF8374B3348002436
:1064D0001C7006F0CBFA4E2089F80040FAF71AFB40
:1064E000384B198888423EF4A3AC4E20FAF706FBDD
:1064F000FEF79EBC0020FDF727F8324A1388B3FA56
:1065000083F35B0901201380FDF71EF8264B234817
:1065100000221A7006F0AAFA23682B932B9BC8F866
:106520000030FEF785BC0120FDF70EF81E4B1B481E
:1065300000241C7006F09AFA4E2089F80040FAF701
:10654000E9FA204B198888423EF472AC4E20FAF7E3
:10655000D5FAFEF76DBC0020FCF7F6FF194A138848
:10656000B3FA83F35B0901201380FCF7EDFF0E4BB8
:106570000A4800221A7006F079FA23682A932A9BA7
:10658000C8F80030FEF754BCEC9EFF1FA09EFF1F12
:106590001E9EFF1F9C8DFF1FAC9EFF1F049FFF1FB1
:1065A000389EFF1F588AFF1F909EFF1F588CFF1FA9
:1065B000908DFF1FFC9DFF1F949EFF1FEC9DFF1FF2
:1065C000CC9EFF1FCA9DFF1F409EFF1F589EFF1FAE
:1065D000B2EB630FFEF679AFAD4EAE4D33782A883D
:1065E000B3FA83F382F002025B0911464220337052
:1065F0002A80FAF783FA21460D2007F059FA9620EF
:1066000007F092FA01210D2007F052FA962007F0C8
:106610008BFA21460D2007F04BFA962007F084FAFA
:1066200001210D2007F044FAFEF702BC012323707C
:10663000FEF765BF2368DFF894821E9396481E9B81
:10664000D8F8001000685B1A834215D9934B19786B
:10665000012916BF01221A701A70914B08BF154606
:1066600018782946FAF7BAF98E4806F0FFF9236838
:106670001F931F9BC8F800308B4B1A78002A3EF4FA
:10668000D7AB00221A70FAF77BF8884A884B894901
:10669000894812781B780968007802EB43034A1E88
:1066A00003EB80030B2A3EF6C3AB01A151F822F0A5
:1066B0009B67000093670000314E000051670000A7
:1066C000314E0000314E0000314E000045670000A1
:1066D000314E0000E1660000314E000013670000FB
:1066E000002B3EF4A5AB754A754D128803F11900D5
:1066F000013B4000022425F813201146012300F03D
:10670000FE0033703C70FAF7F9F96E4B1C70FEF71F
:106710008FBB002B3EF48CAB03F11900684D013B9D
:106720000022400025F813201146012300F0FE004E
:10673000022433703C70FAF7E1F9624B03221A70BD
:10674000FEF776BB002201233A703370FEF770BB70
:10675000534C207801287EF66BAB0021FAF73EF906
:1067600023784E4D013BDBB2184601212370FAF726
:1067700035F9002434238DE818004A482C70402352
:106780000B223F2105F054F9464806F06FF9FEF759
:106790004FBBFCF71DFDFEF74BBB414C2078052895
:1067A0003EF646AB0021FAF719F923783B4D013349
:1067B000DBB2184601212370FAF710F900243423C4
:1067C0008DE8180037482C7040230B223F2105F03C
:1067D0002FF9344806F04AF9FEF72ABB2368DFF8A0
:1067E000EC803E932C4A3E9BD8F8001012685B1A4E
:1067F000934219D9294A2B481378012B0CBF002347
:1068000001231370304A0193B2F90030392219463E
:106810000092322205F03EF9224806F027F923685B
:106820003F933F9BC8F800301F4A1378002B3EF47B
:10683000FFAA204B1B680021013B1170072B3EF67D
:10684000F7AA01A252F823F077690000516900000D
:10685000314E0000D1680000314E0000314E000082
:10686000314E000069680000174B0E48B3F9003044
:10687000012439228DE814001424194632223C7078
:1068800005F008F9074806F0F1F8FEF7D1BA00BFA5
:10689000C29DFF1FEE9EFF1F908DFF1F909EFF1F4A
:1068A0003289FF1F049FFF1FFC9DFF1FD59EFF1F06
:1068B000309FFF1F949EFF1F319FFF1F6C9EFF1F85
:1068C000789DFF1F669DFF1FAC9EFF1F409EFF1F10
:1068D000B44EB54BB54F32881B6839681A448A42AA
:1068E000BEF6A6AAB24D3280B5F90030B1484FF0DD
:1068F000000E392219468DE80440322205F0CAF80C
:10690000AD4B3A6819683388521A5C2A41F34682C3
:10691000591A5D23561C03FB01F393FBF6F61B3655
:1069200033B2012139220191009219463222A14845
:106930002E6005F0AFF89F4806F098F82368419361
:10694000419A9E4BC8F8002000221A70FEF770BAD8
:10695000974B9848B3F90030012439228DE8140090
:106960001424194632223C7005F094F8914806F040
:106970007DF8FEF75DBA8B4E8B4A9148914933887A
:106980001268008809689A1A43189A427EF750AA3A
:10699000874D3280B5F900308648392200271946E4
:1069A0008DE88400322205F075F8834A7F4B116828
:1069B0001A683388521A5C2A41F33C82591A5D23C3
:1069C000561C03FB01F393FBF6F61B3633B2012191
:1069D0003922019100921946322276482E6005F044
:1069E00059F8744806F042F823684093409A734B74
:1069F000C8F8002000221A70FEF71ABA2C93724AC7
:106A00002C9BD8F8000012681B1A934211D96B4BCB
:106A10001A78012A18BF012119706C4B1878F9F700
:106A2000DDFF644806F022F823682D932D9BC8F8FB
:106A30000030674B1A78002A3EF4FAA900221A7037
:106A4000F9F79EFE634A644B6449654812781B78E7
:106A50000968007802EB43034A1E03EB80030B2A0C
:106A60003EF6E6A901A151F822F000BF576B0000E5
:106A70004F6B0000314E00000D6B0000314E0000E6
:106A8000314E0000314E0000016B0000314E00001D
:106A90009D6A0000314E0000CF6A0000002B3EF4DA
:106AA000C7A9504A504D128803F11900013B40001C
:106AB000022425F813201146012300F0FE00337054
:106AC0003C70FAF71BF8494B1C70FEF7B1B9002B6C
:106AD0003EF4AEA903F11900434D013B00224000F2
:106AE00025F813201146012300F0FE000224337024
:106AF0003C70FAF703F83D4B03221A70FEF798B981
:106B0000002201233A703370FEF792B92F4C20789F
:106B100001287EF68DA90021F9F760FF2378274D23
:106B2000013BDBB2184601212370F9F757FF00241F
:106B300034238DE818001F482C7040230B223F217E
:106B400004F076FF1B4805F091FFFEF771B9FCF7E2
:106B500059FDFEF76DB91D4C207805283EF668A951
:106B60000021F9F73BFF2378144D0133DBB21846BF
:106B700001212370F9F732FF002434238DE8180037
:106B80000C482C7040230B223F2104F051FF094890
:106B900005F06CFFFEF74CB9002101201170187050
:106BA000FEF750BCCC9EFF1FB89EFF1FE48DFF1F59
:106BB000AC9EFF1F049FFF1F688AFF1F909EFF1F50
:106BC000EC9DFF1F9C8DFF1F908DFF1F948DFF1F5D
:106BD000FC9DFF1FD59EFF1F309FFF1F949EFF1F30
:106BE000319FFF1F6C9EFF1F789DFF1F669DFF1F3B
:106BF000AA4E3378002B40F0B1832368DFF8D082AF
:106C00004293A74A429BD8F8001012685B1A93423D
:106C100010D9A44B1A78012A0CBF0020012018704B
:106C2000F9F7F2FEA04805F021FF23684393439B48
:106C3000C8F800309D4A1378002B3EF4F9A89C4B0D
:106C40001B680021013B1170072B3EF6F1A801A241
:106C500052F823F0E76C0000DF6C0000314E0000BA
:106C6000A96C0000314E0000314E0000314E000092
:106C7000756C000001230A203B703370F9F74AFF5E
:106C80008C4B1988884202D00A20F9F737FF0C2074
:106C9000F9F740FF884B198888423EF4C9A80C20B8
:106CA000F9F72CFFFEF7C4B8012314220A20337031
:106CB0003A70F9F72FFF7F4B1988884202D00A20DB
:106CC000F9F71CFF0C20F9F725FF7B4B1988884248
:106CD0003EF4AEA80C20F9F711FFFEF7A9B81F2368
:106CE0003B70FEF7A5B8012328220A2033703A70C2
:106CF000F9F710FF6F4B1988884202D00A20F9F784
:106D0000FDFE0C20F9F706FF6B4B198888423EF414
:106D10008FA80C20F9F7F2FEFEF78AB8FCF7C6FF41
:106D2000664A0121002311703370FFF7F3BAAF21D7
:106D30005D4805F001FD642201233A703370FEF7CF
:106D400077B82368DFF888814493554A449BD8F884
:106D5000001012685B1A934219D9524A52481378AC
:106D6000012B0CBF002301231370554A0193B2F984
:106D700000301A2219460092142204F08BFE4A4871
:106D800005F074FE23684593459BC8F80030474AD8
:106D90001378002B3EF44CA8454B1B680021013BA7
:106DA0001170072B3EF644A801A252F823F000BF51
:106DB000D56E0000776E0000314E0000F76D0000C8
:106DC000314E0000314E0000314E0000D16D000008
:106DD0003B4B3548B3F9003001241A228DE81400EA
:106DE0001E24194614223C7004F054FE2E4805F06F
:106DF0003DFEFEF71DB82F4E324B334F32881B68D5
:106E000039681A448A42BEF613A82D4D3280B5F96E
:106E1000003025484FF0000E1A2219468DE8044034
:106E2000142204F037FE294B3A6819683388521A45
:106E30005C2A41F3AB80591A5D23561C03FB01F316
:106E400093FBF6F61B3633B201211A220191009210
:106E50001946142214482E6004F01CFE124805F056
:106E600005FE23684793479A0E4BC8F8002000227E
:106E70001A70FDF7DDBF124B0B48B3F90030012447
:106E80001A228DE814002024194614223C7004F0C4
:106E900001FE054805F0EAFDFDF7CABF588CFF1F4B
:106EA000908DFF1F909EFF1F049FFF1FFC9DFF1FE3
:106EB000949EFF1F349EFF1FBC9DFF1F749DFF1FEC
:106EC000609DFF1FA49EFF1F3C8BFF1FE88DFF1FCF
:106ED000409EFF1FAD4EAE4AAE4F338812683968F0
:106EE0009A1A8A427DF7A4AFAB4D3280B5F90030D3
:106EF000AA484FF0000E1A2219468DE804401422C9
:106F000004F0C8FDA64B39681A683388521A5C2A07
:106F100041F39480591A5D23561C03FB01F393FB44
:106F2000F6F61B3633B201211A220191009219465E
:106F300014229A482E6004F0ADFD984805F096FDA5
:106F400023684693469A974BC8F8002000221A708F
:106F5000FDF76EBF00201870FEF770BA0021012007
:106F600011701870FEF725B92368DFF86482489322
:106F70008D4A489BD8F8001012685B1A934219D9C1
:106F8000884A86481378012B0CBF00230123137015
:106F9000864A0193B2F90030392219460092322212
:106FA00004F078FD7D4805F061FD23684993499B15
:106FB000C8F800307E4A1378002B3DF439AF7D4B82
:106FC0001B680021013B1170072B3DF631AF01A278
:106FD00052F823F0C17000009B700000314E000099
:106FE0001B700000314E0000314E0000314E000099
:106FF000F56F00006D4B6948B3F900300124392268
:107000008DE814001E24194632223C7004F042FD23
:10701000624805F02BFDFDF70BBF674E5C4B604FE0
:1070200032881B6839681A448A42BDF601AF5F4D49
:107030003280B5F9003059484FF0000E3922194618
:107040008DE80440322204F025FD524B3A6819685D
:107050003388521A5C2A41F37D80591A5D23561CED
:1070600003FB01F393FBF6F61B3633B20121392201
:10707000019100921946322248482E6004F00AFD20
:10708000464805F0F3FC23684B934B9A454BC8F8F0
:10709000002000221A70FDF7CBBE444B3F48B3F9E5
:1070A0000030012439228DE814001E2419463222B2
:1070B0003C7004F0EFFC394805F0D8FCFDF7B8BE91
:1070C0003D4E334A31483D4933881268008809688B
:1070D0009A1A43189A427DF7ABAE344D3280B5F917
:1070E00000302E483922002719468DE884003222CC
:1070F00004F0D0FC274A2A4B11681A683388521AC8
:107100005C2A41F34780591A5D23561C03FB01F3A7
:1071100093FBF6F61B3633B201213922019100921E
:10712000194632221D482E6004F0B4FC1B4805F0BD
:107130009DFC23684A934A9A1A4BC8F80020002203
:107140001A70FDF775BE1E4A1E4E13881E48012B8D
:107150008CBF03F1FF33802313801C4A00230121DD
:10716000337003701170FEF712BB154A154E138869
:1071700015487F2B94BF013301231380134A00234A
:107180000121337003701170FEF7C6BA349EFF1FE1
:10719000A49EFF1FE88DFF1F609DFF1F049FFF1F20
:1071A0003C8BFF1F909EFF1F908DFF1FAC9EFF1F0B
:1071B000FC9DFF1F949EFF1FBC9DFF1F9C8DFF1F0A
:1071C0006C9EFF1FF69DFF1F669DFF1F9D9DFF1F6D
:1071D000409EFF1FC04DC14C2B782288B3FA83F329
:1071E00082F004025B09114642202B702280F9F7DD
:1071F00085FC00210D2006F05BFC962006F094FC37
:1072000001210D2006F054FC962006F08DFC002193
:107210000D2006F04DFC962006F086FC01210D2085
:1072200006F046FCFDF704BEAD4E3378002B40F06F
:107230004F832368DFF8E0824C93AA4A4C9BD8F82E
:10724000001012685B1A934210D9A74B1A78012AD2
:107250000CBF002001201870F9F7D6FBA34805F0F9
:1072600005FC23684D934D9BC8F80030A04A137865
:10727000002B3DF4DDAD9F4B1B680021013B1170DD
:10728000072B3DF6D5AD01A252F823F01F73000085
:1072900017730000314E0000E1720000314E000013
:1072A000314E0000314E0000AD720000012322205B
:1072B0003B703370F9F72EFC8F4B1988884202D04F
:1072C0002220F9F71BFC2420F9F724FC8B4B1988AA
:1072D00088423DF4ADAD2420F9F710FCFDF7A8BDC0
:1072E00001231E22222033703A70F9F713FC824BDF
:1072F0001988884202D02220F9F700FC2420F9F7EF
:1073000009FC7E4B198888423DF492AD2420F9F7A0
:10731000F5FBFDF78DBD29233B70FDF789BD0123EA
:107320003C22222033703A70F9F7F4FB724B198833
:10733000884202D02220F9F7E1FB2420F9F7EAFB8A
:107340006E4B198888423DF473AD2420F9F7D6FBC3
:10735000FDF76EBD00201870FDF727BFFCF782FB1C
:10736000674A012100231170337046E46549012307
:1073700000220B7033703A70FEF7A5B92368DFF86E
:1073800098814E93574A4E9BD8F8001012685B1AAA
:1073900093421AD9544B5C491A785448012A0CBFBD
:1073A000002201221A701A78B1F9003001921A22D3
:1073B00019460092142204F06DFB4C4805F056FB70
:1073C00023684F934F9BC8F80030494A1378002B2D
:1073D0003DF42EAD474B1B680021013B1170072B7C
:1073E0003DF626AD01A252F823F000BF1D75000046
:1073F000B3740000314E000033740000314E0000C1
:10740000314E0000314E00000D7400003E4B3748F5
:10741000B3F9003001241A228DE8140028241946FB
:1074200014223C7004F036FB304805F01FFBFDF7DA
:10743000FFBC314E354B364F32881B6839681A44D1
:107440008A42BDF6F5AC304D3280B5F900302748A0
:107450004FF0000E1A2219468DE80440142204F061
:1074600019FB2C4B3A6819683388521A5C2A41F38D
:107470002882591A5D23561C03FB01F393FBF6F691
:107480001B3633B201211A220191009219461422AF
:1074900016482E6004F0FEFA144805F0E7FA236857
:1074A0005193519A104BC8F8002000221A70FDF732
:1074B000BFBC154B0D48B3F9003001241A228DE8EA
:1074C00014002A24194614223C7004F0E3FA0748F9
:1074D00005F0CCFAFDF7ACBC1C9EFF1FEE9EFF1F13
:1074E000588CFF1F908DFF1F909EFF1F049FFF1F52
:1074F000FC9DFF1F949EFF1F969DFF1F4E9EFF1F2A
:10750000749DFF1F9D9DFF1F609DFF1F549EFF1FC9
:107510005C8AFF1FFC8DFF1F409EFF1FB94EBA4AB9
:10752000BA4F3388126839689A1A8A427DF780AC5C
:10753000B74D3280B5F90030B6484FF0000E1A2230
:1075400019468DE80440142204F0A4FAB24B3968BD
:107550001A683388521A5C2A41F3C581591A5D238F
:10756000561C03FB01F393FBF6F61B3633B20121E5
:107570001A220191009219461422A6482E6004F0A6
:1075800089FAA44805F072FA23685093509AA34BE5
:10759000C8F8002000221A70FDF74ABC2368DFF803
:1075A0009C8252939E4A529BD8F8001012685B1A34
:1075B00093421AD9994B9B491A789648012A0CBFD5
:1075C000002201221A701A78B1F900300192392292
:1075D00019460092322204F05DFA8E4805F046FA10
:1075E00023685393539BC8F800308F4A1378002BBD
:1075F0003DF41EAC8D4B1B680021013B1170072B25
:107600003DF616AC01A252F823F000BFF976000057
:10761000D3760000314E000053760000314E00005A
:10762000314E0000314E00002D7600007D4B794830
:10763000B3F90030012439228DE8140028241946BA
:1076400032223C7004F026FA724805F00FFAFDF77A
:10765000EFBB774E6C4B704F32881B6839681A4409
:107660008A42BDF6E5AB6F4D3280B5F9003069480E
:107670004FF0000E392219468DE80440322204F002
:1076800009FA624B3A6819683388521A5C2A40F347
:107690004986591A5D23561C03FB01F393FBF6F64A
:1076A0001B3633B201213922019100921946322250
:1076B00058482E6004F0EEF9564805F0D7F92368D3
:1076C0005593559A554BC8F8002000221A70FDF7C3
:1076D000AFBB544B4F48B3F90030012439228DE839
:1076E00014002824194632223C7004F0D3F949488A
:1076F00005F0BCF9FDF79CBB4D4E434A41484D494E
:1077000033881268008809689A1A43189A427DF7EC
:107710008FAB444D3280B5F900303E483922002706
:1077200019468DE88400322204F0B4F9374A3A4B06
:1077300011681A683388521A5C2A41F3DD80591A9D
:107740005D23561C03FB01F393FBF6F61B3633B2A5
:107750000121392201910092194632222D482E60D2
:1077600004F098F92B4805F081F923685493549A52
:107770002A4BC8F8002000221A70FDF759BB2E4E84
:107780003378002B40F0F0822368DFF8B080569306
:10779000234A569BD8F8001012685B1A934211D9FD
:1077A0001E4B1A78012A0CBF002201221A70187889
:1077B000F9F72AF9174805F059F923685793579BA9
:1077C000C8F80030184A1378002B3DF431AB174B42
:1077D0001B680021013B1170072B3DF629AB01A26C
:1077E00052F823F08B78000083780000314E0000BF
:1077F00061780000314E0000314E0000314E000033
:1078000041780000969DFF1F549EFF1FFC8DFF1FB7
:10781000609DFF1F049FFF1F5C8AFF1F909EFF1F3C
:10782000908DFF1FAC9EFF1FFC9DFF1F949EFF1FAE
:107830004E9EFF1F9C8DFF1F588CFF1F409EFF1FF9
:1078400001232A203B703370F9F764F9BF4B198884
:1078500088423DF4EDAA2A20F9F750F9FDF7E8BA7D
:10786000012328222A2033703A70F9F753F9B74BD5
:10787000198888423DF4DCAA2A20F9F73FF9FDF780
:10788000D7BA3D233B70FDF7D3BA01230A222A2041
:1078900033703A70F9F73EF9AC4B198888423DF4E1
:1078A000C7AA2A20F9F72AF9FDF7C2BA5E1A5C23A3
:1078B00003FB06F393FBF2F61B36FEF7A5BB5E1A3D
:1078C0005C2303FB06F393FBF2F61B36FEF7EFBBDC
:1078D000FCF710FB9E4A0121002311703370A8E4CD
:1078E0002368DFF89C8258939A4A589BD8F8001076
:1078F00012685B1A93421AD9974B98491A7898489C
:10790000012A0CBF002201221A701A78B1F9003046
:1079100001921A2219460092142204F0BBF89048F2
:1079200005F0A4F823685993599BC8F800308D4A94
:107930001378002B3DF47CAA8B4B1B680021013B84
:107940001170072B3DF674AA01A252F823F000BF74
:10795000737A00004D7A0000314E000097790000E4
:10796000314E0000314E0000314E000071790000B0
:107970007A4B7B48B3F9003001241A228DE81400B9
:107980003C24194614223C7004F084F8744805F035
:107990006DF8FDF74DBA6D4E744A754F3388126815
:1079A000D7F800E01A447245BDF642AA7149724BFD
:1079B000DFF8D09108681D68D9F8001093B2CEEBBB
:1079C00001012A1A91423380644DCEEB0303CCBFF0
:1079D00002FB03335343694AC8BF013193FBF1F300
:1079E000B5F90010034413604FF0000E1A220B4645
:1079F0008DE804405A48142204F04CF8D9F80010DD
:107A00003A683388521A5C2A40F36487591A5D2316
:107A1000561C03FB01F393FBF6F61B3633B2012130
:107A20001A2201910092194614224D482E6004F04A
:107A300031F84B4805F01AF823685B935B9A464B84
:107A4000C8F8002000221A70FDF7F2B9434B4448F1
:107A5000B3F9003001241A228DE814003C241946A1
:107A600014223C7004F016F83D4804F0FFFFFDF7C7
:107A7000DFB9364E3D4ADFF80C9133881268D9F8E9
:107A800000509A1AAA427DF7D3A93B4B384F394987
:107A9000D7F800E01868096893B2CEEB0505421AE2
:107AA00095423380CEEB030341F3A08302FB033303
:107AB0006A1C93FBF2F31944284D304AB5F90030A3
:107AC00011604FF0000E1A2219468DE80440244838
:107AD000142203F0DFFFD9F800103A683388521AF5
:107AE0005C2A41F37A83591A5D23561C03FB01F388
:107AF00093FBF6F61B3633B201211A220191009254
:107B00001946142216482E6003F0C4FF144804F0EE
:107B1000ADFF23685A935A9A0F4BC8F800200022F1
:107B20001A70FDF785B95E1A5C2303FB06F393FB1D
:107B3000F2F61B36FEF75BBB5E1A5C2303FB06F313
:107B400093FBF2F61B36FEF7C2BB00BFF49EFF1F8D
:107B5000749DFF1F908DFF1F909EFF1F609DFF1F54
:107B6000049FFF1FFC9DFF1F949EFF1FE09DFF1FB2
:107B7000408CFF1F608AFF1F5C8CFF1F548CFF1F0F
:107B8000409EFF1FF48DFF1FAF4A1378B3FA83F3B3
:107B90005B0901201370FAF7C9F9AC4BAC4800221D
:107BA0001A7004F063FFAB4A138883F00803194688
:107BB00042201380F8F7A2FFFDF73AB9A64E3378BA
:107BC0001BB1FBF799F900233370A44D29780029E4
:107BD00000F086802368DFF8A4825C93A04A5C9B57
:107BE000D8F8001012685B1A934211D9974B1A7893
:107BF000012A0CBF002201221A701878FCF730FE0F
:107C0000934804F033FF23685D935D9BC8F8003010
:107C1000944A1378002B3DF40BA9934B1B68002169
:107C2000013B1170072B3DF603A901A252F823F086
:107C3000A589000073890000314E00003D890000D5
:107C4000314E0000314E0000314E00000B89000023
:107C5000814E3378002B40F0A281844D2A78002A8F
:107C600000F00E812368DFF8148278937C4A789BB9
:107C7000D8F8001012685B1A934211D9734B1A7826
:107C8000012A0CBF002201221A701878FCF7F0FBC1
:107C90006F4804F0EBFE23687993799BC8F80030B5
:107CA000704A1378002B3DF4C3A86F4B1B6800216A
:107CB000013B1170072B3DF6BBA801A252F823F03F
:107CC000B58A0000878A0000314E0000538A000008
:107CD000314E0000314E0000314E0000258A000078
:107CE000634D2A78002A00F0B2812368DFF88C8186
:107CF00062935B4A629BD8F8000012681B1A934299
:107D000011D9524B1A78012A16BF012219701A7024
:107D10001878FBF7D5FA4E4804F0A8FE2368639361
:107D2000639BC8F800304F4A1378002B3DF480A8BD
:107D30004D4B1B680021013B1170072B3DF678A8C5
:107D400001A252F823F000BF519300001F930000DE
:107D5000314E0000ED920000314E0000314E000027
:107D6000314E0000BB920000FBF7C0FD414A0121EB
:107D700000231170337007E55E1A5C2303FB06F3E2
:107D800093FBF2F61B36FDF7BDBF5E1A5C2303FBC7
:107D900006F393FBF2F61B36FEF707B85E1A5C2378
:107DA00003FB06F393FBF2F61B36FEF7B9BD324D2B
:107DB0002978002900F0FE802368DFF8C0809293C4
:107DC0002749929BD8F8000009681B1A8B4210D9EA
:107DD0001E4B1978012918BF01221A701878F8F77C
:107DE00033FE1B4804F042FE23689393939BC8F82C
:107DF00000301C4A1378002B3DF41AA81A4B1B685C
:107E00000021013B1170072B3DF612A801A252F888
:107E100023F000BF31940000E7930000314E0000D2
:107E2000B1930000314E0000314E0000314E000091
:107E3000839300005E1A5C2303FB06F393FBF2F6C8
:107E40001B36FEF7C3BD00BFE29EFF1F909EFF1FC3
:107E5000049FFF1FEE9EFF1F588CFF1F5A9DFF1FA0
:107E6000908DFF1FFC9DFF1F949EFF1F4C9EFF1FC8
:107E7000D49EFF1F749DFF1F089EFF1F409EFF1F83
:107E8000B94D297800293DD02368DFF804837C931D
:107E9000B6497C9BD8F8000009681B1A8B4210D9A0
:107EA000B34B1978012918BF01221A701878FAF714
:107EB0001BFEB04804F0DAFD23687D937D9BC8F873
:107EC0000030AD4A1378002B3CF4B2AFAB4B1B68CB
:107ED0000021013B1170072B3CF6AAAF01A252F81A
:107EE00023F000BF19860000EB850000314E000032
:107EF000B5850000314E0000314E0000314E0000CB
:107F0000878500009E4D2A78002A00F01D8723688F
:107F1000DFF87C828093954A809BD8F80000126835
:107F20001B1A934211D9924B1A78012A16BF0122CB
:107F300019701A701878FCF7FFFA8E4804F096FD55
:107F400023688193819BC8F800308B4A1378002BFB
:107F50003CF46EAF894B1B680021013B1170072B6D
:107F60003CF666AF01A252F823F000BFDF860000A6
:107F7000B1860000314E00007D860000314E0000C9
:107F8000314E0000314E00004F8600005E1A5C2327
:107F900003FB06F393FBF2F61B36FEF754BFFAF72A
:107FA000CDFF0023337058E6FAF7EAFF0023337061
:107FB000FCF782BF734D2A78002A00F005862368FB
:107FC000DFF8CC819693694A969BD8F80000126836
:107FD0001B1A934211D9664B1A78012A16BF012247
:107FE00019701A701878F8F74DFD624804F03EFDDC
:107FF00023689793979BC8F800305F4A1378002B4B
:108000003CF416AF5D4B1B680021013B1170072B40
:108010003CF60EAF01A252F823F000BF5D8B0000CA
:108020002F8B0000314E00008D8B0000314E000080
:10803000314E0000314E0000018B00005E1A5C23BF
:1080400003FB06F393FBF2F61B36FEF76BBF4E4DB8
:10805000297800293CD02368DFF8348166934349AE
:10806000669BD8F8000009681B1A8B4210D9404B58
:108070001978012918BF01221A701878FAF76CFCD8
:108080003C4804F0F3FC23686793679BC8F8003012
:10809000394A1378002B3CF4CBAE384B1B680021D7
:1080A000013B1170072B3CF6C3AE01A252F823F03E
:1080B000878800001F880000314E00004D880000B6
:1080C000314E0000314E0000314E00001387000099
:1080D0002E4D2A78002A66D02368DFF8B4806A9390
:1080E000224A6A9BD8F8000012681B1A934211D9E1
:1080F0001F4B1A78012A16BF012219701A701878BE
:10810000FCF776FC1B4804F0B1FC23686B936B9B77
:10811000C8F80030184A1378002B3CF489AE174B8E
:108120001B680021013B1170072B3CF681AE01A2B8
:1081300052F823F0ED870000A3870000314E0000C5
:108140006F870000314E0000314E0000314E0000BC
:10815000418700005E1A5C2303FB06F393FBF2F6F3
:108160001B36FEF782BF00BF589DFF1F908DFF1F7B
:10817000909EFF1F049FFF1FFC9DFF1F949EFF1FEB
:10818000649DFF1FE49DFF1F949DFF1F2F9FFF1FF6
:10819000409EFF1F5E1A5C2303FB06F393FBF2F67F
:1081A0001B36FEF7B8BFBA4D297800293CD02368AA
:1081B000DFF800836E93B7496E9BD8F8000009681A
:1081C0001B1A8B4210D9B44B1978012918BF012210
:1081D0001A701878FBF7AEFAB04804F047FC236831
:1081E0006F936F9BC8F80030AD4A1378002B3CF4B6
:1081F0001FAEAC4B1B680021013B1170072B3CF6F6
:1082000017AE01A252F823F015850000E7840000A4
:10821000314E000047850000314E0000314E000015
:10822000314E0000B98400009F4D23682A78DFF8A2
:108230008482002A3AD07293964A729BD8F8000042
:1082400012681B1A934211D9934B1A78012A16BF50
:10825000012219701A701878FAF7B8FC8F4804F0E8
:1082600005FC23687393739BC8F800308C4A13781D
:10827000002B3CF4DDAD8B4B1B680021013B1170E2
:10828000072B3CF6D5AD01A252F823F05D84000027
:108290002F840000314E0000FB830000314E0000AF
:1082A000314E0000314E0000CD83000076937949B5
:1082B000769BD8F8000009681B1A8B4212D9764BBE
:1082C0001978012918BF01221A70784A1978107894
:1082D000F8F784FB714804F0C9FB23687793779B18
:1082E000C8F800306E4A1378002B3CF4A1AD6D4BFA
:1082F0001B680021013B1170072B3CF699AD01A2D0
:1083000052F823F08B83000083830000314E00007D
:1083100041830000314E0000314E0000314E00001C
:10832000378300005E1A5C2303FB06F393FBF2F62F
:108330001B36FFF7B6B901233B703370FCF778BDED
:108340005A4C207801287CF673AD0021F8F746FBE3
:108350002378514D013BDBB2184601212370F8F719
:108360003DFB002434238DE818004C482C7040233A
:108370000B223F2103F05CFB484804F077FBFCF73D
:1083800057BDFCF711FCFCF753BD484C207805287D
:108390003CF64EAD0021F8F721FB23783E4D01332A
:1083A000DBB2184601212370F8F718FB00243423B0
:1083B0008DE8180039482C7040230B223F2103F030
:1083C00037FB364804F052FBFCF732BD0120FAF7C8
:1083D000FDFB314B314800241C7004F047FB30207A
:1083E0002C70F8F797FB324B198888423CF420AD8B
:1083F0003020F8F783FBFCF71BBD0020FAF7E6FB03
:108400002B4A1388082B94BF0133002301201380CB
:10841000FAF7DCFB204B214800221A7004F026FBFF
:1084200023687593759BC8F80030FCF701BD0120E7
:10843000FAF7CCFB184B194800241C7004F016FB0B
:1084400030202C70F8F766FB194B198888423CF4F1
:10845000EFAC3020F8F752FBFCF7EABC0020FAF74B
:10846000B5FB134A1388002B00F08780013B138073
:108470000120FAF7ABFB084B084800221A7004F001
:10848000F5FA23687493749BC8F80030FCF7D0BCED
:10849000BE9DFF1F908DFF1F909EFF1F049FFF1F1B
:1084A000FC9DFF1F949EFF1FF49DFF1F648AFF1F0A
:1084B000689DFF1F409EFF1F0120FBF73BF9C44B47
:1084C000C44800241C7004F0D1FA2E202C70F8F758
:1084D00021FBC14B198888423CF4AAAC2E20F8F746
:1084E0000DFBFCF7A5BC0120FBF724F9B84BB948FC
:1084F00000241C7004F0BAFA2E202C70F8F70AFB46
:10850000B54B198888423CF493AC2E20F8F7F6FA64
:10851000FCF78EBC0020FBF70DF9AF4A1388002B47
:108520002ED0013B13800120FBF704F9A84BA9488A
:1085300000221A7004F09AFA23687093709BC8F8AE
:108540000030FCF775BC0020FBF7F4F8A24A138852
:108550001D2B94BF0133002301201380FBF7EAF8A1
:108560009B4B9C4800221A7004F080FA2368719398
:10857000719BC8F80030FCF75BBC0923138077E7D8
:108580001E231380CFE70120FAF7AEFA904B9148F3
:1085900000241C7004F06AFA1A202C70F8F7BAFA5A
:1085A0008E4B198888423CF443AC1A20F8F7A6FA9F
:1085B000FCF73EBC894D2B880B2B3CF639AC0020D8
:1085C000FAF792FA2B88012003442B80FAF78CFAF1
:1085D0007F4B804800221A7004F048FA23687F938A
:1085E0007F9BC8F80030FCF723BC0120FAF77CFA27
:1085F000774B784800241C7004F038FA1A202C704D
:10860000F8F788FA754B198888423CF411AC1A20A7
:10861000F8F774FAFCF70CBC704D2B88002B3CF477
:1086200007AC0020FAF760FA2B880120013B2B8071
:10863000FAF75AFA664B674800221A7004F016FAE5
:1086400023687E937E9BC8F80030FCF7F1BB0120C5
:10865000FBF772FF5E4B5F4800241C7004F006FAC3
:108660001C202C70F8F756FA5D4B198888423CF4B0
:10867000DFAB1C20F8F742FAFCF7DABB0020FBF76F
:108680005BFF574A1388032B94BF0133002301205B
:108690001380FBF751FF4E4B4E4800221A7004F036
:1086A000E5F923688393839BC8F80030FCF7C0BBCF
:1086B0000120FBF741FF464B464800241C7004F0A4
:1086C000D5F91C202C70F8F725FA454B19888842FB
:1086D0003CF4AEAB1C20F8F711FAFCF7A9BB002064
:1086E000FBF72AFF3E4A1388002B00F0C980013BAC
:1086F00013800120FBF720FF354B364800221A700B
:1087000004F0B4F923688293829BC8F80030FCF728
:108710008FBB0120FAF720F92D4B2E4800241C7046
:1087200004F0A4F916202C70F8F7F4F92D4B1988F1
:1087300088423CF47DAB1620F8F7E0F9FCF778BBF3
:108740000120FCF755F9224B224800241C7004F04C
:108750008DF92C202C70F8F7DDF9234B198888420D
:108760003CF466AB2C20F8F7C9F9FCF761BB00209C
:10877000FCF73EF91C4A13880B2B94BF01330023EE
:1087800001201380FCF734F9114B124800221A70B3
:1087900004F06CF923686D936D9BC8F80030FCF70A
:1087A00047BB0120FCF724F9094B0A4800241C7040
:1087B00004F05CF92C202C70F8F7ACF90A4B1988FE
:1087C00088423CF435AB2C20F8F798F9FCF730BB25
:1087D000909EFF1F049FFF1FBC9EFF1FD49DFF1F85
:1087E000CC9DFF1F5C9DFF1FAA9DFF1F0020FCF773
:1087F000FFF8BD4A1388002B5DD0013B1380012098
:10880000FCF7F6F8B94BBA4800221A7004F02EF9BA
:1088100023686C936C9BC8F80030FCF709BB0120FF
:10882000FAF79AF8B14BB24800241C7004F01EF914
:1088300016202C70F8F76EF9AE4B198888423CF47C
:10884000F7AA1620F8F75AF9FCF7F2BA0020FAF75F
:1088500083F8A84A13887E2B94BF0133002301209C
:108860001380FAF779F8A14BA14800221A7004F09E
:10887000FDF823686993699BC8F80030FCF7D8BA03
:108880000423138035E70020FAF766F8994A138825
:10889000A3B1013B13800120FAF75EF8934B944893
:1088A00000221A7004F0E2F823686893689BC8F805
:1088B0000030FCF7BDBA0C231380A0E77F231380A0
:1088C000E9E75E1A5C2303FB06F393FBF2F61B3623
:1088D000FEF7D7BD5E1A5C2303FB06F393FBF2F6AB
:1088E0001B36FFF79BB85E1A5C2303FB06F393FB72
:1088F000F2F61B36FEF73ABE5E1A5C2303FB06F364
:1089000093FBF2F61B36FEF722BF0120FBF7A8FF10
:10891000764B774800241C7004F0A8F812202C70C5
:10892000F8F7F8F8744B198888423CF481AA1220B1
:10893000F8F7E4F8F8F792FCFCF77ABA6E4D2B885A
:10894000092B4FF0000046D8FBF78AFF2B88012047
:1089500003442B80FBF784FF644B654800221A70A8
:1089600004F084F823686093609BC8F80030FCF73B
:108970005FBA0120FBF774FF5C4B5D4800241C705C
:1089800004F074F812202C70F8F7C4F85A4B1988C8
:1089900088423CF44DAA1220F8F7B0F8F8F75EFCD4
:1089A000FCF746BA544D2E8846B30020FBF758FF1B
:1089B0002B880120013B2B80FBF752FF4B4B4C488F
:1089C00000221A7004F052F823685E935E9BC8F888
:1089D0000030FCF72DBAFBF743FF002601202E8064
:1089E000FBF73EFF414B42481E7004F03FF82368FE
:1089F0006193619BC8F80030FCF71ABA3046FBF768
:108A00002FFF0A2301202B80FBF72AFF374B384822
:108A10001E7004F02BF823685F935F9BC8F800304A
:108A2000FCF706BA0120FBF723FD304B3048002449
:108A30001C7004F01BF818202C70F8F76BF82F4B03
:108A4000198888423CF4F4A91820F8F757F8FCF785
:108A5000EFB90020FBF70CFD284A1388012B94BFC7
:108A60000133002301201380FBF702FD1F4B204838
:108A700000221A7003F0FAFF23687B937B9BC8F8EF
:108A80000030FCF7D5B90120FBF7F2FC174B184872
:108A900000241C7003F0EAFF18202C70F8F73AF855
:108AA000164B198888423CF4C3A91820F8F726F819
:108AB000FCF7BEB90020FBF7DBFC104A1388002B43
:108AC0007FD0013B13800120FBF7D2FC074B084805
:108AD00000221A7003F0CAFF23687A937A9BC8F8C1
:108AE0000030FCF7A5B900BFAA9DFF1F909EFF1F95
:108AF000049FFF1F5C9DFF1F989EFF1F289EFF1F66
:108B00000120F7F7BFFFB14BB14800241C7003F000
:108B1000ADFF52202C70F7F7FDFFAE4B198888424D
:108B20003CF486A95220F7F7E9FFFCF781B9012050
:108B3000F7F7A8FFA54BA64800241C7003F096FF8A
:108B400052202C70F7F7E6FFA24B198888423CF4BC
:108B50006FA95220F7F7D2FFFCF76AB90020F7F7A8
:108B600091FF9C4A13880BB1013B13800120F7F75A
:108B700089FF964B964800221A7003F077FF23680E
:108B80009893989BC8F80030FCF752B90020F7F78B
:108B900079FF904A1388032B98BF01334FF00100EF
:108BA00098BF1380F7F76EFF884B894800221A7030
:108BB00003F05CFF23689993999BC8F80030FCF799
:108BC00037B9022313807EE7834D297800293DD0F1
:108BD0002368DFF820829A9380499A9BD8F8000096
:108BE00009681B1A8B4210D9784B1978012918BFD4
:108BF00001221A701878F7F763FF754803F036FF03
:108C000023689B939B9BC8F80030754A1378002B10
:108C10003CF40EA9734B1B680021013B1170072B1C
:108C20003CF606A901A252F823F000BFC19500004E
:108C300093950000314E00005D950000314E00001C
:108C4000314E0000314E00002F950000664D236824
:108C50002A78DFF8A081002A3AD09E935F4A9E9B33
:108C6000D8F8000012681B1A934211D9574B1A7892
:108C7000012A16BF012219701A701878FAF77EFBC4
:108C8000534803F0F3FE23689F939F9BC8F800307E
:108C9000534A1378002B3CF4CBA8524B1B6800219D
:108CA000013B1170072B3CF6C3A801A252F823F038
:108CB000899200005B920000314E00002992000072
:108CC000314E0000314E0000314E0000FB9100009B
:108CD000A2934249A29BD8F8000009681B1A8B4254
:108CE00012D93A4B1978012918BF01221A703F4A4C
:108CF00019781078F7F772FE354803F0B7FE23684D
:108D0000A393A39BC8F80030354A1378002B3CF49A
:108D10008FA8344B1B680021013B1170072B3CF6D8
:108D200087A801A252F823F09991000091910000C8
:108D3000314E00004F910000314E0000314E0000D6
:108D4000314E000043910000294D2978002953D06D
:108D50002368DFF8A08084932049849BD8F8000022
:108D600009681B1A8B4210D9184B1978012918BFB2
:108D700001221A701878FAF74BFD154803F076FEB9
:108D800023688593859BC8F80030154A1378002B1B
:108D90003CF44EA8134B1B680021013B1170072BBC
:108DA0003CF646A801A252F823F000BF0D91000046
:108DB000B7900000314E000081900000314E00005D
:108DC000314E0000314E000053900000909EFF1F76
:108DD000049FFF1F948AFF1FE09EFF1F908DFF1FBF
:108DE000FC9DFF1F949EFF1FE19EFF1F488AFF1FEF
:108DF000C99DFF1F409EFF1FBA4D23682A78DFF8E8
:108E00000883002A3AD08893B74A889BD8F8000094
:108E100012681B1A934211D9B44B1A78012A16BF53
:108E2000012219701A701878FBF7ACFAB04803F0F9
:108E30001DFE23688993899BC8F80030AD4A1378DA
:108E4000002B3BF4F5AFAC4B1B680021013B1170CC
:108E5000072B3BF6EDAF01A252F823F01D90000066
:108E6000EF8F0000314E0000238F0000314E0000D4
:108E7000314E0000314E0000F58E00008C939A496F
:108E80008C9BD8F8000009681B1A8B4212D9974BAB
:108E90001978012918BF01221A70984A1978107898
:108EA000F7F79CFD924803F0E1FD23688D938D9BBD
:108EB000C8F800308F4A1378002B3BF4B9AF8E4BC3
:108EC0001B680021013B1170072B3BF6B1AF01A2DB
:108ED00052F823F0AD8F0000A58F0000314E000046
:108EE000638F0000314E0000314E0000314E000013
:108EF000598F00000120FBF745FA7C4B7C48002489
:108F00001C7003F0B3FD32202C70F7F703FE7C4B8E
:108F1000198888423BF48CAF3220F7F7EFFDFBF75E
:108F200087BF774D2B88172B3BF682AF0020FBF7CE
:108F300029FA2B88012003442B80FBF723FA6B4B83
:108F40006B4800221A7003F091FD23688B938B9B72
:108F5000C8F80030FBF76CBF01233B703370FBF7A0
:108F600067BF664C207801287BF662AF0021F7F7D7
:108F700035FD23785D4D013BDBB21846012123709E
:108F8000F7F72CFD002434238DE8180058482C7086
:108F900040230B223F2102F04BFD554803F066FDB4
:108FA000FBF746BFFBF756FBFBF742BF534C20785D
:108FB00005283BF63DAF0021F7F710FD23784B4D18
:108FC0000133DBB2184601212370F7F707FD0024B7
:108FD00034238DE8180046482C7040230B223F2193
:108FE00002F026FD424803F041FDFBF721BF0120BE
:108FF000FBF7C8F93D4B3E4800241C7003F036FDDA
:1090000032202C70F7F786FD3D4B198888423BF4DF
:109010000FAF3220F7F772FDFBF70ABF384D2B88F0
:10902000002B3BF405AF0020FBF7ACF92B880120A7
:10903000013B2B80FBF7A6F92C4B2D4800221A7020
:1090400003F014FD23688A938A9BC8F80030FBF76D
:10905000EFBE0120FAF7DCFB244B254800241C70EE
:1090600003F004FD20202C70F7F754FD254B1988E0
:1090700088423BF4DDAE2020F7F740FDFBF7D8BE79
:10908000204D2B88452B3BF6D3AE0020FAF7C0FBD2
:109090002B88012003442B80FAF7BAFB134B1448AA
:1090A00000221A7003F0E2FC23688793879BC8F8BC
:1090B0000030FBF7BDBE0120FAF7AAFB0B4B0C48B2
:1090C00000241C7003F0D2FC20202C70F7F722FD46
:1090D0000C4B198888423BF4ABAE2020F7F70EFD0D
:1090E000FBF7A6BE9E9DFF1F908DFF1F909EFF1F4A
:1090F000049FFF1FFC9DFF1F949EFF1F548AFF1FAC
:10910000CE9EFF1FDE9EFF1F409EFF1FC14D2B887E
:10911000002B3BF48DAE0020FAF77AFB2B88012060
:10912000013B2B80FAF774FBBB4BBC4800221A7042
:1091300003F09CFC23688693869BC8F80030FBF7FD
:1091400077BE5A2201233A703370FBF771BEB44CDC
:10915000207801287BF66CAE0021F7F73FFC2378DE
:10916000AD4D013BDBB2184601212370F7F736FC09
:10917000002434238DE81800A8482C7040230B22CB
:109180003F2102F055FCA54803F070FCFBF750BEF0
:10919000FAF752F9FBF74CBEA14C207804283BF6B5
:1091A00047AE0021F7F71AFC23789B4D0133DBB261
:1091B000184601212370F7F711FC002434238DE8B1
:1091C000180096482C7040230B223F2102F030FCFF
:1091D000924803F04BFCFBF72BBE5E1A5C2303FBAB
:1091E00006F393FBF2F61B36FEF785BC02FB03F396
:1091F00093FBF5F21144FEF75FBC0120FAF7BEF8CD
:10920000854B864800241C7003F030FC56202C70DF
:10921000F7F780FC834B198888423BF409AE56204F
:10922000F7F76CFCFBF704BE0020FAF7A7F87D4ABD
:109230001388B3FA83F35B0901201380FAF79EF8D1
:10924000754B764800221A7003F010FC2368A19336
:10925000A19BC8F80030FBF7EBBD0120FAF78EF8B0
:109260006D4B6E4800241C7003F000FC56202C70DF
:10927000F7F750FC6B4B198888423BF4D9AD562068
:10928000F7F73CFCFBF7D4BD0020FAF777F8654A06
:109290001388B3FA83F35B0901201380FAF76EF8A1
:1092A0005D4B5E4800221A7003F0E0FB2368A09338
:1092B000A09BC8F80030FBF7BBBD0120FAF700F80F
:1092C000554B564800241C7003F0D0FB14202C7022
:1092D000F7F720FC544B198888423BF4A9AD1420C1
:1092E000F7F70CFCF7F7BAFFFBF7A2BD0020F9F780
:1092F000E7FF4D4A1388B3FA83F35B09012013801B
:10930000F9F7DEFF444B454800221A7003F0AEFB2C
:1093100023686593659BC8F80030FBF789BD012081
:10932000F9F7CEFF3C4B3D4800241C7003F09EFB38
:1093300014202C70F7F7EEFB3B4B198888423BF466
:1093400077AD1420F7F7DAFBF7F788FFFBF770BD6E
:109350000020F9F7B5FF344A1388B3FA83F35B09A9
:1093600001201380F9F7ACFF2B4B2C4800221A7018
:1093700003F07CFB23686493649BC8F80030FBF720
:1093800057BD0120F7F760FB234B244800241C70D5
:1093900003F06CFB50202C70F7F7BCFB234B1988B3
:1093A00088423BF445AD5020F7F7A8FBFBF740BDE2
:1093B0001E4D2B880B2B3BF63BAD0020F7F744FBF3
:1093C0002B88012003442B80F7F73EFB124B1348F8
:1093D00000221A7003F04AFB23689593959BC8F806
:1093E0000030FBF725BD0120F7F72EFB0A4B0B4899
:1093F00000241C7003F03AFB50202C70F7F78AFB16
:109400000A4B198888423BF413AD5020F7F776FBDE
:10941000FBF70EBDDE9EFF1F909EFF1F049FFF1FE8
:10942000488AFF1FFE9DFF1F1A9EFF1FB88CFF1F5B
:10943000714D2B88012B7BF6FBAC0020F7F704FB6A
:109440002B880120013B2B80F7F7FEFA6B4B6C4811
:1094500000221A7003F00AFB23689493949BC8F8C7
:109460000030FBF7E5BC0120F9F7D8FA634B6448FC
:1094700000241C7003F0FAFA1E202C70F7F74AFB48
:10948000604B198888423BF4D3AC1E20F7F736FBBB
:10949000FBF7CEBC5B4D2B88082B3BF6C9AC0020FC
:1094A000F9F7BCFA2B88012003442B80F9F7B6FAB0
:1094B000524B534800221A7003F0D8FA2368919354
:1094C000919BC8F80030FBF7B3BC0120F9F7A6FA6E
:1094D0004A4B4B4800241C7003F0C8FA1E202C7025
:1094E000F7F718FB474B198888423BF4A1AC1E20C4
:1094F000F7F704FBFBF79CBC424D2B88002B3BF499
:1095000097AC0020F9F78AFA2B880120013B2B80C9
:10951000F9F784FA394B3A4800221A7003F0A6FA98
:1095200023689093909BC8F80030FBF781BC012022
:10953000F7F7C6FA314B324800241C7003F096FA54
:1095400054202C70F7F7E6FA2F4B198888423BF429
:109550006FAC5420F7F7D2FAFBF76ABC2A4D2B8880
:109560001D2B3BF665AC0020F7F7AAFA2B880120EB
:1095700003442B80F7F7A4FA204B214800221A70ED
:1095800003F074FA23689D939D9BC8F80030FBF7A5
:109590004FBC0120F7F794FA184B194800241C70AF
:1095A00003F064FA54202C70F7F7B4FA164B1988BC
:1095B00088423BF43DAC5420F7F7A0FAFBF738BCE7
:1095C000114D2B88012B7BF633AC0020F7F778FA8E
:1095D0002B880120013B2B80F7F772FA074B0848D4
:1095E00000221A7003F042FA23689C939C9BC8F8EF
:1095F0000030FBF71DBC00BFB88CFF1F909EFF1F03
:10960000049FFF1FC09DFF1FBA8CFF1F2DE9F04F65
:109610000E2093B003F0A2FC06F0BCFE0146AD485C
:10962000AD4FAE4E02F0B6F8AA4802F089F807F046
:10963000E1F83D6880F30C00012D306000F085807A
:10964000022DDFF808B300F09181032D00F00F82A6
:10965000A34CA44DDFF8F892DFF8F8822368A24FFC
:109660000E930E9B3A689B1A022B1ED9DFF8E8A2D4
:109670009AF80030002B00F0BE829C4B1A78002A2A
:109680000CBF012200221A7000F0B8829AF8003054
:10969000002B40F0B882F7F7DFFEF7F70FF8F7F787
:1096A000F9FD23680F930F9B3B602368904F109345
:1096B000904A109B396812685B1A93422DD8336820
:1096C000BBF800002A68C9F800208342B8F80020DF
:1096D00014DA101AB0F5805F4FF0000318DAC3EB0C
:1096E000033393FBF0F0F6F7FBFE0146282004F06D
:1096F000D1F8FBF7F7FA13B0BDE8F08F9342D4BF6F
:10970000C0EB0303C0EB0203101AB0F5805FE6DB89
:109710001A03013092FBF0F0E5E7F8F7ABF8764B6F
:109720001B7823B9754B1B78002B00F0F5810D20B9
:1097300004F0C4F9B0FA80F149090D2004F0B8F939
:1097400023681193119B3B60B9E7DFF810A26C4AC4
:10975000BAF800301178994209D0DBB21370002BAF
:1097600000F00C82102BA8BF1023664A1360DFF8AC
:10977000F081654AB8F800301178994204D0634C02
:109780002178002940F0EA81DFF8C0B1544CBBF8E1
:109790000030834280F2BA8122685D4B09920999B8
:1097A0005C4A1960022310603B605B4B187838BB41
:1097B0005A4B1B7823BB5A4B1F68002003F0CEFB8B
:1097C000A7F21F37874202DC564B00221A70002096
:1097D00004F09CFB544B554D1A682978544F904225
:1097E000D4BF002301238B423B7002D0904200F390
:1097F0003A832B70DFF858913A4DDFF858812DE706
:109800004C4BDFF860911F88B9F80020DFF858E171
:109810001744DEF800207F109742474A05DA1168A6
:109820008F4202DA002840F0598303933C4B0292A6
:109830001F460020CDF810E0019303F08FFB3F6836
:10984000029A039BA7F5487E704580F299813348C0
:109850000078002800F094811888DDF810E0B9F84D
:109860000030DEF80010126803445B108B4280F277
:109870008D81934240F38A81F6F782FF2F49086871
:10988000421C002A40F35085802A00F34C852C4D61
:109890002C4B2D4F2D881B880A6039682B44B1EB67
:1098A000630FC1F24B80A0F148030F2B00F2A0819F
:1098B000A0F1470300210D20AAF8003004F0F8F8C9
:1098C000962004F031F901210D2004F0F1F8019BFC
:1098D0001F6872E7709EFF1FC89EFF1FB09EFF1F8C
:1098E000409FFF1FF89EFF1F489EFF1FC89DFF1F40
:1098F0000C9EFF1FF88BFF1F209EFF1FA99EFF1FBE
:10990000379EFF1F049EFF1FF69DFF1F9D9DFF1F9B
:10991000F09DFF1F649EFF1FC29DFF1F1C9EFF1F27
:10992000709DFF1FDD9EFF1F548CFF1F599DFF1F61
:10993000BF9DFF1FBC9DFF1F009FFF1FF89DFF1FC6
:10994000969DFF1F4E9EFF1FC49DFF1F1E9EFF1F63
:10995000249EFF1FEC9EFF1FE29EFF1F609EFF1FC5
:109960006C9EFF1F349EFF1FD09DFF1FBBF8003071
:10997000984240F3EB80A54CA54923680A93A54A79
:109980000A9B096812885B1A934202D8002A7FF466
:1099900060AEF6F7F5FEA04A33681168BBF8002008
:1099A000DFF8C4828B42B8BF0B469342B8F8000080
:1099B0009A4980F23C869A4B09881A60002900F087
:1099C0000983984B04931970974DF7F7DFFC2868CB
:1099D0007F2840F33986954B7F3883FB0032C317CD
:1099E000C3EB620303EB4303A0EB83007330904BA4
:1099F00002931B882860002B40F08A878D4B0193CF
:109A00001B78002B00F0BC838B4B19461B78002B76
:109A100000F0B6834FF0000A0394CDF81480DFF80D
:109A20002092049CD0468A460CE003F17300C0B239
:109A30002178F7F791FE9AF8003008F101084345C4
:109A400040F39B832B6859F8040F784A1844A0F11F
:109A50007F0382FB032ED917C1EB6E0101EB41019D
:109A60007F28A3EB8103E0DCF6F728FDDFE7BBF8F6
:109A70000030984280F2FC80704B1B78002B40F045
:109A8000F780DFF8E8A19AF800007F2800F39282BF
:109A9000F6F714FD664B02931B88C0B28AF80000EB
:109AA000002B40F0C586634B01931B78002B00F020
:109AB000D082614B19461B78002B00F0CA82604CA3
:109AC0005A4D4FF0000889460BE003F17300C0B215
:109AD000F7F752F899F8003008F10108434540F3D0
:109AE000B88254F8043F9AF800001844A0F17F03AC
:109AF00085FB0321DA17C2EB610202EB42027F28E9
:109B0000A3EB8203E1DCF6F7D9FCE0E74B4B1B78D3
:109B1000002B3FF44AAE3FE6464B1B78002B7FF408
:109B200006AE484B1B78002B7FF401AE434B1B78ED
:109B3000002B7FF4FCAD0D2003F0C0FF00287FF464
:109B4000FFAD01210D2003F0B3FFF9E53B4B1B787E
:109B5000002B7FF410AF01233B6079E5DBB21846A0
:109B60001370F6F7E7FF334B374A30681946002386
:109B70001370344A23700B70137005E62B46F4E51E
:109B80001988B9F8003012680B445B109342BFF695
:109B900014AE002003F0E2F9019B1F68A7F548739B
:109BA0009842BFF60AAE294B1A78002A7FF405AE18
:109BB000274F01251D70F6F7E3FD3B78002B40F0A1
:109BC000FA84244B1B78002B40F0C386224B1B7871
:109BD000002B00F04B87214B1B784BB9204B1B7897
:109BE00033B1B8F800301F4A0A33A8F800301570B6
:109BF000019B1F68E1E5F7F7C9FB3EE5F7F74CF875
:109C0000F7F762FD4DE5F7F7C1FB44E5409FFF1F05
:109C1000F09DFF1FBC9EFF1F649EFF1F5C9DFF1FEA
:109C2000D89EFF1F009EFF1FF89EFF1FABAAAA2A07
:109C3000CA9DFF1FE39EFF1F008BFF1FA89DFF1FF4
:109C4000D88AFF1F5B9DFF1FA99EFF1FDD9EFF1F80
:109C5000449EFF1FC49EFF1F2C9FFF1F2D9FFF1FB1
:109C60002E9FFF1F9D9DFF1FEC9EFF1FA89EFF1FA5
:109C70009C4DDFF8CC92F6F783FD2868D9F80030C8
:109C8000984200F05184984C984B22680B920B9AA2
:109C90001A6023680C9396490C9B09889B1A8B4287
:109CA00040F2D2807F2840F34684924B7F3883FB7A
:109CB0000032C317C3EB620303EB4303A0EB830043
:109CC0007330DFF880A29AF80030834200F0BC8045
:109CD000894A1288002A00F0BF84DFF86C827F2B4B
:109CE00040F38F8583487F3B80FB0320DA17C2EB6C
:109CF000600000EB4000A3EB800073307F4B0193CA
:109D00001B78C0B28AF80000002B40F0F3847C4B33
:109D100005931B78002B40F054867A4B03931B78F5
:109D2000002B40F0B886784B0293039B1B7883B3DB
:109D3000764B9AF800001B6818447F2840F362862F
:109D40006C4B7F3883FB0032C317C3EB620303EB1A
:109D50004303A0EB83007330C0B2F6F70DFF6C4AEB
:109D60006C4B12789AF8000053F8223018447F2880
:109D700040F344865F4B7F3883FB0032C317C3EB4D
:109D8000620303EB4303A0EB83007330C0B2F6F72A
:109D9000F3FE019B1B78002B00F0C185029B5A4FFC
:109DA0001B880493002B00F0F88528687F2840F377
:109DB0004F84504B7F3883FB0032C317C3EB6203E1
:109DC00003EB4303A0EB83007330049B2860002B5C
:109DD00040F0D685019B1B78002B00F0E7824E4BAC
:109DE00019461B78002B00F0E1824C4B4C4A04943E
:109DF0000027CDF818A0CDF81C801C46B846924626
:109E00000F460CE003F17300C0B29AF80010F7F7A8
:109E1000A3FC3B7808F10108434540F3C2822B685C
:109E200054F8040F334A1844A0F17F0382FB032E39
:109E3000D917C1EB6E0101EB41017F28A3EB810330
:109E4000E0DCF6F73BFBDFE7DFF8FC80BBF8002047
:109E500033689A42BFF602AC23680D93314B0D9ADA
:109E60001A60FFF7FBBBF6F78BFC2F4B1978002924
:109E70006CD12E4B1B7843B1204A01921278002AF4
:109E800000F0E484019800220270294A1278002A26
:109E90007BD1002940F07482002B40F0718225496B
:109EA000164891F800E016490591164903911449A6
:109EB000214A0B7013490190137003700B70BEF1AF
:109EC000000F00F02E8300211170019A3B78117071
:109ED000039F059A0120387011708AE4174B019393
:109EE000CAE400BFF89EFF1F409FFF1F689EFF1F30
:109EF000DE9EFF1FABAAAA2A5C9DFF1FE39EFF1FE9
:109F00005B9DFF1F209EFF1FCA9DFF1F048BFF1F2D
:109F1000019EFF1F448CFF1F008BFF1FD88AFF1F6D
:109F2000009EFF1F409EFF1F2E9FFF1FD59EFF1FFD
:109F3000C49EFF1F9C9DFF1FA99EFF1F709DFF1FBA
:109F4000249EFF1FA89EFF1FEC9EFF1FB84A92F899
:109F500000C0BCF1000F40F08A84B6480190B648BA
:109F6000B64B0390B3481B7880F800C0B2484FF05E
:109F7000010E80F800C082F800E0002B40F06984F8
:109F8000AF4B1B78002B00F0FB81AE4B05931946BD
:109F90001B78002B40F0F181AB4AA7481278037080
:109FA000012303900B70002A00F0BB82A14BA04A52
:109FB000019388E7A3F155337F3803F1004383FB16
:109FC0000032C317C3EB620303EB4303A0EB830030
:109FD00073305FE513469842D4BFC2EB0001C2EB79
:109FE0000301821AB2F5804FAABF8903C1EB813108
:109FF000013291FBF2F0F6F773FAC0F3C61006F0E7
:10A00000C9F9924B0546188806F0C4F99049814673
:10A01000284606F013FA0146484606F00FFA29468C
:10A0200006F004F94FF07E51054606F0A5FB002826
:10A0300040F006858749284606F0BCFB002840F022
:10A04000E884284606F0FCFBC0B2834B04931870EA
:10A05000BAE47C4B1B78002B45D09AF80030A3F172
:10A060000C007F2840F307847C4A8B3B82FB032152
:10A07000DA17C2EB610202EB4202A3EB820303F1A7
:10A080007300C0B2F6F778FD019B1B785BB3744B8D
:10A0900019461B783BB3734C704D4FF0000889464E
:10A0A0000AE003F17300C0B2F6F766FD99F80030DC
:10A0B00008F10108434516DD54F8043F9AF80020E2
:10A0C0001A44A2F18B0385FB0310D917C1EB600181
:10A0D000A2F10C0001EB41017F28A3EB8103E0DC3E
:10A0E000F6F7ECF9DFE7544B1B7883B35E4B9AF835
:10A0F00000001B6818447F2840F3C383574B7F3808
:10A1000083FB0032C317C3EB620303EB4303A0EBF3
:10A1100083007330C0B2F6F72FFD544A544B1278C7
:10A120009AF8000053F8223018447F2840F3A683A1
:10A130004A4B7F3883FB0032C317C3EB620303EB48
:10A140004303A0EB83007330C0B2F6F715FD029B0A
:10A150001B88002B00F07583354B1B78002B40F0DB
:10A160006B83444B444C454DDFF81491DFF8148168
:10A1700000221A6001233B6068E6039CDDF814802E
:10A180002B4B1B78002B40F0B8832B682D4A12789C
:10A19000002A7DD0A3F10C007F2840F3D7832F48FD
:10A1A0008B3B80FB0320DA17C2EB600000EB400022
:10A1B000A3EB800303F17300049BC0B21978F7F797
:10A1C000CBFA019B1B78002B61D0254B19461B78DD
:10A1D000002B5CD04FF0000A0194CDF80C80DFF822
:10A1E0008490049CD0468A460BE003F17300C0B211
:10A1F0002178F7F7B1FA9AF8003008F101084345E1
:10A2000042DD2B6859F8041F144A1944A1F18B034D
:10A21000D81782FB032EC0EB6E0EA1F10C000EEBE3
:10A220004E0E7F28A3EB8E03DFDCF6F747F9DEE75F
:10A23000A99EFF1FE39EFF1F209EFF1FD59EFF1FAD
:10A24000C49EFF1F5B9DFF1F9C9DFF1F689DFF1FFE
:10A25000CDCCCC3D0000FE42009EFF1FABAAAA2A37
:10A26000008BFF1FD88AFF1F048BFF1F019EFF1F5B
:10A27000448CFF1FD89EFF1F409FFF1FF89EFF1FAB
:10A28000249EFF1FEC9EFF1F019CDDF80C802B68B5
:10A29000AB4A1278002A39D0AA4A106818447F289D
:10A2A00040F35183A84AA0F17F0382FB0320DA1711
:10A2B000C2EB600000EB4000A3EB80007330049B16
:10A2C000C0B21978F7F748FAA0490B78022B9ABF69
:10A2D0005A1CD2B200220A709D492B6851F8220004
:10A2E00018447F2840F32C83974B7F3883FB003240
:10A2F000C317C3EB620303EB4303A0EB830073308C
:10A30000049BC0B21978F7F727FA2B68029A1288D3
:10A31000002A00F0EB828F4ADFF874921370032357
:10A320003B60FFF79BB980258B4A8C4B10888C4A89
:10A330001B8812680D600344B2EB630FBFF658AC84
:10A34000884B1978002940F06182B8F80030864ABD
:10A35000AB423FF44DAC854B158001250D201D709F
:10A3600003F0A6FB962003F0DFFB29460D2003F047
:10A370009FFB019B1F68FFF720BA059A002313700B
:10A38000784B1B78002B00F0CC806D4B03931B782F
:10A39000002B00F0878303993B7800220A70FFF7B7
:10A3A00028BA049CDDF818A0DDF81C80059B1B78FA
:10A3B000002B52D02B68A3F10C007F2840F31583AB
:10A3C000614A8B3B82FB0321DA17C2EB610202EB8D
:10A3D0004202A3EB820303F17300654B04931978E7
:10A3E000C0B2F7F7B9F901990B78B3B361490B78AB
:10A3F0009BB3614806940027CDF81CA00446DDF805
:10A4000010A0CDF81080B8460F460BE002F17300A3
:10A41000C0B29AF80010F7F79FF93A7808F10108EE
:10A42000424515DD2A6854F8040F474B1044A0F14B
:10A430008B0283FB023ED117C1EB6E010C3801EB9E
:10A4400041017F28A2EB8102E0DCF6F737F8DFE775
:10A45000069CDDF81CA0DDF81080039B1B78002B08
:10A4600039D0384B28681B6818447F2840F3C382D2
:10A47000354B7F3883FB0032C317C3EB620303EB1A
:10A480004303A0EB83007330394B04931978C0B2B7
:10A49000F7F762F92D490B78022B9ABF5A1CD2B2FA
:10A4A00000220A702A492B6851F8220018447F289C
:10A4B00040F39E82244B7F3883FB0032C317C3EBEB
:10A4C000620303EB4303A0EB83007330049BC0B231
:10A4D0001978F7F741F9029B1B88002B00F057828F
:10A4E000019B1B783BB9059B1B7823B9039B1B7809
:10A4F000002B00F01983214B1B78D3B11D490B7839
:10A50000082B16D81E482A6800681E4F0133DBB29C
:10A5100003F1FF3E101A47F82E000B708AF8002056
:10A5200094E43B78FFF765B9174B184C1A68FFF7AE
:10A53000B0BB2A68F2E7F5F7C1FFFFF7C2BB00BF67
:10A54000209EFF1F048BFF1FABAAAA2A019EFF1F9C
:10A55000448CFF1FA89EFF1F4E9EFF1F969DFF1F4E
:10A56000C49DFF1F9C9DFF1F6C9EFF1F9D9DFF1F95
:10A57000009EFF1F008BFF1FD88AFF1FA99EFF1F91
:10A58000A09DFF1FDC8AFF1F689EFF1F409FFF1FCB
:10A59000249EFF1FBC4B1B78002B7FF429ABBB4BC9
:10A5A000BB4A1B78243B83F3470319465B201360A7
:10A5B000F6F712FE3B78032B7FF41AABB54D2A78E1
:10A5C000002A40F0A682B44F3B78002B40F09582E1
:10A5D000DFF8B48298F80030002B40F08282AF4B55
:10A5E0001B78002B40F07182AD4A1380AD4B1B7875
:10A5F000002B40F05E82AC4B7F221A802B78002B20
:10A600007FF4F6AA3B78002B7FF4F2AA98F800308A
:10A61000002B7FF4EDAAA54A7F2107201380F6F7CF
:10A62000DBFD7F210B20F6F7D7FDFFF7E1BAA04D48
:10A6300009888342A8BF03462B6000297FF4C1A983
:10A640009A423FF7CEACC6E4F5F738FFFFF7CFB933
:10A65000F5F734FFFFF7B9BB9549BBF800000F6869
:10A66000DFF884828742B8F8001005DB8F42D4BF40
:10A67000C0EB0702C0EB0102081AB0F5804FAABF79
:10A680009203C2EB8232013092FBF0F00293F5F7B5
:10A6900027FFC0F3C61005F07DFE864A07461088E6
:10A6A00005F078FE84490190384605F0C7FE019A0E
:10A6B0000146104605F0C2FE394605F0B7FD4FF0E1
:10A6C0007E51074606F058F8029B002840F0E181D1
:10A6D0007A490193384606F06DF8019B002840F056
:10A6E000AD81384606F0ACF8019BC0B2744A1070D8
:10A6F000FFF7F5BA734B02931B88002B40F055818E
:10A70000714B0593714B0393714B1A461B7843B3FE
:10A71000704B0494002706951C463D46174608E0FA
:10A7200003F17300C0B2F6F727FA3B780135AB426C
:10A7300015DD54F8043F9AF80000674A1844A0F168
:10A740007F0382FB032ED917C1EB6E0101EB4101A0
:10A750007F28A3EB8103E3DCF5F7B0FEE2E7049C7E
:10A76000069D059B1B78002B3FF4DFAA9AF800306A
:10A77000A3F10C007F2840F34981574A8B3B82FBB1
:10A780000321DA17C2EB610202EB4202A3EB820360
:10A7900003F17300C0B2F6F7EFF9019B1B78002BB1
:10A7A00000F018814A4B19461B78002B00F0C68137
:10A7B000484B0494002706951C463D460F4609E089
:10A7C00002F17300C0B2F6F7D7F93A780135AA4220
:10A7D00040F3228154F8042F9AF800003E4B1044B5
:10A7E000A0F18B0283FB023ED117C1EB6E010C3846
:10A7F00001EB41017F28A2EB8102E1DCF5F75EFE6F
:10A80000E0E71846F5F75AFEFFF778BA4B2D40F30C
:10A8100007811835802DB8F80030304AA8BF802550
:10A82000AB423FF4E5A92E4B15800125002195E5AB
:10A83000F6F7A2F9FFF737B900214020F6F7CCFC74
:10A840008FE49AF80000F6F797F985E41F48254A47
:10A8500003904FF0000C82F800C00198039A4FF06B
:10A86000010E80F800E082F800C0FFF70EBB002365
:10A870001370FFF7FEBAF5F721FE02E4F5F71EFEAE
:10A8800062E4F5F71BFE45E42E9FFF1FF69EFF1FB7
:10A89000B89DFF1FC49EFF1F2D9FFF1F2C9FFF1FF2
:10A8A0001A9EFF1FD59EFF1F5C9DFF1F989EFF1FD6
:10A8B000D89EFF1F689DFF1FCDCCCC3D0000FE42FF
:10A8C000009EFF1FCA9DFF1F5B9DFF1F209EFF1F55
:10A8D000008BFF1FD88AFF1FABAAAA2A6C9EFF1FFE
:10A8E0009D9DFF1FA99EFF1FEC9EFF1F049AD8B2DB
:10A8F0001178F6F731FF2B680DE57F214020F6F740
:10A900006BFC9349934A2B680B60002111703DE466
:10A91000049BC0B21978F6F71FFFFFF76FB8059BCD
:10A920001B78002B7FF43AAA039B1B78002B7FF443
:10A9300035AA029B1B880493FFF737BA1546FFE43C
:10A94000F5F7BCFDDCE4F5F7B9FDB8E4F5F7B6FDC5
:10A9500032E4814B1B78002B75D0804B1B78002B89
:10A960007FF446A97E4B1B78002B3FF441A9B8F831
:10A9700000307C4A0A3BA8F800301570FFF738B960
:10A98000794BC0B21978F6F7E7FEFFF723BA764B9A
:10A9900028781978F6F7E0FEA2E59AF80000F6F7B5
:10A9A000EBF83B880493FFF700BA704B0593704BAC
:10A9B0000393F6F7E1F8019B1B78002B7FF4A4AE1C
:10A9C000CFE66C4B02931B88002B40F0BE80684B97
:10A9D0000393CBE6039B1B78002B7FF4A9A9059B6F
:10A9E0001B78002B7FF4DAA9A3E7F5F767FDF4E401
:10A9F000F5F764FD6AE5F5F761FD45E5F5F75EFD00
:10AA0000FFF7C4B9F5F75AFDFFF7A6B9F5F756FDFC
:10AA1000C0E67F20FFF719BB049C069DFFF785B9B0
:10AA2000243D002DB8F8003040F38380AB423FF462
:10AA3000DFA8ADB24B4BA8F80050F6E67F2055E6F4
:10AA40000120FFF702BB454B1B78002B7FF4D0A8F9
:10AA5000434B1B78002B3FF4CBA8B8F80030414A99
:10AA6000013BA8F800301570FFF7C2B83B4B1B78CC
:10AA7000002B7FF48FAD3A4B1B78002B3FF4B8A826
:10AA8000B8F80030374A0133A8F800301570FFF7E6
:10AA9000AFB801202AE6374B02931B88002B3FF406
:10AAA00044A986E7344B0193304B344A0593FFF7B2
:10AAB0000ABA334B00227F2107201A80F6F78CFB5D
:10AAC0007F210B20F6F788FB98E52E4B01227F2192
:10AAD00007201A80F6F780FB7F210B20F6F77CFB1E
:10AAE00084E5294B04227F2107201A80F6F774FBA6
:10AAF00000210B20F6F770FB71E5234B02227F212A
:10AB000007201A80F6F768FB7F210B20F6F764FB1D
:10AB10005EE51D4A002107201380F6F75DFB7F21CB
:10AB20000B20F6F759FB4EE59AF80000F6F724F8EB
:10AB3000E1E4012B3FF45CA801257BE7039B1B7834
:10AB4000002B7FF4F5A8FFF729B9094B039330E7F1
:10AB5000A09DFF1F008BFF1F2C9FFF1F2D9FFF1F1E
:10AB60002E9FFF1F9D9DFF1F009EFF1F5B9DFF1FD0
:10AB7000209EFF1FCA9DFF1FE39EFF1FA99EFF1F70
:10AB80005C9DFF1F1A9EFF1F989EFF1F00207047AD
:10AB900090F8392090F83800101A704790F8383043
:10ABA00090F839209A4205D95A1C034480F838207D
:10ABB000187E70474FF0FF30704700BF90F8383074
:10ABC00090F839209A4286BF1B18187E4FF0FF304C
:10ABD000704700BF704700BF38B50546B0F85E004B
:10ABE00090B195F85D301446C3F1210294420CD81F
:10ABF00005F13B001844224601F0D0FF95F85D3086
:10AC0000234485F85D30204638BD01201446287164
:10AC1000EEE700BFB0F85E306BB190F85D30202BEE
:10AC200007D8C218013380F85D30012082F83B104C
:10AC30007047012303710020704700BF0023426961
:10AC400080F8383080F8393080F85C3080F85D303A
:10AC500080F85E3080F85F3006CA30B40D68046951
:10AC600043662A4383660A60A370426990F86130A4
:10AC70001649146813441D7A5B7B01EBC5051B0262
:10AC80006D6803F4E06343F064032B6090F8623076
:10AC900013449D7CDB7D01EBC5011B02496803F475
:10ACA000E06343F064030B6021685368194205D0E8
:10ACB000036927225A70036904229A7103692022CA
:10ACC0005A71036980229A7030BC7047D03C0100F1
:10ACD00043690CCB12681A420CD0094B99420AD92D
:10ACE000084B9942036994BF1A220D225A700369D6
:10ACF00004229A717047036927225A70F7E700BF50
:10AD00007F1A06003F420F0010B50269D378DBB20C
:10AD1000D90604463DD510215806D17038D503F028
:10AD2000040303F0FF02002B51D03D49626E002363
:10AD30000B7084F85D30002A5BD0904794F85D304A
:10AD4000002B56D02369D0229A70236994F83B20B7
:10AD50001A712369012284F85C200222DA7010BD86
:10AD6000304B84F860009C424AD02F4B9C4252D01A
:10AD700094F8391013791F29DBB207D828480078D6
:10AD800020B16018013184F8391003760223D370A2
:10AD900010BD5906C3D4917801F0100101F0FF00F5
:10ADA0000029DDD013F001031ED194F85C1094F853
:10ADB0005D00884281BF4B1C091984F85C3091F812
:10ADC0003B3013712369D0229A702269DEE7236930
:10ADD00084F83920C0229A702369114A1979012117
:10ADE00011700222DA7010BDC023937022691379AA
:10ADF000CCE70122002384F85D2084F83B30A1E7F2
:10AE0000626994F86130094913440322187A02F008
:10AE10006FFC2269ACE7626994F861300449F3E79A
:10AE2000389FFF1F008EFF1F6C8EFF1F91AE00002A
:10AE30009DAE00000369DB7803F0200373B190F846
:10AE400060300133DBB2012B80F860301AD94269DF
:10AE500090F861301344187A02F0C6BC70B54269AC
:10AE600003F0FF0590F8613013440446187A02F0AD
:10AE7000BBFCA36E5BB184F8385094F83900BDE890
:10AE80007040184790F85F30002BE0D0704770BDDD
:10AE90000148FFF7CFBF00BF008EFF1F0148FFF73B
:10AEA000C9BF00BF6C8EFF1F2DE9F047374FDFF899
:10AEB000E0903B68026982B006460093DDF80080AE
:10AEC0000021A025D3789B065BD53B680193019BAD
:10AED000C8EB03030F2BF5D949B1102BF2D000209A
:10AEE0009070336980229A7002B0BDE8F087726971
:10AEF00096F8613013440521187A02F0EDFD72696D
:10AF000096F861301344012193F812A0504602F0E4
:10AF1000E3FD09240021504602F0CAFD2B46013B07
:10AF2000FDD10121504602F0C3FD2B46013BFDD16E
:10AF3000013CEFD1706996F8611001444FF4A072A2
:10AF40000C7A4B7B09EBC4011B02496803F4E063F4
:10AF500043F064030B6096F862300344997CDB7D18
:10AF600009EBC1011B02496803F4E06343F0640389
:10AF70000B60013AFDD13269D3789B064FF0010195
:10AF8000A3D4012002B0BDE8F08700BF409FFF1F9F
:10AF9000D03C0100F0B503691222DA70026993789F
:10AFA00003F0200385B004460D46002B5ED0B42389
:10AFB00093703C4922690B680093009E05E00B6882
:10AFC0000193019B9B1B042B42D8D37803F02003F1
:10AFD00003F0FF00002BF2D094F85D30002B31D04D
:10AFE0004FF0000E4FF0020C04EB0E0393F83B30D1
:10AFF00013710B680393039F206907E09B060DD52F
:10B000000B680293029BDB1B052B28D8C378DBB2AD
:10B0100003F0020202F0FF06002AEFD080F803C01E
:10B020002669F378DBB2DF0632462DD49F062BD596
:10B03000DB0731D40EF1010E94F85D305FFA8EFE1D
:10B040007345D1D800201DBB002384F85E3004E096
:10B050009070236980229A70042005B0F0BD86703C
:10B060002369802204209A7005B0F0BD03F0FF062A
:10B07000FFF71AFF10B9042005B0F0BD236984F86A
:10B080005F60B0229A7094E78023B3700420DAE7FF
:10B0900026698023B370D7E7BEF1000F0CBF0220F2
:10B0A0000320F6E7409FFF1F2DE9F04106690025C8
:10B0B000122780F8385080F83950F770D0F810C057
:10B0C0009CF802E00EF0200E88B004468846154633
:10B0D0001E46BEF1000F49D0B4238CF80230784BE5
:10B0E00021691A680092DDF800E006E01A68019212
:10B0F0000198CEEB0000042830D8C87800F020007A
:10B1000000F0FF070028F1D04FEA480242F00102A8
:10B11000D2B20A711A680292DDF808E0206906E0EE
:10B120001A6803920399CEEB010105292AD8C17848
:10B1300001F0020101F0FF070029F1D04FF0020CED
:10B1400080F803C02269D17811F0110722D12DBBFC
:10B15000002E0CBFA0238023937003E08F7023691F
:10B1600080229A70384608B0BDE8F0810EF0FF07E3
:10B17000FFF79AFE0028F5D0236984F85F70B022AB
:10B180009A70ACE787702369802238469A7008B0BD
:10B19000BDE8F081802393700027E3E7012D75D08F
:10B1A000A021917021690A79BE4667464FF0A80C2C
:10B1B0001A680492049805E01A680592059A121A12
:10B1C000052A4AD8CA7802F0020202F0FF08002AD3
:10B1D000F2D0CF702169CA78D2B212F0100F0846AF
:10B1E0005AD1920658D5013DEDB2012D49D0BEF19C
:10B1F0001F0F3BD90A79012DDAD11A680692069DF4
:10B2000005E01A680792079A521B052A46D8C278A9
:10B2100002F0020202F0FF01002AF2D00223C37002
:10B220002269D378DBB2D9063AD49B0634D5B02351
:10B23000BEF11F0F93703FD8226904EB0E03127901
:10B240001A760EF1010E5FFA8EFE16B12369802286
:10B250009A7084F839E0774684E781F802802369A0
:10B2600080229A70774684F839E07BE704EB0E027F
:10B2700091F8048082F818800EF1010E5FFA8EFEBC
:10B28000B9E781F802C021690846B0E7A8219170AA
:10B290002069BE460279B0E7774663E78170DEE752
:10B2A0001021A023D170013BFDD12269937803F0D6
:10B2B000F7037746937055E723691B79C5E700BF0D
:10B2C000409FFF1F0148FFF71FBD00BF008EFF1FFB
:10B2D0000148FFF719BD00BF6C8EFF1F704700BF0C
:10B2E00038B5144C037801225B000546204684F8EB
:10B2F0003B3084F85E2084F85D20FFF78BFC20460D
:10B300000021FFF747FE0B4C2978012320461A46FF
:10B31000FFF7CAFE0128F6D194F8383094F83920A6
:10B320009A4205D9E218013384F83830107E38BDCE
:10B33000FF2038BD008EFF1F38B51B4C037801225B
:10B340005B000546204684F83B3084F85E2084F894
:10B350005D20FFF75FFC20460021FFF71BFE124C2B
:10B360002978204601230222FFF79EFE0228F6D10B
:10B3700094F8382094F839108A420FD2531CDBB26B
:10B38000A018994284F83830007E0AD9234402324A
:10B390001B7E84F8382040EA032038BD4FF6FF704A
:10B3A00038BD40F47F4038BD008EFF1F0C2901D905
:10B3B000002070470231490001F0FE01FFF7BCBFD9
:10B3C00070B50C4C0378164601255B00204684F8C6
:10B3D0003B3084F85E5084F85D50FFF71BFC31462B
:10B3E0002046FFF717FC29462046BDE87040FFF7CE
:10B3F000D1BD00BF008EFF1FF8B505460F461646AB
:10B40000412421463A462846FFF7DAFF611C023400
:10B41000C9B232462846E4B2FFF7D2FF592CF0D128
:10B42000F8BD00BF38B504460D463548FFF706FCA9
:10B430006322802120462570FFF7C2FF012002F021
:10B4400073FB204600225E21FFF7BAFF20465D21F4
:10B45000FFF746FF242801D0002038BD20460622F1
:10B460000C21FFF7C9FF204601222B21FFF7A8FF7F
:10B47000204601222C21FFF7A3FF20460E222D217A
:10B48000FFF79EFF204600222E21FFF799FF20465E
:10B4900001222F21FFF794FF204605223021FFF7DC
:10B4A0008FFF204601223121FFF78AFF204600222C
:10B4B0003221FFF785FF204600223321FFF780FF6E
:10B4C000204600223421FFF77BFF20460022352151
:10B4D000FFF776FF204600225B21FFF771FF204631
:10B4E00010225C21FFF76CFF204620225D21FFF730
:10B4F00067FF20468F225E21FFF762FF012038BDE3
:10B50000008EFF1F10B4047F4160022CC26002D085
:10B5100010BC03F08BBC836810BC1847F0B4464BDA
:10B52000464A186BDC6A01791170454922790A7024
:10B530009A6A00790870002A46D05968C9688A4218
:10B540003ED82168CC8B240402F1FF3065D4C0F3CF
:10B550000E00C883C88B80B2C882196B0968C88B7B
:10B56000000452D4C2F30E00C883C88B002480B2FA
:10B5700012F1FF32C88218BF01229C62D96A2E489C
:10B5800009680D6800F12404A54236D00068C4683B
:10B5900014F0804F0C680D6815BF2488247802359C
:10B5A000013544F000440D604463196B254B097963
:10B5B0001970214912B1CA6A12791A70F0BC704729
:10B5C000521A9A620122D9E7586B196805681E4C15
:10B5D0000A63CC62CC682D681C4E24F0804403279B
:10B5E000B542CC6083F825701FD1037F4260022BE7
:10B5F000C2601ED0F0BC03F019BC016890F82400B2
:10B60000CC6840F000404863CFE7CC8BC2F3080021
:10B6100004F47E442043C883A7E7CC8BC0F3080022
:10B6200004F47E442043C88394E72B461146F0BCC3
:10B6300018478368F0BC1847D88EFF1F1F80004052
:10B640001C8000401B80004000000FFF05B500007B
:10B6500090E80C00F0B41C6859682568164F174E26
:10B6600029432160164D17491760D6601561116096
:10B67000417A154A5C180A3194F8244053F8215055
:10B6800002EBC40149680D60017A5C1803EB81018B
:10B69000247ECD6902EBC40149680D60817A581897
:10B6A00003EB810390F83000596B02EBC002F0BC51
:10B6B00053681960704700BF01401F000110003837
:10B6C0000110007800001F80D03C010038B504460E
:10B6D000104621700A491D4604F0B0FE01464FF0A5
:10B6E0007E5004F05FFF074904F0A8FEE56060604B
:10B6F0002561656102F0F6F9E061204638BD00BFC2
:10B70000DB0FC9400024744938B504461046217047
:10B7100009491D4604F092FE01464FF07E5004F0A8
:10B7200041FF064904F08AFEE560606025616561BD
:10B7300002F0D8F9E06138BDDB0FC940002474493C
:10B7400038B503780446032B20D8DFE803F01A1835
:10B750001002C168406904F067FD0D490546606844
:10B7600004F020FF0146284604F01CFF38BD0849BC
:10B77000406804F017FFE16804F060FE38BDC0685F
:10B7800038BDC168406904F04FFD38BD002038BDA8
:10B790000024744970B504460E4602F0A3F905462C
:10B7A000E069281A04F0F6FDE3682361E56166614B
:10B7B000A0610146606804F0F5FE0146A0601048F3
:10B7C00004F0F0FE04F0C6F903F066FE04F0D8FCC5
:10B7D000054601464FF07E5004F026FD616904F0F5
:10B7E0002DFE21690646284604F028FE0146304613
:10B7F00004F01CFDE0602046BDE87040FFF7A0BFEC
:10B80000000080BF704700BF2DE9F04F85B099461A
:10B81000BDF93870BDF83CA0BB1AC1EB090B002B79
:10B82000B8BF5B42BBF1000FB8BFCBF1000B5B456B
:10B830000D4616460093804648DC4D453A46334651
:10B840004CDC194613460A46C5EB09019B1A89B21E
:10B85000002B0CB2B8BF5B4204EBD474BE42ACBF49
:10B860004FF0FF3201224D45039102924FEA6404EA
:10B8700029DC9BB201930DE0D8F80070BF69B8478E
:10B88000019BE41AA3B21CB20135002C2DB211DBCE
:10B89000A94518DB009B5B452A4653463146404686
:10B8A000EADCD8F8002053469769294632464046DC
:10B8B000B847E5E7029A1644039AA94502EB030448
:10B8C00036B224B2E6DA05B0BDE8F08F4A462B4620
:10B8D000B94635464D4517461E46B2DD3046294627
:10B8E0003E464D4607468946AEE700BF10B40468A1
:10B8F0002469A44610BC604730B40468BDF8085001
:10B900000295A46BA44630BC604700BF30B4046805
:10B91000BDF808500295E46BA44630BC604700BFF8
:10B9200070B40468BDF90C60BDF81050039604951E
:10B93000246CA44670BC6047704700BF10B582B04D
:10B94000B0F90C2001910168009200220C6CB0F952
:10B950000A301146A04702B010BD00BF704700BFBB
:10B9600001F003010129C17506D0032904D0C28862
:10B9700003894281838170470289C3884281838120
:10B98000704700BF2DE9F0410568134E6F6986B01E
:10B99000B7420446BDF8308010D1013B13441BB2BE
:10B9A0000093CDF804800B46AD6A2046A847236873
:10B9B000DB6AB3420AD106B0BDE8F0810593049278
:10B9C0000391B84703A925680EC9E6E7204606B0EB
:10B9D000BDE8F041184700BF39B900002DE9F0413A
:10B9E0000568124E6F6986B0B7420446BDF83080D4
:10B9F0000FD1013BCDF804800B4400921BB2AD6A1D
:10BA00002046A8472368DB6AB3420AD106B0BDE8E6
:10BA1000F081059304920391B84703A925680EC9E4
:10BA2000E7E7204606B0BDE8F041184739B9000005
:10BA30002DE9F04F0568DFF858B06F6985B05F45B4
:10BA40000646BDF93890BDF83CA00C46904615D18D
:10BA50001F19BC420CDACDF800A0214601342D6A32
:10BA60004B464246304624B2A847BC423568F2DB1A
:10BA7000EB6A5B4507D105B0BDE8F08F0393B8478B
:10BA80003568039BE4E7304605B0BDE8F04F184742
:10BA900039B900002DE9F04387B099420546BDF958
:10BAA0003840BDF83C6025D0A24212D00768DFF8CC
:10BAB0008080D7F81490C14532D18DE850002846D7
:10BAC000BC6AA0472B68DB6A434524D107B0BDE8B8
:10BAD000F083994202DD08461946034628680E960F
:10BAE000C46B01335B1A1BB22846A44607B0BDE8FD
:10BAF000F0436047A24202DD134622461C462868F6
:10BB00000E96631C846B9B1A1BB22846A44607B092
:10BB1000BDE8F0436047284607B0BDE8F04318474A
:10BB2000059304920391C84703A92F680EC9C4E77F
:10BB300039B900002DE9F04FD0F800E0DFF890901F
:10BB4000DEF814B083B0CB450446BDF93080BDF8B3
:10BB500034A00D4617461E4631D1CDF800A0DEF8C0
:10BB600024B0294633463A462046D8472368CDF8C4
:10BB700000A008F1FF323A44D3F824B0294612B2AB
:10BB800033462046D8472368CDF800A02946D3F88D
:10BB900020B03A4643462046D8472068CDF800A05A
:10BBA000711E29444346056A09B23A462046A84711
:10BBB0002368DB6A4B4506D103B0BDE8F08FD84758
:10BBC000D4F800E0C9E7204603B0BDE8F04F1847BD
:10BBD00039B90000F0B4002401264FF6FF75094F73
:10BBE00007600471C475C48104824476C46186759B
:10BBF000067685824582C180028141818281F0BCC6
:10BC0000704700BFE43601002DE9F04F85B00668AB
:10BC1000BDF84450BDF93880CDF800800446019548
:10BC2000D6F848B00392BDF93C60BDF94070894632
:10BC30009A46D84723680195009742465146D3F863
:10BC4000488020463346C0472068039B0E930F95DB
:10BC5000856C4B463A4631462046AC4605B0BDE8B9
:10BC6000F04F60472DE9F04F87B01746BDF94040CF
:10BC700000912546E91D059344BF2B4603F10E01B3
:10BC80000268BDF8486053690294C91003912B49BA
:10BC9000BDF9444001968B42824645D1002C3CDDE3
:10BCA000029B3C445E1EB6B24FF0000923B20493DF
:10BCB00001364D46029B002B28DD059B002403EB3B
:10BCC000090806E0EDB22B0604F1010411D4A642E6
:10BCD0001CD0A1B211F0070F23B24FEA4505F1D1F4
:10BCE000002BB8BF0733DB10013418F803502B06C4
:10BCF000EDD5009BD2F818B019443A4609B2019B21
:10BD00005046D847A642DAF80020E2D1039B01371B
:10BD10009944049B3FB2BB42CCD1D36A074A9342B9
:10BD200006D107B0BDE8F08F9847DAF80020B5E7F4
:10BD3000504607B0BDE8F04F184700BF39B90000C2
:10BD400070B4BDF90C60BDF91050BDF814400396F5
:10BD50000495059470BCFFF785BF00BF2DE9F04F37
:10BD600093B090460591C1691090BDF8700007909E
:10BD7000BDF874909DF878A00493002900F0CD8060
:10BD80000A7A0AC9894604998A1AD2B203EBC20315
:10BD9000BAF1010FDA780B9293F905201E8893F817
:10BDA00002B00F9293F9064079D913B2099323B2E6
:10BDB0000C93109B1A68A94B1193194653698B4237
:10BDC00040F0A6800B9B002B55D01FFA88F3002172
:10BDD0000D93C8462344DDF8409006910E930F461C
:10BDE0000C46BBF1000F3FD0BDF818100C9B039719
:10BDF0001FFA8AF0CB1813FB00F304900E9801444D
:10BE00000D98034409B21BB20A910893002505E07E
:10BE10000135EBB264009B45E4B222D9039B2B446D
:10BE2000590703D1731C18F806409EB22306EFD5BC
:10BE3000099BBDF81000E91811FB00F10598BAF153
:10BE4000010F0FFA8AF301441CD007980190009368
:10BE5000D26909B217464846089AB847D9F800206F
:10BE6000D6E7039F5F44FFB2069B0B99013306930D
:10BE7000DBB29942B5D8D36A119A934243D113B039
:10BE8000BDE8F08F0F9B191893690A9A29441F4641
:10BE900009B2079B4846B847D9F80020B8E7002305
:10BEA0000C93099385E70A9A0D9B0132013B52B22C
:10BEB00013F0FF030A920D936FD1DDF81890079BE2
:10BEC000DDF83C80DDF820A04B4517D0BAF1010F1A
:10BED00000F0C8800B9A109DCDF804900BEB8B01FD
:10BEE0004FEACB030A4400931146DEF81C40534648
:10BEF000424609B22846A047D5F800E0DEF82C30CB
:10BF0000119A9342BBD0109813B0BDE8F04F184778
:10BF1000109D284698472A6854E7109A0598B2F968
:10BF20000A308342ABDDB2F90C304345A7DD06236E
:10BF300013FB0A03002BA2DD08EBCA03002B9EDDD6
:10BF4000537E2BB9049BAF2B02D90133DBB2049390
:10BF5000109BD3F800E0414B11931A46DEF81430E1
:10BF6000934240F08E801FFA88F30E9308339BB201
:10BF7000BDF81420059305230D9300230A93CDF8F3
:10BF80003C800FFA8AF3DDF84080CDF818900B92D0
:10BF90001FFA8AFBCDF820A099460A9ABDF8100036
:10BFA0000B9C0E9D0523194611FB00232C481146BE
:10BFB000C75C039702FB0B4214FA81F312B21BB267
:10BFC00009920C932C462E461CE0089B0999012BE4
:10BFD0002AB24B4640462DD0079F0197CDF80090DE
:10BFE000DEF81CA0D047D8F800E0039B5B080134C2
:10BFF0000393059BA4B25D445E44A342ADB2B6B2C6
:10C000003FF451AF039BD807DFD4079B069A9342B6
:10C01000EBD0089B012B16D0069B0193CDF8009026
:10C02000DEF81CA009994B4632B24046D047D8F8FA
:10C0300000E0DAE7DEF818A0079B0C9922B2D0479F
:10C04000D8F800E0D1E7DEF818A00C991346404676
:10C0500022B2D047D8F800E0C7E700BF39B90000E6
:10C06000343701000B99109DCDF800900531DEF8B2
:10C07000204009B2424608232846A047D5F800E0F0
:10C080003CE7109C20469847D4F800E06BE700BFDF
:10C09000F0B5C36985B004462BB30A2968D00D29D1
:10C0A0004AD01A7A914247D3587A884244D35D687D
:10C0B0008A1A05EBC205AA78002A50D0E878002831
:10C0C0004DD0207E00283AD095F905E0B4F90E0055
:10C0D000A67DB4F90A70724406FB0202BA4262DC21
:10C0E000B4F9102030E00A2956D00D2924D0027E60
:10C0F000002A4BD0B0F90E00A57DB4F90A600622E3
:10C1000012FB0502B2423EDD228AE38102EBC50248
:10C1100012B218462282A78A668A02950B468DE8DB
:10C12000C00001462046FFF719FEA37DE28903EB1C
:10C13000430302EB4303E381012005B0F0BDA67D7C
:10C14000B4F90E00B4F91020B4F814E0678A02962E
:10C150000B468DE8804001462046FFF7FFFD297918
:10C16000E389A27D012001FB0233E38105B0F0BD2C
:10C170000022C2819A7A817D038A01FB0233038205
:10C18000012005B0F0BDB4F91020C4E7857DB4F9F5
:10C190001020B0F90E00BEE7028A817DC38102EB58
:10C1A000C1030382C8E70020E0819B7A228A03FB57
:10C1B000062212B22282C7E7C1810282704700BF05
:10C1C000002908BF01218175704700BF818241822B
:10C1D000704700BFC07D7047B0F90A00704700BFCC
:10C1E000B0F90C00704700BFF0B5C47DBDF8145025
:10C1F000022C75D0032C6ED0012C32D0002A79DBB2
:10C20000B0F90840944265DD002978DBB0F906609A
:10C210005818B042C4BF731A1BB2002B5ADD002A53
:10C220001046B8BFD01D012440F3CF0002F0070232
:10C23000704E01EBC01104FA02F2A5423144D2B2B1
:10C2400000F0A480C0F09580022D43D1013B11FA8B
:10C2500083F04B1E13F8011F514083421970F9D12E
:10C26000F0BDC488013CA21A12B2002A7BDBB0F9EF
:10C27000064094422EDD00293DDBB0F908605818D5
:10C28000B042C4BF731A1BB2002B23DDC9B2C80869
:10C29000584C02EBC01211F00701DBB204EB0200B4
:10C2A00039D0C1F10801C9B2534E8B42765C2AD213
:10C2B000C3EB010EFF2747FA0EF7012D06EA07062A
:10C2C00074D06ED3022D40F09480A75C7E40A654BB
:10C2D0008B421DD2F0BD0489E41A611A09B2C4E789
:10C2E0000689C488013EB21AE41A12B2611A002A01
:10C2F00009B285DAF0BD0B441BB20021BDE70B4447
:10C300001BB2002182E7012D50D04AD3022DDCD090
:10C310005B1ADBB28030072B18D9022D4ED0A3F167
:10C320000806C6F3C406B11C00EBC111012D0CBFF9
:10C33000FF24002400F1800202F8804C80328A42FF
:10C34000FAD1013600EBC61003F00703002BC1D071
:10C350002A4A012DD35C2DD006D3022DBAD1027802
:10C3600053400370F0BDF0BD027822EA030303706E
:10C37000F0BD013BD24311FA83F0D2B24B1E13F849
:10C38000011F114083421970F9D1F0BD013B11FA30
:10C3900083F04B1E13F8011F114383421970F9D12A
:10C3A000F0BDA75C27EA0606A65491E7A75C3E43CA
:10C3B000A6548DE7027813430370F0BDA3F108057E
:10C3C000C5F3C405AC1C00EBC41400F1800212F8E4
:10C3D000801CC94302F8801C8032A242F7D101358B
:10C3E00013F0070300EBC5103FF474AF034AD35CAE
:10C3F000B5E7F0BD208FFF1F188FFF1F108FFF1FA5
:10C40000F0B5C47DBDF81450022C76D0032C6FD04B
:10C41000012C37D000297ADBB0F906408C4230DDA0
:10C42000002A79DBB0F908609818B042C4BFB31A8B
:10C430001BB2002B25DDD2B2D008754C01EBC01128
:10C4400012F00702DBB204EB010071D0C2F1080266
:10C45000D2B2704E9342B65C62D2C3EB020EFF279B
:10C4600047FA0EF7012D06EA070600F0AC80C0F08F
:10C47000A580022D40F0CA80675C7E4066549342DE
:10C4800053D2F0BDC488E41AA21A12B2002977DB95
:10C49000B0F908408C42F4DD002A39DBB0F90660BF
:10C4A0009818B042C4BFB31A1BB2002BE9DD0029B3
:10C4B0000846B8BFC81D012440F3CF0001F00701B2
:10C4C000534E02EBC01004FA01F1A54206EB000244
:10C4D000C9B268D05AD3022DD3D1013B12FA83F0EE
:10C4E000531E13F8012F4A4083421A70F9D1F0BD50
:10C4F0000489013C611A09B2C8E7C6880489013E73
:10C50000711AE41A09B2A21A002912B284DAF0BD33
:10C5100013441BB20022C1E713441BB2002281E77F
:10C52000012D50D04AD3022DA6D09B1ADBB2803009
:10C53000072B18D9022D4ED0A3F10806C6F3C40666
:10C54000B11C00EBC111012D0CBFFF24002400F130
:10C55000800202F8804C80328A42FAD1013600EB28
:10C56000C61003F00703002B8BD02B4A012DD35CA0
:10C570002DD006D3022D84D1027853400370F0BD34
:10C58000F0BD027822EA03030370F0BD013BC9430A
:10C5900012FA83F0C9B2531E13F8012F0A408342E6
:10C5A0001A70F9D1F0BD013B12FA83F0531E13F853
:10C5B000012F0A4383421A70F9D1F0BD675C27EA64
:10C5C000060666545BE7675C3E43665457E70278AD
:10C5D00013430370F0BDA3F10805C5F3C405AC1CFB
:10C5E00000EBC41400F1800111F8802CD24301F853
:10C5F000802C8031A142F7D1013513F0070300EB05
:10C60000C5103FF43EAF044AD35CB5E7F0BD00BFB0
:10C61000208FFF1F188FFF1F108FFF1FF8B50D1EF3
:10C6200006DB14461F460646FFF7D6FD854200DBB3
:10C63000F8BD002CFCDB3046FFF7D2FD8442F7DA70
:10C640003046FFF7C7FD02284BD0032843D001280E
:10C6500004D1F388013B1B1B2C461DB2012F03D0D4
:10C6600026D3022F12D0F8BD002C2346B8BFE31DFD
:10C6700043F3CF0305EBC3151E4804F00704435DE5
:10C68000012101FA04F41C434455F8BD002C234653
:10C69000B8BFE31D43F3CF0305EBC315154804F002
:10C6A0000704435D012101FA04F45C404455F8BDE0
:10C6B000002C2346B8BFE31D43F3CF0305EBC3159E
:10C6C0000C4804F00704435D012101FA04F423EA55
:10C6D00004044455F8BD3389013B5B1B25461CB25D
:10C6E000BCE7F18832890139013A4D1B141B2DB288
:10C6F00024B2B3E7208FFF1F38B5402204460D4611
:10C700008021FFF767FAFF23064A84F8255084F852
:10C71000223084F8263084F8243084F823302260D4
:10C72000204638BD3C3C01004FF4806200210148A6
:10C7300004F038BC208FFF1FF8B590F92230013388
:10C7400004460F4642D0012190F8260001F0B0F9CE
:10C75000002194F8240001F0ABF9002194F82600A0
:10C7600001F0A6F994F8273083B1254B1A684FF0F1
:10C770000043D3625763D36A002BFCDA936B94F8BF
:10C7800026000121BDE8F84001F092B90826802575
:10C79000002194F8230001F08BF917EA05034FF00C
:10C7A000010194F8220008BF194601F081F9012126
:10C7B00094F82300CD4001F07BF9013EE8D194F8D4
:10C7C00026000121BDE8F84001F072B90D4C90F847
:10C7D000203001255B002046002184F83B3084F89E
:10C7E0005E5084F85D50FEF715FA39462046FEF794
:10C7F00011FA29462046BDE8F840FEF7CBBB00BF42
:10C80000D88EFF1F008EFF1FF8B50D4690F922103D
:10C8100080F820200131044680F821501F4600F0A6
:10C82000AD80012190F8240001F056F9012194F81F
:10C83000260001F051F994F82730002B00F0D38046
:10C84000804E3046FEF704FFF37A002B40F0DB8089
:10C8500033687D4AD968914206D07C4E7C487D4938
:10C860001E60DA6018611960E7B194F925000028AC
:10C8700018DBC0B2012101F02FF9012194F8250045
:10C8800001F016F9012001F04FF9002194F825007C
:10C8900001F00EF90A2001F047F9012194F8250072
:10C8A00001F006F9AE212046FFF746FFD5212046CC
:10C8B000FFF742FF80212046FFF73EFFA8212046D8
:10C8C000FFF73AFF3F212046FFF736FFD3212046EE
:10C8D000FFF732FF00212046FFF72EFF40212046C0
:10C8E000FFF72AFF8D212046FFF726FF012D4DD0AF
:10C8F00014212046FFF720FF20212046FFF71CFFD0
:10C9000000212046FFF718FFA1212046FFF714FF62
:10C91000C8212046FFF710FFDA212046FFF70CFF61
:10C9200012212046FFF708FF81212046FFF704FF70
:10C93000CF212046FFF700FFD9212046FFF7FCFE5C
:10C94000F1212046FFF7F8FE2046DB21FFF7F4FE39
:10C9500020464021FFF7F0FE2046A421FFF7ECFE21
:10C960002046A621FFF7E8FE20462E21FFF7E4FE31
:10C970002046AF21BDE8F840FFF7DEBE3648FEF79F
:10C980005DF936493448FEF7A3F96DE720461021DA
:10C99000FFF7D2FE20462021FFF7CEFE20460021E1
:10C9A000FFF7CAFE2046A121FFF7C6FE2046C82198
:10C9B000FFF7C2FE2046DA21FFF7BEFE2046122115
:10C9C000FFF7BAFE20468121FFF7B6FE20469F21E1
:10C9D000FFF7B2FE2046D921FFF7AEFE2221204606
:10C9E000FFF7AAFEB0E7012194F8220001F074F8E5
:10C9F000012194F8230001F06FF894F82730002B00
:10CA00003FF432AF1CE772B6F37AD8071A4606D560
:10CA10001349F26808680240B2610A601A46990731
:10CA200006D5104933690868F27A0340F3610B6058
:10CA3000530705D50C4A736911680B4033621360C4
:10CA400062B605E7D88EFF1F0000013801403F00A5
:10CA50000000017800003F80008EFF1F801A060052
:10CA600080E100E084E100E088E100E02DE9F84F9A
:10CA700021210546FFF760FE28460021FFF75CFEF6
:10CA800028467F21FFF758FE28462221FFF754FE53
:10CA900028460021FFF750FE28460721FFF74CFEED
:10CAA00095F92230013349D0012195F82600DFF8AD
:10CAB000E480DFF8E4B000F0FBFF012195F82400EA
:10CAC00000F0F6FF002195F8260000F0F1FF08F5D0
:10CAD00080694FF0004A95F8273018F8017F0BBBAA
:10CAE00008268024002195F8230000F0E1FF17EAD2
:10CAF00004034FF0010195F8220008BF194600F029
:10CB0000D7FF012195F82300CC4000F0D1FF013E72
:10CB1000E8D1C845DFD195F826000121BDE8F84FDE
:10CB200000F0C6BFDBF80020C2F82CA05763D36A20
:10CB3000002BFCDAC845936BCDD1ECE7DFF85080D1
:10CB4000124F00244FF0010995F82030104888F862
:10CB50005E905B00402188F83B3088F85D90FEF7DE
:10CB600059F804F11006B6B2395D09480134A4B28F
:10CB7000FEF750F8B442F7D101210548FEF70AFA52
:10CB8000B4F5806FE0D1BDE8F88F00BF208FFF1FA4
:10CB9000008EFF1F1F8FFF1FD88EFF1F844641EAA4
:10CBA000000313F003036DD1403A41D351F8043B25
:10CBB00040F8043B51F8043B40F8043B51F8043B77
:10CBC00040F8043B51F8043B40F8043B51F8043B67
:10CBD00040F8043B51F8043B40F8043B51F8043B57
:10CBE00040F8043B51F8043B40F8043B51F8043B47
:10CBF00040F8043B51F8043B40F8043B51F8043B37
:10CC000040F8043B51F8043B40F8043B51F8043B26
:10CC100040F8043B51F8043B40F8043B51F8043B16
:10CC200040F8043B51F8043B40F8043B403ABDD285
:10CC3000303211D351F8043B40F8043B51F8043B27
:10CC400040F8043B51F8043B40F8043B51F8043BE6
:10CC500040F8043B103AEDD20C3205D351F8043BB6
:10CC600040F8043B043AF9D2043208D0D2071CBF82
:10CC700011F8013B00F8013B01D30B8803806046AB
:10CC8000704700BF082A13D38B078DD010F0030321
:10CC90008AD0C3F10403D21ADB071CBF11F8013B91
:10CCA00000F8013B80D331F8023B20F8023B7BE7E0
:10CCB000043AD9D3013A11F8013B00F8013BF9D20B
:10CCC0000B7803704B7843708B78837060467047A5
:10CCD000374A384913681B06FCD40B6813F08003ED
:10CCE000F8D172B634490A78002A5FD0334A344802
:10CCF000F0B4344C176806682568D4680C303E449C
:10CD0000143200681268304F35442C4420440244E9
:10CD1000C2F34E022D4E2E482E4D2F4C42F40042AF
:10CD20003A60376806682D682C4A24680C303E4407
:10CD3000006812682A4F35442C4420440244C2F350
:10CD40004E02284E2848294D294C42F400423A60B0
:10CD5000376806682D68274A24680C303E4400680E
:10CD60001268254F35442C4420440244C2F34E023D
:10CD7000224E2348234D244C42F400423A60376847
:10CD800006682D68214A24680C303E440068126809
:10CD900035442C4420440244C2F34E021C4842F461
:10CDA000004202600B7062B6F0BC704762B670471A
:10CDB00024B0034024B00B403A9FFF1F38B003401B
:10CDC0003CB0034040B003402CB0034058B0034097
:10CDD0005CB0034060B0034064B003406CB00340FB
:10CDE00030B0034038B00B403CB00B4040B00B407B
:10CDF00044B00B404CB00B402CB00B4058B00B4033
:10CE00005CB00B4060B00B4064B00B406CB00B40AA
:10CE100030B00B4030B42948294A2A4B2A4D6024AF
:10CE2000E121047011701B78284C082B30D00A2B9C
:10CE30002748284937D00C2B0CBF35223D2212231E
:10CE40002A60236002600B60234B24491B78244A2C
:10CE5000BBB101230B601360224B23491B78234A8B
:10CE6000012B26D9042B0FD9082B1ED9102B94BFC8
:10CE7000862387230B6013601D4B01221A7030BC80
:10CE800070470B601360E7E784230B601360F3E7E0
:10CE900000F58E200F490830012213232A602360F9
:10CEA00002600B60D0E73922F7E785230B6013603F
:10CEB000E2E780230B601360DEE700BF004007401D
:10CEC000014007402093FF1F08B003400CB003400F
:10CED00008B00B400CB00B403D9FFF1F20B003403B
:10CEE00020B00B402193FF1F24B0034024B00B401F
:10CEF0003A9FFF1F0C2830B417D91023984228BF3F
:10CF000018461C46104A114D1178181A8C42287088
:10CF100018D00F4913700B7823B10E490E4A002325
:10CF20000B60136030BCFFF775BF0A2802D90C23D1
:10CF30001C46E7E7082802D90A231C46E2E7082333
:10CF40001C46DFE730BC70472093FF1F399FFF1F4F
:10CF50003A9FFF1F24B0034024B00B4028282FD84D
:10CF6000334B2DE9F0411E5CFF2E2BD0314B1B784B
:10CF7000002B2AD132062CD472B62F4D2F4C2F46BF
:10CF8000012326602B7062B672B623681B060CD490
:10CF90003B781BB9F4E72B78002BF1D062B602F096
:10CFA000B9F872B623681806F5D5254B1B68002220
:10CFB0002A7062B6234A107843FA00F0BDE8F08187
:10CFC000002070470020BDE8F081FFF781FE3206A7
:10CFD000D2D572B61C4DDFF87C801C4C06F04007A1
:10CFE000FFB206F03F06D8F80030DFB123F010039F
:10CFF000C8F8003001232660134A2B7062B672B65F
:10D00000236819060CD413781BB9ECE72B78002B96
:10D01000E9D062B602F07EF872B623681B06F5D539
:10D020000B4BC3E743F01003C8F80030E2E700BF42
:10D030008C3C01003A9FFF1F3C9FFF1F00B0034044
:10D0400010B00340399FFF1F3B9FFF1F00B00B40F4
:10D0500010B00B400CB00B400A4A0B49136843F464
:10D06000805313600B7843B9084BC0221A70084BE9
:10D0700080F30C0000B218807047044B80221A70B5
:10D08000F5E700BF2C8004403D9FFF1F21C00C40EE
:10D0900000C00C40F0B51B4B1B4E596818689A68CD
:10D0A000DB6885B06C460FC4337899071DD5174AE5
:10D0B000174C1378174913F0700318BF1370164AF2
:10D0C000164B8027177000263320032226706D46EA
:10D0D00008701A7072B6043C45F001052046A84756
:10D0E00062B6237813F0700309D10D4B064901E0B5
:10D0F000013B02D00A78D207FAD505B0F0BD237003
:10D1000005B0F0BDB83C0100010002400000024043
:10D11000040002400B000240070002400A000240E7
:10D12000410D0300B0F5006F0AD210B5094B1B7812
:10D13000DB07044606D504F1A0500078C0B210BD4C
:10D1400000207047FFF7A6FF04F1A0500078C0B29E
:10D1500010BD00BF01000240B0F5006F17D238B516
:10D160000F4B1B78DA070D46044611D504F1A05089
:10D170000378AB420AD00B4A137813F0700318BF40
:10D180001370074A05701378DB07FCD538BD70476C
:10D19000FFF780FF04F1A0500378AB42EBD1F5E735
:10D1A000010002400000024008B5104C08E023686E
:10D1B00059050DD423681A050FD42368DB0411D454
:10D1C00023685803F3D500F0A1FF23685905F1D572
:10D1D00001F0FEFF23681A05EFD502F08FF82368EF
:10D1E000DB04EDD500F026FEEAE700BF3480044002
:10D1F00008B5FFF7D9FF00BF014B10221A80704716
:10D2000000200540704700BF094908B50B6830B1E0
:10D210006A461844A2F58052904202D2086018462D
:10D2200008BD03F06DFB0C2303604FF0FF3008BD19
:10D230002493FF1FFEE700BFEFF3138070B9EFF3F5
:10D2400010836BB9EFF305825AB94FF48070EFF396
:10D2500011832BB1984228BF184670474FF0FF301A
:10D2600070470F2A01D81846F1E7014BD05CEEE772
:10D27000F0E300E0F0B44D1E2E46002400E001343F
:10D28000B0FBF2F302FB1300092800F130078ABF5C
:10D290003730F8B2C0B206F8010F1846002BEED1B5
:10D2A0000A1953704CB1107815F8016F28700133CA
:10D2B000E01A834202F80169F5DB0846F0BC7047CA
:10D2C0002DE9F04F0D4685B085EAE57901468246A5
:10D2D00017461C46A9EBE57903F076FA002840F0E2
:10D2E0002F812AF000484046C74903F06DFA002814
:10D2F00047D14046C44903F049FA0646002840D1C8
:10D300000021504603F038FA002814BF04200320FF
:10D3100048451DDB002DC0F274815046002103F00A
:10D320002BFA254648BB49214E22462321706270C4
:10D33000A3700334002E00F07681A019202304F896
:10D34000013BA042FBD10023037005B0BDE8F08F84
:10D35000002DC0EB0906E0DA002E00F05281A5197D
:10D36000202304F8013BAC42FBD15046002103F0DE
:10D3700003FA002800F0228100262D232B706C1C5C
:10D38000D1E702AB01AA3946504603F0A9FABB46E1
:10D390008046DDF80490002F57D0C9F10003BB424E
:10D3A00000F39480404604F06BF80646B145B8BFE0
:10D3B0000136B9F1000F40F098800136DDF808E041
:10D3C000BEF1000F53D00136A81B002804EB060164
:10D3D00053DC23462D221A700133B9F1000F63D1BB
:10D3E00037B11A46302002F8020B2E20587013462F
:10D3F0008B4220D25F1C98F800201A708F4208F1EF
:10D40000010819D0019A4FF02E0E0BE083F801E0CD
:10D4100002338B4203F101070DD218F8010B18708B
:10D420008F4209D0013A0192002AEFD03B468B424D
:10D4300003F10107F1D31946002DC0F2A9800023A2
:10D4400020460B7005B0BDE8F08FB9F1000FA4D1F4
:10D4500090F800806D496E4A012301939946B8F116
:10D46000340F8CBF884690464FF0FF3397E7A81BD8
:10D47000002804EB060140F3D8800144224601381D
:10D480004FF0200C02F801CBC2F101030344234406
:10D49000002BF7DC20EAE07301332344BEF1000FD8
:10D4A00098D1B9F1000F9BD0A2DA002FA0D01A4674
:10D4B000302002F8020B2E275F70C9EB020302F83E
:10D4C000010B9342FBD10022019291E7C7F10009C1
:10D4D0000126B1453046B8BF0136B9F1000FDFF87B
:10D4E0003081CDF804903FF468AFBFF667AF002FEE
:10D4F0003FF464AF09EB0703984207F102067FF699
:10D500005DAF002F07DD5046424902F097FFBBF1A7
:10D51000010B8246F7D102AB03AA5946504603F0ED
:10D52000DFF9DDF80490039A7B1CC9EB02029A42F2
:10D5300008BF09F10109804608BFCDF804903DE716
:10D540000021504603F018F9002814BF04200320DE
:10D5500048453BDA002DC0EB09063BDB4FF07E531C
:10D560005046002163F31E0003F006F9254600280B
:10D5700041D14E2341222370A37062700334002EE8
:10D5800051D0A019202304F8013B8442FBD1DAE6F4
:10D59000A8194342002B6FEA00007FF750AF0A46FC
:10D5A000202502F8015BC2F1010303440B44002B68
:10D5B000F7DC20EAE0730133194440E749214E22A9
:10D5C000462329706A70AB70E81CBCE6002D16DBA0
:10D5D0000026C3E79EB1A519202304F8013BAC4205
:10D5E000FBD14FF07E535046002163F31E0003F041
:10D5F000C3F888B100262D232B706C1CB9E7254693
:10D60000EFE72546B1E600BFFFFF7F7FCC3C01007E
:10D61000C83C0100000020414E2341222B70AB701A
:10D620006A70E81C8FE620468DE62346D5E600BFEB
:10D63000704700BF10B40F4B53F8302092F880426F
:10D640002CB1012369B182F8803010BC704703EB24
:10D65000C0035B681A6841B922F002021A6010BC6C
:10D66000704782F8003110BC704742F003021A6024
:10D6700010BC7047D03C01001C4A02EBC0030129DA
:10D680005B6811D004291BD052F83000002280F8CA
:10D69000802229B1022920D0032922D01A607047A4
:10D6A0004FF480721A60704752F830004FF4A27243
:10D6B00080F880121A601A6822F020021A607047FF
:10D6C00052F830104FF4A272012081F880021A60E3
:10D6D0001A6842F020021A60704740F203121A6082
:10D6E00070474FF481721A60704700BFD03C010050
:10D6F000212817D8F8B5042A13D8DFE802F0494CDE
:10D700004F1446002C4872B6236823F4702343F06C
:10D710008072C4F384011643236040F821502660D0
:10D7200062B6F8BD70474FF41026244B03EBC003DC
:10D730000D465C68216811F4E06134D0204B214A29
:10D740002149C3F89C2104F140422048C3F8A411A8
:10D75000A2F592211E4FC3F8A0017C291D48C3F8F1
:10D76000A871C3F8AC01CDD9A2F594237C2B18D9AC
:10D77000A2F596237C2B19D9A2F598237C2B17D9D7
:10D78000A2F59A227C2A15D9F8BD4FF43026CCE7B1
:10D790004FF40026C9E74FF44026C6E74FF4202691
:10D7A000C3E70D48AFE7FFF767FFC7E70B48AAE7F6
:10D7B0000B48A8E70B48A6E72893FF1FD03C0100C1
:10D7C0000082FF1FF188FF1F9988FF1FC588FF1F78
:10D7D0006D88FF1F4188FF1F6093FF1FB093FF1FDD
:10D7E000E093FF1F0094FF1F1A4B03EBC00010B41F
:10D7F000426802F14043A3F592217C2905D9A3F5A3
:10D8000094217C2913D8144900E0144972B6136896
:10D81000134C23F08773C2F3840023F4803343F066
:10D820008073136041F8204062B610BC7047A3F5C6
:10D8300096217C2909D9A3F598217C2907D9A3F53C
:10D840009A237C2BF1D80749E0E70749DEE707492F
:10D85000DCE700BFD03C01006093FF1F2893FF1F4F
:10D8600031D600000094FF1FB093FF1FE093FF1F0D
:10D8700030B4054B054D064C002210211A602A6079
:10D880002060196030BC704714D0034004D00340BE
:10D8900000D00340282838B52ED0002904464FDD9B
:10D8A0005F4B1B78012505FA03F28A4202D8212832
:10D8B00037D938BD0338C2B2012A3AD9202C4AD010
:10D8C000192C48D0574A126802FB011222FA03F3BE
:10D8D0001D2800F29B80DFE800F0928B847D9999EF
:10D8E000766F99999999999999999968615A5399E3
:10D8F0004C99999999999945494B1B780B2B08D9C3
:10D900000C2B1CBF0C3B19410846BDE83840FFF703
:10D91000A3BBC3F10C0399400846BDE83840FFF7AC
:10D920009BBB2946FFF786FE2946BDE83840FFF736
:10D93000A3BE3D4A126802FB011222FA03F3C7E7B5
:10D940002128B6D80021FFF775FE20460121BDE849
:10D950003840FFF791BE354A126802FB011222FAE5
:10D9600003F3B5E73249334A0B604FF45173136048
:10D9700038BD3149314A0B604FF45173136038BDE3
:10D980002F49304A0B6040F24443136038BD2E49A2
:10D990002E4A0B6040F24443136038BD2C492D4A97
:10D9A0000B6040F24443136038BD2B492B4A0B6097
:10D9B00040F24443136038BD29492A4A0B6040F2C3
:10D9C0004443136038BD2849284A0B6040F2444361
:10D9D000136038BD2649274A0B6040F24443136068
:10D9E00038BD2549254A0B6040F24443136038BDD9
:10D9F0002349244A0B604FF45173136038BD224908
:10DA0000224A0B604FF45173136038BD212C3FF64E
:10DA100050AF7F29D4BF00210121204693E700BFEA
:10DA20000894FF1F088003400890034008800B40C3
:10DA300010800B4048A0044018800B404CA00440CC
:10DA40001880034008B004401080034004B0044034
:10DA50004080034018C004403880034014C0044094
:10DA60002880034010B00440208003400CB00440E4
:10DA70003080034010C00440488003401CC0044074
:10DA800018900340349004401090034030900440BC
:10DA900038B1102828BF1020044AC3B21078137080
:10DAA0007047024A01231078137070470894FF1FD3
:10DAB000212801D8FFF7BEBD704700BF212806D836
:10DAC000044B53F8303093F80002C0B27047002086
:10DAD000704700BFD03C0100212801D8FFF7CCBD22
:10DAE000704700BF72B60C490C4B0D4A1B680868A2
:10DAF000126862B6520102D5322B88BF0130094943
:10DB0000C3F5BB334FF47A72FF33A1FB031302FB5F
:10DB100000F000EB93107047409FFF1F18E000E0FB
:10DB200004ED00E0ABAAAAAA2DE9F843054672B6B7
:10DB3000204F214B214A1B683C68126862B6520193
:10DB400002D5322B88BF013495B3C3F5BB331C4ECD
:10DB5000DFF86490DFF86480FF334FF47A72A6FB3D
:10DB6000031302FB04F404EB931472B6D9F800100B
:10DB70003A68D8F800E062B6C1F5BB33FF33A6FBC4
:10DB800003031EF0806FC4EB93134FF47A7002D03E
:10DB9000322988BF013200FB0233B3F57A7F04D308
:10DBA000013D05D004F57A74DFE701F0B3FADCE754
:10DBB000BDE8F883409FFF1F18E000E004ED00E09F
:10DBC000ABAAAAAAF8B52D4B2D49DFF8D0E0DFF8B3
:10DBD000D0C02C4E2C4D2D4C2D4A2E4F4FF4000012
:10DBE00018604FF0807018604FF0007018604FF0B0
:10DBF000806018604FF000601860002008602823E3
:10DC00004BF6FF71CCF80010CEF800303360136093
:10DC10002B6023603B60B3629362092245F8242C99
:10DC2000C4F8D80F05F57F65C7F8D41F07F5FF279F
:10DC300007F5FA67C6F8F83F2B6006F5FF26C4F82B
:10DC4000D42F05F5FD2504F5FF24386006F2F4769F
:10DC50001148316005F5FF6504F5FD642B60236014
:10DC60000260FFF7D7F81920FFF75EFF00F05AFEB9
:10DC700040F21310BDE8F840FFF756BF08E100E09E
:10DC80000480034014800340248003402C80034020
:10DC90001C8003403480034000800B400C80034014
:10DCA000088003402DE9F84F214B1B6807460BB154
:10DCB00001221A70DFF888901E4D99F80040DFF8B5
:10DCC00084801D4E0134272C8ABF4FF0000A5FFA72
:10DCD00084FA5446AB462B78A34216D1FFF7ACFA30
:10DCE00040281FDC33791B06F5D59BF80030013343
:10DCF000272B86BF00221346DAB218F80330DBB2B6
:10DD0000F3712A702B78A342E8D00C490A4BFFB27A
:10DD100008F804700120AC22087089F800A0DA70BD
:10DD2000BDE8F88FFF28D6DD01F0F4F9D3E700BF96
:10DD3000B89FFF1FB59FFF1F00C00640B49FFF1F85
:10DD4000BC9FFF1F4C9FFF1F1C4BDFF894C01A683D
:10DD50001B49F0B542F480521A4D1A60DFF884E096
:10DD6000194F1A4E1A4C00238CF800304FF45172A0
:10DD70002B701F2840F213358EF800303B70337043
:10DD800025600A6012D819460124124A124D1170FA
:10DD90001248547000212C27402693724FF400340F
:10DDA00091701174D7702E700460F0BDC0F34431CF
:10DDB000C0F3471400F01F03E7E700BF34800440BE
:10DDC0000CC00440499FFF1FB59FFF1FB49FFF1F5A
:10DDD00008C0044000C0064031E400E004E100E077
:10DDE000489FFF1FBC9FFF1F034B1B68DB0401D52F
:10DDF000FFF758BF704700BF3480044010B5044C93
:10DE0000237823B101F086F92378002BFAD110BDD5
:10DE1000B49FFF1F054A064B10781B78C0B2DBB2D7
:10DE2000984238BF4030C01A704700BF489FFF1F5C
:10DE3000499FFF1F30B42B4B1A7994061FD52A48EF
:10DE4000DA790378294901333F2B0978C8BF0023C9
:10DE50008B42D2B203D0264CD9B2E2540170254A8B
:10DE6000116861B1244A1278D2B2934236BFC2F12E
:10DE700040029B1A9B18272BC4BF01230B70194A21
:10DE8000D378DBB2180611D45A060DD5154B1B7981
:10DE90005B0609D5194B1A491B6800220A7003B1A9
:10DEA0001A70104B2C22DA7030BC704711790906B9
:10DEB000EAD5144910480C780178C9B28C420DD0CB
:10DEC0004A1C272A84BF00210A460F4D054C98BFE3
:10DED000D1B2AA5CD2B2E2710170D5E76C21D170E7
:10DEE000D2E700BF00C00640489FFF1F499FFF1FA9
:10DEF000749FFF1F449FFF1FB59FFF1FB89FFF1F09
:10DF0000B49FFF1FBC9FFF1F4C9FFF1F21282FD8CE
:10DF1000184B195CFF292BD0174B184ADFF870C03B
:10DF200003EBC000F0B54368DFF868E0144F154D0F
:10DF3000154E00241C60DEF80030012043F0200361
:10DF40008840CEF8003014604FF4A07338602E6023
:10DF5000C2F800C0013BFDD113689B05FCD420230F
:10DF6000013BFDD1094B09B233F8110080B2F0BD7D
:10DF700000207047E03D0100D03C0100005004400B
:10DF800008500440045004400000020300510440C3
:10DF900080014A0038800440431E032B14D872B617
:10DFA0000A4951F8230068B170B4094C058834F867
:10DFB0001320466841F82360521B24F8132062B6F0
:10DFC00070BC704762B670470020704718A0FF1FF2
:10DFD00028A2FF1F013803280BD872B6074B53F84D
:10DFE000203043B100205B680130002BFBD162B6CA
:10DFF0007047002070471846F9E700BF6CA0FF1F6C
:10E00000F0B472B61A491B4E012311F8014B194F97
:10E010009A00240742F0010505D556F8324064B154
:10E0200056F83520BAB10133052BEED162B6124B4A
:10E0300000221A70F0BC00F0F1BC0F4C0F4D21789B
:10E0400047F8325007EB431308304A1E58602270DD
:10E0500062B6F0BC70470849094B0A7847F835307A
:10E0600007EBC5030830013A58600A7062B6F0E762
:10E070002C3E01000080FF1F95A0FF1F880040007C
:10E08000C8004000431E032B1DD81B4A400140F02E
:10E09000100030B4104472B6184CE25C032A1BD84E
:10E0A000DFE802F00212151703220D88E25410F087
:10E0B000080F14BFC823882343EA054308310360CF
:10E0C000416062B630BC704708300222EDE705229D
:10E0D000EBE708300422E8E7094A52F8230038B198
:10E0E000084A52F82300416042F8231062B6E9E77B
:10E0F00042F82310034AF7E70080FF1FA4A0FF1F88
:10E100006CA0FF1F7CA0FF1F00BE70472DE9F04FE1
:10E11000DFF814A3DFF814B387B044E0AC4F4FEA44
:10E12000930807EBC809013ED9F8042003F008035F
:10E13000F6B2A2F1080003F0FF04002B40F0FE80CD
:10E1400057F838301B0C99B222F8081C002B00F04D
:10E15000EC80A04B22F8064C42F8044C53F82620E1
:10E16000002A00F0CD819C4D55F8263058609B4C1C
:10E1700045F8260034F81630194424F8161000F03B
:10E180002DFC002800F0C081954A964B19F0080F2D
:10E1900000F1080018BF1346C9F8040047F83830EA
:10E1A00008238AF800309AF80040E4B261071CD5D1
:10E1B0008D4B1B78B3B18D490A7802F0FF0322B171
:10E1C000013BDBB20B7003B900BE89490A7802F04B
:10E1D000FF032AB1013BDBB20B70002B00F066811C
:10E1E00000F092FC04238AF8003004F0080303F0E6
:10E1F000FF02002B00F0C6809BF80030DBB21E0946
:10E200008CD19A08724F57F8321007EBC200C1F355
:10E210008301013940680C2900F28380DFE801F0B6
:10E2200078788181818181814281818107000168C3
:10E23000704D714B40680193694B47F832306F4E17
:10E24000686040F2816288B26B4B29600024012132
:10E2500090421C603C61BC61317000F2E980B0F515
:10E26000D06F80F00F82B0F5817F00F0DA8100F28C
:10E270006B81802800F00182822840F0D881A88834
:10E280005F4B00F07F00042800F2D2815D4A8000DD
:10E290000344147054701878840740F1028311709D
:10E2A000022174E1544B01931A6832B3564B534E1A
:10E2B000564819883478057840298E4645F002087A
:10E2C00028BF4FF0400E002C84F001043470CEEBD8
:10E2D00001010CBF8824C82407EBC80689B285F069
:10E2E000010544EA0E447260198047F838407244D0
:10E2F0000570002966D0019B1A603E4B1A88B2F562
:10E30000A06F0ED100219A785970414B1A7008E025
:10E310003849404C0D68A54200F09980304947F8D3
:10E3200032103D4A012313703AE72D4A2D4B19F064
:10E33000080F18BF134647F8383031E700F06EFB7E
:10E34000364A374952F82630002B00F0E4805868EE
:10E350008C5D42F8260003F10802C9F80420032C62
:10E3600005D8DFE804F02C02292602228A551A88F3
:10E3700019F0080F0CBF8823C82343EA024347F86B
:10E3800038300DE7E00700F19480210600F1D280DB
:10E39000A20706D5234A244913780220DBB2137062
:10E3A0000870E30602D5204B10221A7007B0BDE8B2
:10E3B000F08F04228A55DAE705228A55D7E703222F
:10E3C0008A55D4E7BEF1400F18BF002293E700BF83
:10E3D0000080FF1F18A0FF1FC49FFF1F28A2FF1F60
:10E3E000C800400088004000A0A0FF1F29A0FF1F18
:10E3F000C0A0FF1F8CA0FF1FC09FFF1F28A0FF1FF2
:10E40000C020074098A0FF1FD49FFF1F94A0FF1FAC
:10E410009820074021090003942007406CA0FF1FAB
:10E42000A4A0FF1F882007408020074090200740BD
:10E43000B0F5106F00F03E8140F2A28040F621124C
:10E44000904240F01C82A44A0123137069E74C6893
:10E45000A2498C427FF462AF0178A9297FF45EAFB4
:10E46000417845297FF45AAF8178C2297FF456AFAD
:10E47000C1786B297FF452AF99489A4E017834786D
:10E4800081F00105002C41F0020105700CBF8820CD
:10E49000C82084F0010447F8310007EBC10192481D
:10E4A0003470002505244D60047037E700F09EFCB1
:10E4B00096E68E4B88488A491A614FF0020E80F822
:10E4C00000E08B4F0A708B49196099608A4E8B4D22
:10E4D0008B4C9A610D213970FF213170DFF848E2D1
:10E4E00029702270874D884A8EF800109F270124DA
:10E4F00006F8047C5D600470DA6007B0BDE8F08F58
:10E5000043F82600814D32E6814A47F838001378F7
:10E510000133137044E68B5D032B00F2A78001A248
:10E5200052F823F0A1E10000A1E100007BE500002A
:10E5300075E500006E49714B80220D2008701A703D
:10E54000A2077FF52EAF25E740F20232904240F05D
:10E550008E81AA8802F07F02042A68D86D88002D77
:10E5600065D16348029192001044027842F00202A1
:10E57000027048E101238B5512E600238B550FE60C
:10E58000B0F5086F53D16348634A00781070ED8886
:10E590008D4280F09B815248047844F0020C07EBD6
:10E5A000CC01402DAE464FF0010328BF4FF0400E86
:10E5B0004A6002EB0E09CEEB05014FEA0E480293CA
:10E5C0000025C82242EA080384F0010247F83C30E3
:10E5D00035700270DFF814C1424BDFF8048151BB83
:10E5E000BEF1400F7FF42FAF42F0020207EBC203EF
:10E5F000DFF8F8E0C3F8049095BB0D0445F08805FA
:10E600009DF8083033704029047009EB01034EF87F
:10E6100032507FF418AF0021404A01981180036006
:10E6200011E7AA8802F07F02042A40F22D81304BC4
:10E630000F221A7007E74029D6D942F002020CEBEC
:10E64000C200C0F804907DB135489DF808501D7097
:10E65000403988F8004009F140034CF83200DBE70C
:10E660000D0445F0C805CBE72248EEE719F0080F86
:10E670000CBF022303238B5592E5274A0221147015
:10E68000547084E727494A68002AD0D06C88B5F8CE
:10E6900004E003E00C314A68002AC8D00B88A3428A
:10E6A000F8D14B887345F5D1240A032C0CBF11789F
:10E6B00009896CE7174A0D4CA978117004F180059F
:10E6C00002E00834AC4231D0236A1A06F9D5606AF8
:10E6D000083800F0A3F9F4E7942007400100040093
:10E6E00094A0FF1F28A0FF1F29A0FF1F0080FF1F6D
:10E6F000C020074088004000882007408020074055
:10E7000098200740D89FFF1F2CA0FF1FC49FFF1F0A
:10E7100095A0FF1FA0A0FF1F98A0FF1FD49FFF1F61
:10E72000C8004000303E01008C2007406F49704B0C
:10E73000704A02917049714D714C059603954FF0E6
:10E740000009884616461D460494286828B1446886
:10E7500000F064F92046002CF9D100232B60039BC4
:10E7600030681A46002342F8293028B1446800F086
:10E7700055F92046002CF9D100223260029A98F80F
:10E7800000301146002241F8042B049A0291023B0A
:10E790004FF0000122F81910032B07D8DFE803F02F
:10E7A000470247024FF0010388F8003009F10109E0
:10E7B000B9F1040F05F1040506F1040608F101089A
:10E7C000C3D1504B059EDFF85491DFF854810021EE
:10E7D0001970012518F8013B09F8043B1B072BD4DD
:10E7E000AC0044F0020244F00304002347F8323046
:10E7F00047F83430444B994505F10105EAD13378A7
:10E80000029383F001050021894688468E460A4618
:10E810003E48047844F0020C07EBCC030393029BC0
:10E82000002B039B5A600CBF8822C822CAE64FF017
:10E83000000388F80030B9E700F0D0F8AC0007EB2F
:10E84000451300F10802002837D05A60304B47F8D2
:10E85000343000F0C3F844F0010307EBC30200F1C9
:10E86000080100B351602B4A47F83320B9E7B0F5EF
:10E87000A06F7FF4DCAE012300250293C3E740F6CE
:10E8800021229042F7D0D2E66D88002D7FF4CFAEE2
:10E890002148029192001044027822F00202027094
:10E8A000B1E7022173E6174B44F001021B7847F8E9
:10E8B0003200144A0133137093E7124B114A1B784C
:10E8C000AC00013347F834001370C2E740298E468C
:10E8D0004FF0010328BF4FF0400ECEEB01014FEA8D
:10E8E0000E4802EB0E090025029391E77CA0FF1F62
:10E8F00018A0FF1F6CA0FF1FA4A0FF1FC49FFF1F35
:10E9000028A2FF1F95A0FF1FD420074094A0FF1F3F
:10E9100088004000C8004000C0200740C4200740D5
:10E920002C3E01002DE9F843204C00F06DFD002243
:10E9300004F1880023461A605A60083383424FF07E
:10E940000001F8D11A4A1B4F13681B4D1B481C4E7F
:10E95000DFF87880DFF878C0DFF87890DFF878E0CB
:10E9600043F480231360C4F307233B70C4F30743CD
:10E970002B70240EFF2302F528320470114D88F805
:10E98000003011488CF80030D4323370012389F8FC
:10E99000003070268EF800104FF40074102107F834
:10E9A000183C2E7004601170BDE8F8830080FF1FD2
:10E9B000348004409C200740B0200740B42007402A
:10E9C0001020074049E400E008E100E08020074013
:10E9D00088200740942007400021074072B60D4868
:10E9E0000268B2FA82F30F2B10DC4FF00041D940DD
:10E9F00022EA0102026062B6074803EBC303DB00B0
:10EA0000C2180021C15010465160704762B6002004
:10EA1000704700BF0C94FF1FBC83FF1F0D4B0E4AB5
:10EA2000C31AA2FB03231B090F2B0CD80B4A127825
:10EA300052B972B60A484FF00041026821FA03F356
:10EA40001A43026062B67047064A1278002AF0D074
:10EA5000FFF7D6BABC83FF1F398EE33895A0FF1F9E
:10EA60000C94FF1FA0A0FF1F2DE9F843224E234F57
:10EA70003168012380463B70C1B1214D4B8801EBC9
:10EA80008300013300220F2BC0F808802A7004D8BD
:10EA90004B8000233B70BDE8F88340230B800320AC
:10EAA000FFF7F0FAFFF79AFF3060F2E7DFF85490D3
:10EAB00099F80030002BEED0114D45F6215408E0B6
:10EAC000013C12D02B7883B900F024FB99F8003078
:10EAD0007BB10320FFF77EFA0528F1D8FFF77EFF10
:10EAE000014630600028EBD0C8E701232B70BDE859
:10EAF000F883BDE8F88300BFACA0FF1FA8A0FF1FEC
:10EB0000B0A0FF1FA0A0FF1F094B1B787BB910B559
:10EB1000084C216809B14B8803B910BD9B000B80DC
:10EB20000320FFF7AFFAFFF759FF206010BD7047D1
:10EB3000A8A0FF1FACA0FF1F70B5124E33788BB199
:10EB4000114D286840B14388C218147A6CB9FFF798
:10EB500065FF33782C602BB10220FFF71DFA286087
:10EB60000028F0D14FF0FF3070BD0288013393428E
:10EB700002D24380204670BDFFF750FF002320469D
:10EB80002B6070BDA0A0FF1FBCA0FF1F70B50D4E75
:10EB900033788BB10C4D286840B1438803441C7A0C
:10EBA0006CB9FFF73BFF33782C602BB10220FFF7E5
:10EBB000F3F928600028F0D14FF0FF3070BD2046F7
:10EBC00070BD00BFA0A0FF1FBCA0FF1F38B5164D31
:10EBD0002868E0B101884488A14213DD03191B7A3B
:10EBE00083B104F10803C2180C1B002302E012F8E1
:10EBF000011F21B10133A342F9D1204638BD1C4683
:10EC0000204638BDFFF70AFF0020286038BD074BBB
:10EC10001B780BB9002038BD0220FFF7BDF9286032
:10EC20000028D7D1F6E700BFBCA0FF1FA0A0FF1FA0
:10EC30002DE9F04F3D4D012283B02A7071B3DFF80A
:10EC4000F8A0DFF8F880DFF8E89083460E46DAF89F
:10EC50000000002835D0364B01934488019BC4F155
:10EC60004001B14228BF314667180022BFB21A7076
:10EC7000761A478000F1080249B1013C2244594408
:10EC80001BF8014B02F8014F5945F9D147883F2F36
:10EC900009D8284B05221A70002ED8D100202870E0
:10ECA00003B0BDE8F08F4022224B028001460024D1
:10ECB00001201C70FFF7E6F9CAF80040002EC6D10B
:10ECC000ECE798F800204AB3194B019344F2D95469
:10ECD00001270BE0013C17D099F80020A2B92A7057
:10ECE00000F018FA2F7098F80020BAB10120FFF751
:10ECF00071F90528EED82F70FFF770FECAF80000F2
:10ED00000028AAD1013CE7D10199012200234FF04C
:10ED1000FF300A702B7003B0BDE8F08F00234FF076
:10ED2000FF302B7003B0BDE8F08F00BFB1A0FF1F14
:10ED3000B8A0FF1FC0A0FF1FB4A0FF1FA0A0FF1F0F
:10ED400000B583B002AB012103F8010D1846FFF7AF
:10ED50006FFF03B05DF804FB38B50E4D0E4C2B6809
:10ED6000012020702BB1588800232370C0F140008F
:10ED700038BD0A4B1B7813B90020207038BDFFF74F
:10ED800029F90528F8D8FFF729FE0346286000284E
:10ED9000E9D1F1E7B4A0FF1FB1A0FF1FA0A0FF1FA2
:10EDA0000F4B1B78DBB110B50E4C2168B1B14B880D
:10EDB000A3B10D4800223F2B027007DC07330B4440
:10EDC00001F1470003F8012F8342FBD140230B8060
:10EDD0000120FFF757F90023236010BD10BD7047D5
:10EDE000A0A0FF1FB4A0FF1FC0A0FF1F0D4B1B78EA
:10EDF000BBB910B50C4C216803F0FF024B883F2BC8
:10EE000007DC07330B4401F1470003F8012F83426D
:10EE1000FBD140230B800120FFF734F9002323604E
:10EE200010BD7047B1A0FF1FB4A0FF1F10B4EFF3D7
:10EE3000108272B6437F33B9017F012907D00329BD
:10EE40000FD00123437702B962B610BC7047124C51
:10EE50002168A1B1114943610B6883610860586161
:10EE6000EFE70F4C216881B10E4943610B68836164
:10EE7000086058610C4B4FF080511960E1E7074B77
:10EE80004161816120601860DBE7064B416181616F
:10EE900020601860EEE700BFD4A0FF1FD0A0FF1FC6
:10EEA000C4A0FF1FC8A0FF1F04ED00E070B5EFF382
:10EEB000108272B60C4C206880B10C4E002543695C
:10EEC000236073B19D6102B962B645778368984744
:10EED000EFF3108272B620680028F0D102B962B652
:10EEE00070BD3360EFE700BFC4A0FF1FC8A0FF1FC5
:10EEF000FFF7DCBF184A30B41468002C27D0036831
:10EF000021688B420ED2CB1A00218460C16023603D
:10EF1000E06010600223037530BC704711688B42BB
:10EF2000144608D3A2685B1A0360002AF6D18260F7
:10EF3000C460A060EEE7D268C2608460E060C5682B
:10EF4000CB1A0222A8602360027530BC704784602F
:10EF5000C4601060DEE700BFCCA0FF1FF8B5224EF2
:10EF600034682CB32368002B3AD1204F1D4604E0AF
:10EF70003468ECB12368002B32D1A36803B1DD60A3
:10EF800020693360036825751B68BB4221D1037F6C
:10EF90004560022BC46020D0FFF748FF6368002B58
:10EFA000E6D023602046FFF7A5FF3468002CE1D1AE
:10EFB000EFF3108372B60E4A00211068116003B996
:10EFC00062B628B18468FFF795FF20460028F9D182
:10EFD000F8BD224600219847E0E783689847DDE7BF
:10EFE000013B2360E4E700BFCCA0FF1F05B5000094
:10EFF000DCA0FF1F024A136801331360FFF7AEBFA6
:10F00000409FFF1FF8B572B106460F461446002513
:10F01000336817F8011B1B6830469847013C0544CC
:10F02000F6D12846F8BD1546FBE700BF00B5064AF5
:10F03000036812885B6883B001A9ADF8042002223E
:10F04000984703B05DF804FB043E0100F0B50746A5
:10F050008BB0002A33D0012A08BF0A2251B32124E1
:10F0600000E0F4B2B1FBF2F502FB1511C8B20929B8
:10F0700000F1300198BFC8B20AA988BF37302144D7
:10F0800088BFC0B201F8240C661E2946002DE8D1C5
:10F0900033B1013CE4B20AAB23442D2203F8242C03
:10F0A0003B6801AA11195B683846C4F122029847EF
:10F0B0000BB0F0BD30228DF825202124E8E703684D
:10F0C000C9B21B6898470BB0F0BD00BF0029BABF9A
:10F0D00049422D2300230A22FFF7B8BF08B5F2F7F3
:10F0E00087FFFAF793FA00F015F8FAE7FFF74EBD3D
:10F0F000FFF722BDFFF76ABDFFF752BEFFF72CBE38
:10F1000008461146FFF794BD0846FFF719BE00BF39
:10F11000704700BF38B5224C237803B138BD0123B6
:10F120002370FFF753FD70BB00F042F840BB00F0C6
:10F13000D5F810BBFEF76EFEE0B900232370EFF3A5
:10F140000583002BEAD1EFF3108172B6154B1868D6
:10F15000E0B1154C2278CAB945691D6001232370BE
:10F16000C5B1AA6101B962B60025457783689847A1
:10F170002570D3E700F08EF9DFE700F089F9D9E7D1
:10F1800000F084F9D3E7FFF7C3FFCDE70029C5D12D
:10F1900062B638BD054B1D600029E5D1E3E700BF2D
:10F1A000E0A0FF1FD4A0FF1FD8A0FF1FD0A0FF1F0B
:10F1B000054A064B10781B78C0B2DBB2984238BFC4
:10F1C0004030C01A704700BFE8A0FF1FE9A0FF1F32
:10F1D000F0B4384B1A7912F0300F2CD072B6997DFA
:10F1E00001F0FF0200293DD062B6334F3349387831
:10F1F0000D78334E1C46C0B2EDB2431C402BE17972
:10F2000028BF0023AB4202F1FF32C9B21CBFF15448
:10F21000184612F0FF02F0D12A4B1B68C2B23A70B6
:10F220004BB1A84236BFC5F14005401B4019272805
:10F23000C4BF01221A701F49CA78D2B2150616D46B
:10F2400052060DD51B4B1B795B0609D51E4B1F497A
:10F250001B6800220A7003B11A70164B3C22DA7048
:10F26000F0BC70474022D9795A7462B6E3E70B7953
:10F270001C06E5D5164B174E1C783378E4B2DBB28A
:10F280009C420ED0144D01E0A3420AD00133402B22
:10F2900028BF00230879E85CC0B2C871087D072840
:10F2A000F2D9DBB2034933700B79180644BF7C23D3
:10F2B000CB70C5E700A00640E8A0FF1FE9A0FF1F34
:10F2C0002CA1FF1FE4A0FF1F70A1FF1F6CA1FF1F57
:10F2D00074A1FF1F6DA1FF1FECA0FF1F054A064B85
:10F2E00010781B78C0B2DBB2984238BF4030C01AE9
:10F2F000704700BFE8A1FF1F7DA1FF1FF0B4384B8E
:10F300001A7912F0300F2CD072B6997D01F0FF02FD
:10F3100000293DD062B6334F334938780D78334EEB
:10F320001C46C0B2EDB2431C402BE17928BF00233C
:10F33000AB4202F1FF32C9B21CBFF154184612F0C1
:10F34000FF02F0D12A4B1B68C2B23A704BB1A842FF
:10F3500036BFC5F14005401B40192728C4BF012214
:10F360001A701F49CA78D2B2150616D452060DD5A6
:10F370001B4B1B795B0609D51E4B1F491B680022DE
:10F380000A7003B11A70164B3C22DA70F0BC704759
:10F390004022D9795A7462B6E3E70B791C06E5D5A9
:10F3A000164B174E1C783378E4B2DBB29C420ED079
:10F3B000144D01E0A3420AD00133282B28BF0023BB
:10F3C0000879E85CC0B2C871087D0728F2D9DBB2C1
:10F3D000034933700B79180644BF7C23CB70C5E713
:10F3E00000B00640E8A1FF1F7DA1FF1FA8A1FF1FDD
:10F3F00078A1FF1FECA1FF1F7CA1FF1FF0A1FF1F41
:10F40000E9A1FF1F80A1FF1F70B584B072B6194B30
:10F41000194D1A48702241260F2480211A702E702F
:10F420001A460470197013781B06FCD5144B186823
:10F4300062B6144B144C984298BF00EB800001A9AF
:10F4400098BF40000A22FDF715FF01A920460023BE
:10F4500011F8012B01333AB10A2B20F8022FF7D112
:10F460001623237004B070BD5B00DBB2237004B0C0
:10F4700070BD00BF000002400700024006000240CD
:10F48000080002407F969800E894FF1F704700BF75
:10F49000704700BF704700BF2DE9F043DFF8EC80F4
:10F4A0008BB006460F4600F073F898F90030013330
:10F4B00004460D4637D03046394600F0DFF90028C3
:10F4C00031D02BA3D3E900233046394600F026FE85
:10F4D000814668BB28A3D3E900233046394600F0B3
:10F4E000FFFD00B398F90030254ACDF820900424A0
:10F4F00000200021022BCDE90467CDE902670094CA
:10F500000192CDE906012CD0684600F0BDF940B368
:10F51000089B1BB101F0F4F9089B0360DDE90601CB
:10F520000BB0BDE8F083204629460BB0BDE8F08360
:10F53000134A98F90030019203210022CDE90467B3
:10F54000CDE90267009108922BB90E4B4FF0604253
:10F55000CDE90623D8E70C490020022BCDE90601AE
:10F56000D2D101F0CDF922230360D1E7AFF30080BF
:10F57000EF39FAFE422E864051302DD5104987C012
:10F580009C3E0100FFFFEF470000F07FFE94FF1F4D
:10F590002DE9F04FB04F21F00042BA4283B00C4643
:10F5A0004FEAD17605460DD9AC4FBA4225D9C1F301
:10F5B0001303034340F0EF800EB10020014603B077
:10F5C000BDE8F08FA64B9A4200F2CC80A54B9A4240
:10F5D00000F2DE808AA3D3E9002300F05DF9002267
:10F5E000A14B00F09BFD002800F005812846214634
:10F5F00000229D4B00F050F9E1E783A3D3E90023FB
:10F6000000F08CFD002840F0CB802846214680A3E6
:10F61000D3E9002300F064FD0028CED1934B2846A7
:10F6200003EBC60821467CA3D3E9002300F0E6FAE9
:10F63000D8E9002300F030F900F07AFD804600F0B0
:10F6400077FA77A3D3E9002306460F4600F0D6FAEF
:10F6500002460B462846214600F01CF972A3D3E966
:10F660000023CDE900013046394600F0C7FA824652
:10F670008B4652465B46DDE9000100F00BF905467A
:10F680000C462A4623462846214600F0B7FA68A3CE
:10F69000D3E9002306460F4600F0B0FA66A3D3E98B
:10F6A000002300F0F7F832463B4600F0A7FA64A3C7
:10F6B000D3E9002300F0F0F832463B4600F09EFA12
:10F6C00061A3D3E9002300F0E5F832463B4600F0A1
:10F6D00095FA5FA3D3E9002300F0DEF832463B46FB
:10F6E00000F08CFA02460B462846214600F0D2F87C
:10F6F00006460F462846214632463B46B8F1000FE3
:10F7000056D000F07BFA324604460D463B460020B8
:10F710004FF0804100F0BEF802460B4620462946D5
:10F7200000F096FB02460B465046594600F0B2F8F0
:10F73000DDE9002300F0AEF80B4602464A490020FE
:10F7400000F0A8F86FF47F7398454FDA08F57A78DF
:10F7500001EB085100224FF0B87300F04FFA03B0EC
:10F76000BDE8F08F424B9A423FF658AF414BF40050
:10F770002344D3E9002300F08DF83F4BC6F1010884
:10F780001C44CDE90001D4E900ABC6EB080870E7E2
:10F790004FF0000875E702460B4600F07DF80EE7D3
:10F7A00017A3D3E900231046194600F027FA06E70D
:10F7B00000F024FA0022804689464FF0804330460C
:10F7C000394600F067F802460B464046494600F0CD
:10F7D0003FFB2A46234600F05DF802460B46002018
:10F7E000214900F057F803B0BDE8F08F01EB085154
:10F7F00003B0BDE8F08F804643E700BFAFF3008061
:10F800009C7500883CE4377EEF39FAFE422E864034
:10F8100051302DD5104987C0FE822B654715F73F23
:10F820000000E0FE422EE63F763C7935EF39EA3DB6
:10F83000D0A4BE726937663EF16BD2C541BDBB3EF6
:10F840002CDE25AF6A56113F93BDBE166CC1663FD4
:10F850003E5555555555C53F412E8640FFFFEF7F1C
:10F86000422ED63FFFFF2F3E0000F03FA03E01009A
:10F87000B1A2F03FC03E0100B03E010041F00041A6
:10F8800001F58010C00F70470020704781F00041E3
:10F8900002E000BF83F0004330B54FEA41044FEA75
:10F8A000430594EA050F08BF90EA020F1FBF54EA10
:10F8B000000C55EA020C7FEA645C7FEA655C00F0AC
:10F8C000E2804FEA5454D4EB5555B8BF6D420CDD7D
:10F8D0002C4480EA020281EA030382EA000083EA00
:10F8E000010180EA020281EA0303362D88BF30BDA0
:10F8F00011F0004F4FEA01314FF4801C4CEA1131F6
:10F9000002D0404261EB410113F0004F4FEA033354
:10F910004CEA133302D0524263EB430394EA050FDF
:10F9200000F0A780A4F10104D5F1200E0DDB02FA4E
:10F930000EFC22FA05F2801841F1000103FA0EF2E2
:10F94000801843FA05F359410EE0A5F120050EF1A8
:10F95000200E012A03FA0EFC28BF4CF0020C43FAD9
:10F9600005F3C01851EBE37101F0004507D54FF0E6
:10F97000000EDCF1000C7EEB00006EEB0101B1F536
:10F98000801F1BD3B1F5001F0CD349085FEA30007C
:10F990004FEA3C0C04F101044FEA445212F5800F87
:10F9A00080F09A80BCF1004F08BF5FEA500C50F124
:10F9B000000041EB045141EA050130BD5FEA4C0C07
:10F9C000404141EB010111F4801FA4F10104E9D190
:10F9D00091F0000F04BF01460020B1FA81F308BF87
:10F9E0002033A3F10B03B3F120020CDA0C3208DD53
:10F9F00002F1140CC2F10C0201FA0CF021FA02F12E
:10FA00000CE002F11402D8BFC2F1200C01FA02F19D
:10FA100020FA0CFCDCBF41EA0C019040E41AA2BFC2
:10FA200001EB0451294330BD6FEA04041F3C1CDA8A
:10FA30000C340EDC04F11404C4F1200220FA04F0AA
:10FA400001FA02F340EA030021FA04F345EA030154
:10FA500030BDC4F10C04C4F1200220FA02F001FA16
:10FA600004F340EA0300294630BD21FA04F0294698
:10FA700030BD94F0000F83F4801306BF81F4801131
:10FA80000134013D4EE77FEA645C18BF7FEA655CA4
:10FA900029D094EA050F08BF90EA020F05D054EA76
:10FAA000000C04BF1946104630BD91EA030F1EBF7B
:10FAB0000021002030BD5FEA545C05D1400049417F
:10FAC00028BF41F0004130BD14F580043CBF01F572
:10FAD000801130BD01F0004545F0FE4141F4700158
:10FAE0004FF0000030BD7FEA645C1ABF1946104633
:10FAF0007FEA655C1CBF0B46024650EA013406BF34
:10FB000052EA033591EA030F41F4002130BD00BFF2
:10FB100090F0000F04BF0021704730B54FF48064AF
:10FB200004F132044FF000054FF0000150E700BF30
:10FB300090F0000F04BF0021704730B54FF480648F
:10FB400004F1320410F0004548BF40424FF000017C
:10FB50003EE700BF42004FEAE2014FEA31014FEABF
:10FB600002701FBF12F07F4393F07F4F81F060510E
:10FB7000704792F0000F14BF93F07F4F704730B57D
:10FB80004FF4607401F0004521F0004120E700BF10
:10FB900050EA010208BF704730B54FF000050AE097
:10FBA00050EA010208BF704730B511F0004502D598
:10FBB000404261EB41014FF4806404F132045FEA9A
:10FBC000915C3FF4DCAE4FF003025FEADC0C18BF3F
:10FBD00003325FEADC0C18BF033202EBDC02C2F135
:10FBE000200300FA03FC20FA02F001FA03FE40EAC7
:10FBF0000E0021FA02F11444C1E600BF70B54FF0C7
:10FC0000FF0C4CF4E06C1CEA11541DBF1CEA1355A8
:10FC100094EA0C0F95EA0C0F00F0DEF82C4481EA10
:10FC2000030621EA4C5123EA4C5350EA013518BF30
:10FC300052EA033541F4801143F4801338D0A0FB1D
:10FC400002CE4FF00005E1FB02E506F00042E0FBCA
:10FC500003E54FF00006E1FB03569CF0000F18BFD0
:10FC60004EF0010EA4F1FF04B6F5007F64F5407478
:10FC700004D25FEA4E0E6D4146EB060642EAC6210B
:10FC800041EA55514FEAC52040EA5E504FEACE2E78
:10FC9000B4F1FD0C88BFBCF5E06F1ED8BEF1004F7B
:10FCA00008BF5FEA500E50F1000041EB045170BDF7
:10FCB00006F0004646EA010140EA020081EA03013B
:10FCC000B4EB5C04C2BFD4EB0C0541EA045170BD37
:10FCD00041F480114FF0000E013C00F3AB8014F1B1
:10FCE000360FDEBF002001F0004170BDC4F10004FA
:10FCF000203C35DA0C341BDC04F11404C4F120057B
:10FD000000FA05F320FA04F001FA05F240EA0200D5
:10FD100001F0004221F0004110EBD37021FA04F60B
:10FD200042EB06015EEA430E08BF20EAD37070BDC5
:10FD3000C4F10C04C4F1200500FA04F320FA05F024
:10FD400001FA04F240EA020001F0004110EBD37026
:10FD500041F100015EEA430E08BF20EAD37070BD96
:10FD6000C4F1200500FA05F24EEA020E20FA04F36F
:10FD700001FA05F243EA020321FA04F001F000411E
:10FD800021FA04F220EA020000EBD3705EEA430E8F
:10FD900008BF20EAD37070BD94F0000F0FD101F0BE
:10FDA0000046400041EB010111F4801F08BF013CF7
:10FDB000F7D041EA060195F0000F18BF704703F035
:10FDC0000046520043EB030313F4801F08BF013DBC
:10FDD000F7D043EA0603704794EA0C0F0CEA135578
:10FDE00018BF95EA0C0F0CD050EA410618BF52EA32
:10FDF0004306D1D181EA030101F000414FF0000038
:10FE000070BD50EA410606BF1046194652EA430645
:10FE100019D094EA0C0F02D150EA013613D195EAB9
:10FE20000C0F05D152EA03361CBF104619460AD101
:10FE300081EA030101F0004141F0FE4141F470010B
:10FE40004FF0000070BD41F0FE4141F4780170BDFB
:10FE500070B54FF0FF0C4CF4E06C1CEA11541DBF60
:10FE60001CEA135594EA0C0F95EA0C0F00F0A7F862
:10FE7000A4EB050481EA030E52EA03354FEA01318F
:10FE800000F088804FEA03334FF0805545EA1313A2
:10FE900043EA12634FEA022245EA111545EA10656A
:10FEA0004FEA00260EF000419D4208BF964244F101
:10FEB000FD0404F5407402D25B084FEA3202B61A20
:10FEC00065EB03055B084FEA32024FF480104FF4F4
:10FED000002CB6EB020E75EB030E22BFB61A754668
:10FEE00040EA0C005B084FEA3202B6EB020E75EBFB
:10FEF000030E22BFB61A754640EA5C005B084FEA63
:10FF00003202B6EB020E75EB030E22BFB61A75462F
:10FF100040EA9C005B084FEA3202B6EB020E75EB3A
:10FF2000030E22BFB61A754640EADC0055EA060EFB
:10FF300018D04FEA051545EA16754FEA06164FEA3E
:10FF4000C30343EA52734FEAC2025FEA1C1CC0D1EA
:10FF500011F4801F0BD141EA00014FF000004FF077
:10FF6000004CB6E711F4801F04BF01430020B4F138
:10FF7000FD0C88BFBCF5E06F3FF6AFAEB5EB030CF0
:10FF800004BFB6EB020C5FEA500C50F1000041EBED
:10FF9000045170BD0EF0004E4EEA113114EB5C04BA
:10FFA000C2BFD4EB0C0541EA045170BD41F480118D
:10FFB0004FF0000E013C90E645EA060E8DE60CEA95
:10FFC000135594EA0C0F08BF95EA0C0F3FF43BAFB2
:10FFD00094EA0C0F0AD150EA01347FF434AF95EA69
:10FFE0000C0F7FF425AF104619462CE795EA0C0F4D
:10FFF00006D152EA03353FF4FDAE1046194622E71A
:020000021000EC
:1000000050EA410618BF52EA43067FF4C5AE50EAF3
:1000100041047FF40DAF52EA43057FF4EBAE12E7E3
:100020004FF0FF3C06E000BF4FF0010C02E000BFC4
:100030004FF0010C4DF804CD4FEA410C7FEA6C5CA7
:100040004FEA430C18BF7FEA6C5C1BD001B050EA4A
:10005000410C0CBF52EA430C91EA030F02BF90EA35
:10006000020F0020704710F1000F91EA030F58BFF4
:10007000994208BF90422CBFD8176FEAE37040F056
:10008000010070474FEA410C7FEA6C5C02D150EAF4
:10009000013C07D14FEA430C7FEA6C5CD6D152EAAF
:1000A000033CD3D05DF8040B704700BF8446104674
:1000B00062468C461946634600E000BF01B5FFF773
:1000C000B7FF002848BF10F1000F01BD4DF808ED43
:1000D000FFF7F4FF0CBF012000205DF808FB00BF14
:1000E0004DF808EDFFF7EAFF34BF012000205DF86E
:1000F00008FB00BF4DF808EDFFF7E0FF94BF0120BB
:1001000000205DF808FB00BF4DF808EDFFF7CEFFBB
:1001100094BF012000205DF808FB00BF4DF808EDFA
:10012000FFF7C4FF34BF012000205DF808FB00BFCB
:100130004FEA410212F5001215D211D56FF478730F
:10014000B3EB625212D94FEAC12343F0004343EAB2
:10015000505311F0004F23FA02F018BF404270478D
:100160004FF00000704750EA013005D111F0004017
:1001700008BF6FF0004070474FF00000704700BFAD
:100180004FEA4102B2F1E04324BFB3F5001CDCF1B9
:10019000FE5C0DD901F0004C4FEAC0024CEA5070F1
:1001A000B2F1004F40EB830008BF20F00100704720
:1001B00011F0804F21D113F13872BCBF01F0004023
:1001C000704741F480114FEA5252C2F11802C2F155
:1001D000200C10FA0CF320FA02F018BF40F00100D6
:1001E0004FEAC1234FEAD32303FA0CFC40EA0C0088
:1001F00023FA02F34FEA4303CCE77FEA625307D1C5
:1002000050EA01331EBF4FF0FE4040F440007047FB
:1002100001F0004040F0FE4040F40000704700BF95
:1002200080F0004002E000BF81F0004142001FBFAB
:100230005FEA410392EA030F7FEA226C7FEA236CB4
:100240006AD04FEA1262D2EB1363C1BFD2184140A9
:1002500048404140B8BF5B42192B88BF704710F03F
:10026000004F40F4000020F07F4018BF404211F0E2
:10027000004F41F4000121F07F4118BF494292EA4A
:10028000030F3FD0A2F1010241FA03FC10EB0C0076
:10029000C3F1200301FA03F100F0004302D5494203
:1002A00060EB4000B0F5000F13D3B0F1807F06D3B0
:1002B00040084FEA310102F10102FE2A51D2B1F1A8
:1002C000004F40EBC25008BF20F0010040EA03009D
:1002D0007047490040EB000010F4000FA2F101024A
:1002E000EDD1B0FA80FCACF1080CB2EB0C0200FAD4
:1002F0000CF0AABF00EBC25052421843BCBFD04022
:100300001843704792F0000F81F4000106BF80F49B
:1003100000000132013BB5E74FEA41037FEA226C5E
:1003200018BF7FEA236C21D092EA030F04D092F029
:10033000000F08BF0846704790EA010F1CBF00205D
:10034000704712F07F4F04D1400028BF40F00040BA
:10035000704712F100723CBF00F50000704700F0DA
:10036000004343F0FE4040F4000070477FEA226201
:1003700016BF08467FEA23630146420206BF5FEAD2
:10038000412390EA010F40F4800070474FF00003D2
:1003900004E000BF10F0004348BF40425FEA000C99
:1003A00008BF704743F0964301464FF000001CE041
:1003B00050EA010208BF70474FF000030AE000BF97
:1003C00050EA010208BF704711F0004302D54042D5
:1003D00061EB41015FEA010C02BF84460146002047
:1003E00043F0B64308BFA3F18053A3F50003BCFA62
:1003F0008CF2083AA3EBC25310DB01FA02FC63440F
:1004000000FA02FCC2F12002BCF1004F20FA02F215
:1004100043EB020008BF20F00100704702F1200208
:1004200001FA02FCC2F1200250EA4C0021FA02F269
:1004300043EB020008BF20EADC7070474FF0FF0C6E
:100440001CEAD0521EBF1CEAD15392EA0C0F93EA69
:100450000C0F6FD01A4480EA010C400218BF5FEA0B
:1004600041211ED04FF0006343EA501043EA51117E
:10047000A0FB01310CF00040B1F5000F3EBF490078
:1004800041EAD3715B0040EA010062F17F02FD2A7C
:100490001DD8B3F1004F40EBC25008BF20F001005F
:1004A000704790F0000F0CF0004C08BF49024CEA76
:1004B000502040EA51207F3AC2BFD2F1FF0340EA08
:1004C000C250704740F400004FF00003013A5DDC79
:1004D00012F1190FDCBF00F000407047C2F10002BA
:1004E000410021FA02F1C2F1200200FA02FC5FEAA7
:1004F000310040F1000053EA4C0308BF20EADC70F1
:10050000704792F0000F00F0004C02BF400010F462
:10051000000F013AF9D040EA0C0093F0000F01F00F
:10052000004C02BF490011F4000F013BF9D041EA31
:100530000C018FE70CEAD15392EA0C0F18BF93EA33
:100540000C0F0AD030F0004C18BF31F0004CD8D15D
:1005500080EA010000F00040704790F0000F17BFE4
:1005600090F0004F084691F0000F91F0004F14D02A
:1005700092EA0C0F01D142020FD193EA0C0F03D182
:100580004B0218BF084608D180EA010000F0004085
:1005900040F0FE4040F40000704740F0FE4040F460
:1005A000400070474FF0FF0C1CEAD0521EBF1CEAFF
:1005B000D15392EA0C0F93EA0C0F69D0A2EB03021D
:1005C00080EA010C49024FEA402037D04FF08053B7
:1005D00043EA111143EA10130CF000408B4238BF7C
:1005E0005B0042F17D024FF4000C8B4224BF5B1A8A
:1005F00040EA0C00B3EB510F24BFA3EB510340EAD8
:100600005C00B3EB910F24BFA3EB910340EA9C0085
:10061000B3EBD10F24BFA3EBD10340EADC001B01F5
:1006200018BF5FEA1C1CE0D1FD2A3FF650AF8B4299
:1006300040EBC25008BF20F0010070470CF0004CA6
:100640004CEA50207F32C2BFD2F1FF0340EAC250D1
:10065000704740F400004FF00003013A37E792F092
:10066000000F00F0004C02BF400010F4000F013AF0
:10067000F9D040EA0C0093F0000F01F0004C02BFEB
:10068000490011F4000F013BF9D041EA0C0195E754
:100690000CEAD15392EA0C0F08D142027FF47DAFED
:1006A00093EA0C0F7FF470AF084676E793EA0C0FDD
:1006B00004D14B023FF44CAF08466EE730F0004CDB
:1006C00018BF31F0004CCAD130F000427FF45CAF6B
:1006D00031F000437FF43CAF5FE700BF4FF0FF3CD9
:1006E00006E000BF4FF0010C02E000BF4FF0010C2C
:1006F0004DF804CD4FEA40024FEA41037FEA226CF5
:1007000018BF7FEA236C11D001B052EA530C18BF16
:1007100090EA010F58BFB2EB030088BFC81738BF7B
:100720006FEAE17018BF40F0010070477FEA226C69
:1007300002D15FEA402C05D17FEA236CE4D15FEA65
:10074000412CE1D05DF8040B704700BF8446084699
:100750006146FFE70FB5FFF7C9FF002848BF10F15A
:10076000000F0FBD4DF808EDFFF7F4FF0CBF01209F
:1007700000205DF808FB00BF4DF808EDFFF7EAFF29
:1007800034BF012000205DF808FB00BF4DF808EDE4
:10079000FFF7E0FF94BF012000205DF808FB00BFD9
:1007A0004DF808EDFFF7D2FF94BF012000205DF85F
:1007B00008FB00BF4DF808EDFFF7C8FF34BF01206C
:1007C00000205DF808FB00BF4FEA40024FEA4103FA
:1007D0007FEA226C02D15FEA402C08D17FEA236CC9
:1007E00002D15FEA412C02D14FF0000070474FF078
:1007F000010070474FEA4002B2F1FE4F0FD34FF0B5
:100800009E03B3EB12620DD94FEA002343F000437D
:1008100010F0004F23FA02F018BF404270474FF02B
:100820000000704712F1610F01D1420205D110F0B2
:10083000004008BF6FF0004070474FF00000704765
:1008400042000ED2B2F1FE4F0BD34FF09E03B3EB3A
:10085000126209D44FEA002343F0004323FA02F066
:1008600070474FF00000704712F1610F01D1420252
:1008700002D14FF0FF3070474FF00000704700BFCB
:1008800010B502FB01F100F071F80446D8B150F840
:10089000042C22F00302043A242A18D8132A14D96B
:1008A00000231B2A0360436016D9242A8360C36097
:1008B00011BF00F110020361436100F1180200232F
:1008C000136053609360204610BD0246F7E7002195
:1008D00000F068FB204610BD00F10802EFE700BF02
:1008E000F0B583B016461F460D460024FFF732F9D7
:1008F000009733462A46019400F040FE03B0F0BD55
:10090000014B1868704700BF2899FF1F70B50F4E44
:100910000F4D761BB61018BF002405D0013455F8D2
:10092000043B9847A642F9D10A4E0B4D761B03F0C3
:100930005BFBB61018BF002406D0013455F8043B09
:100940009847A642F9D170BD70BD00BFF43F0100C9
:10095000F43F010000400100F43F0100024B01465A
:10096000186800F003B800BF2899FF1F2DE9F04F69
:1009700001F10B05162D83B0064640F29F8035F03D
:10098000070500F1BF80A94200F2BC8000F058FBCF
:10099000B5F5FC7FC0F09C826B0A00F0BA80042B96
:1009A00000F28381A80900F1390E4FEA4E03383076
:1009B000C44F07EB8303A3F108015C68A14207D190
:1009C000ACE0002A80F2AC80E468A14200F0A6808E
:1009D000636823F003035A1B0F2AF2DDB9493C690F
:1009E00001F1080E744500F0B381636823F003033E
:1009F0005A1B0F2A00F39981002AC1F814E0C1F8AC
:100A000010E080F29E80B3F5007F80F06781DB0804
:100A100003F1010C01229B1002FA03F34A6851F81A
:100A20003C80C4F8088001EBCC091A43A9F1080303
:100A3000E3604A6041F83C40C8F80C408310012450
:100A40009C40944200F28A80144206D120F00300B8
:100A50006400144200F10400FAD007EBC009CC4650
:100A60008046DCF80C108C4507D173E1002A80F237
:100A70008181C9688C4500F06D814B6823F00303C8
:100A80005A1B0F2AF2DD0C46D1F80CC054F8088F1F
:100A90004B1945F001054D6042F00101C8F80CC04A
:100AA0003046CCF808807B613B61C3F80CE0C3F8AA
:100AB00008E059609A5000F0C5FA1FE0102921D8CB
:100AC00000F0BEFA1025062302207E4F07EB8303B9
:100AD000A3F108025C68944200F045816368E16814
:100AE000A56823F00303234430465A68E96042F0C6
:100AF00001028D605A6000F0A5FA0834204603B068
:100B0000BDE8F08F00240C232046336003B0BDE81D
:100B1000F08F80234FF0400E3F2049E770465DE79D
:100B20002344E1685A68A56842F00102E960304652
:100B30008D605A6000F086FA0834204603B0BDE8A4
:100B4000F08F234430465A6842F001025A6000F0A8
:100B500079FA0834204603B0BDE8F08FBC686368BA
:100B600023F00308A84504D3C5EB08030F2B00F3BB
:100B70008C80554BDFF860911A68D9F8003001334A
:100B80002A4404EB080A00F0608102F580520F321B
:100B900022F47F6222F00F0211463046019200F0EB
:100BA00043FCB0F1FF3F8346019A00F05881824533
:100BB00000F2FC80454B1968DA451144196000F0D9
:100BC0005381D9F80000DFF810E101301BBFCAEBF8
:100BD0000B0A5144CEF800B019601BF0070100F079
:100BE0001781C1F10800C1F58051834408315A448E
:100BF000C2F30B02C2EB010949463046019300F0F3
:100C000013FC431C019B00F03F81CBEB00024A44E4
:100C100042F001021968C7F808B04944BC42CBF859
:100C200004201960DFF8A49016D0B8F10F0F40F23D
:100C3000FD806268A8F10C0323F00703E01802F0BE
:100C400001024FF0050E1A430F2B6260C0F804E05A
:100C5000C0F808E000F21C811D4BBC681A68914284
:100C600088BF19601B4B1A689142626888BF19607F
:100C700022F003029542A2EB050301D80F2B04DCFE
:100C8000304600F0DFF9002438E7621943F0010331
:100C900045F0010565603046BA60536000F0D2F956
:100CA0000834204603B0BDE8F08F142B71D9542BC3
:100CB00000F2A480280B00F16F0E4FEA4E036E3055
:100CC00076E600BF2C99FF1FFCA1FF1F00A2FF1FAB
:100CD000F8A1FF1FF4A1FF1F389DFF1F5A0A042A25
:100CE0005ED9142A00F2B38002F15C0149005B3244
:100CF00007EB810C57F82110DFF8DC81ACF1080C10
:100D00008C4500F088804A6822F00302934202D2A8
:100D100089688C45F7D1D1F80CC07A68C4F80CC04A
:100D2000A160CCF80840CC6088E6631942F0010766
:100D300045F00105656030464B610B61C3F80CE07E
:100D4000C3F808E05F609A50083400F07BF9D5E6FC
:100D50004A6873E608F1010818F0030F0CF1080C5B
:100D60007FF47FAE30E0DC68A34208BF02303FF47E
:100D700035AEB3E60B440C465A68C96854F8085FB0
:100D800042F001025A603046E9608D6000F05AF985
:100D9000B4E603F15C0E03F15B004FEA4E0307E695
:100DA0009A0902F1390149003832A1E7BC424A4BA5
:100DB0003FF400AF9C68626822F003025AE759F8DA
:100DC0000839994540F0828010F0030F00F1FF30A0
:100DD000F5D17B6823EA04037B6064009C423FF604
:100DE000BDAE002C3FF4BAAE1C4240467FF435AE97
:100DF00064001C4200F10400FAD02EE6B3F5AA7F8D
:100E000018D8E80B00F1780E4FEA4E037730CFE5A3
:100E10004FF48051EBE60121D8F80430921001FA2A
:100E200002F21A43C8F80420614677E70123CBF8A1
:100E3000043025E740F25452934220D8A80C00F128
:100E40007D0E4FEA4E037C30B2E51032A4E6542A00
:100E500026D81A0B02F16F0149006E3248E7BC68D0
:100E6000626822F0030205E7CAF30B0000287FF452
:100E7000A8AE4244BB6842F001025A60ECE6FE2391
:100E80004FF07F0E7E2093E501224FF00009C1E66E
:100E900004F10801304600F049FCD9F80010DBE607
:100EA000B2F5AA7F05D8DA0B02F178014900773252
:100EB0001EE740F254518A4205D89A0C02F17D0196
:100EC00049007C3214E7FE217E2211E77B6884E72B
:100ED000E808431C5B00F8E52C99FF1F8842F0B539
:100EE0000DD98B1898420AD28118002A51D09A1A2B
:100EF00013F8014D01F8014D9342F9D1F0BD0F2ACD
:100F000048D941EA00039B0746D100F1100401F1E2
:100F10001003154653F8106C44F8106C53F80C6C21
:100F200044F80C6C53F8086C44F8086C103D53F806
:100F3000046C44F8046C0F2D03F1100304F1100449
:100F4000E8D8A2F1100323F00F0302F00F0E1033C4
:100F5000BEF1030F1944034421D91E1F0D467446E8
:100F6000043C55F8047B46F8047F032CF8D8AEF116
:100F7000040424F0030404342344214402F0030253
:100F800062B1013B0A4411F8014B03F8014F8A4258
:100F9000F9D1F0BD0346F3E70346F2E7F0BD724630
:100FA000EEE700BF70B4840746D0541E002A41D03B
:100FB000CDB2034602E0621EE4B3144603F8015BBF
:100FC0009A07F8D1032C2ED9CDB245EA05250F2C6E
:100FD00045EA054519D903F110022646103E0F2EA9
:100FE00042F8105C42F80C5C42F8085C42F8045C81
:100FF00002F11002F2D8A4F1100222F00F0204F064
:101000000F041032032C13440DD91E462246043A15
:10101000032A46F8045BFAD8221F22F003020432A6
:10102000134404F003042CB1C9B21C4403F8011B9F
:10103000A342FBD170BC704714460346C2E700BF11
:10104000704700BF704700BF2DE9F04F174683B0CF
:10105000002900F0C1800E46814607F10B05FFF71D
:10106000EFFF56F804EC162D2EF00304A6F1080845
:1010700040D810221546AF4241D8944275DAC94B88
:10108000996808EB04008842416800F0D98021F09B
:10109000010303445B68DB077DD51EF0010F35D0EB
:1010A00039464846FFF762FC0746E0B156F8043C73
:1010B00023F001034344A0F108029A4200F0448166
:1010C000221F242A00F23181132A00F204810346F0
:1010D0003246116819605168596092689A603146C9
:1010E000484600F023FB4846FFF7ACFF384603B004
:1010F000BDE8F08F25F00705002D2A46BBDA0C234A
:101100000020C9F8003003B0BDE8F08F56F8083C65
:10111000C3EB080ADAF8043023F0030C04EB0C03E9
:101120009342BDDB5746DAF80C1057F8080F221F20
:10113000242AC160886000F21781132A40F21281CC
:101140003168CAF808107168CAF80C101B2A00F23E
:101150002B8108360AF11002316811607168516004
:10116000B16891603E461C46D046631B0F2B1DD8CC
:10117000D8F8043003F0010323434444C8F8043092
:10118000636843F0010363604846FFF75BFF304646
:1011900003B0BDE8F08F21F003012144914221DB2F
:1011A000C36882680C46D3609A60DEE7D8F80420F2
:1011B00008EB050102F00102154343F001020B4464
:1011C000C8F804504A605A6842F0010208315A6077
:1011D000484600F0ABFAD7E7114603B0BDE8F04F40
:1011E000FFF7C4BB1EF0010F7FF45AAF56F8083C5E
:1011F000C3EB080ADAF8043023F0030C01EB0C0E01
:1012000096458BDBC36882685746D3609A6057F86F
:10121000081FDAF80C30CB60221F242A996000F2F4
:101220009980132A62D93368CAF808307368CAF8FB
:101230000C301B2A00F2A08008360AF1100356E099
:1012400021F0030BA34405F11000834559DA1EF089
:10125000010F7FF425AF56F8081CC1EB080ADAF835
:10126000041021F0030CE34458453FF757AF5746AD
:10127000DAF80C1057F8080F221F242AC160886082
:1012800000F2B480132A40F2A5803168CAF8081031
:101290007168CAF80C101B2A00F2AF8008360AF1F8
:1012A00010023168116071685160B16891600AEB99
:1012B0000501C5EB0B0242F0010299604A60DAF8C1
:1012C000043003F001031D434846CAF80450FFF7F9
:1012D000B9FE38465CE733680360736843601B2AD5
:1012E00027D800F1080306F10802F2E63B4632680F
:1012F0001A6072685A60B2689A603E467446D04678
:1013000033E708EB0501C5EB0B0B4BF001029960CD
:101310004A6056F8043C03F001031D43484646F872
:10132000045CFFF78FFE304632E73146FFF7D6FD0B
:10133000D5E6B3688360F368C360242A28D000F13F
:10134000100306F11002C4E650F8043C23F0030336
:101350001C440AE7314638467446D046FFF7BEFDC6
:101360003E4602E73A46F7E6314638461C46D04646
:10137000FFF7B4FD3E46F8E6B368CAF81030F368EC
:10138000CAF81430242A1BD010360AF11803AEE72D
:10139000336903617369436106F1180200F11803B0
:1013A00097E600BF2C99FF1FB168CAF81010F168CA
:1013B000CAF81410242A0FD010360AF11802CBE60E
:1013C0003369CAF818307369CAF81C3018360AF144
:1013D00020038CE73A4664E73269CAF8182072693C
:1013E000CAF81C2018360AF12002B5E63146384604
:1013F0000193FFF773FD019B59E7B168CAF810101C
:10140000F168CAF81410242A03D010360AF1180221
:1014100047E73269CAF818207269CAF81C201836E2
:101420000AF120023DE700BF38B5074C002305460E
:1014300008462360FBF7E8FE431C00D038BD236854
:10144000002BFBD02B6038BD30A2FF1FFFFFFFFF3A
:10145000FFFFFFFFFFFFFFFFFFFFFFFFFFFFFFFF9C
:10146000FFFFFFFFFFFFFFFFFFFFFFFFFFFFFFFF8C
:10147000FFFFFFFFFFFFFFFFFFFFFFFFFFFFFFFF7C
:1014800090F800F06DE9024520F007016FF0000CC4
:1014900010F0070491F820F040F049804FF000046C
:1014A0006FF00700D1E9002391F840F000F1080047
:1014B00082FA4CF2A4FA8CF283FA4CF3A2FA8CF37F
:1014C0004BBBD1E9022382FA4CF200F10800A4FAE6
:1014D0008CF283FA4CF3A2FA8CF3E3B9D1E904233A
:1014E00082FA4CF200F10800A4FA8CF283FA4CF371
:1014F000A2FA8CF37BB9D1E9062301F1200182FA2B
:101500004CF200F10800A4FA8CF283FA4CF3A2FA30
:101510008CF3002BC6D0002A04BF04301A4612BA3E
:10152000B2FA82F2FDE8024500EBD2007047D1E941
:10153000002304F00305C4F100004FEAC50514F0D0
:10154000040F91F840F00CFA05F562EA05021CBFA1
:1015500063EA050362464FF00004A9E7024B13B1AA
:10156000024800F005B8704700000000691601004D
:10157000002301461A46184600F0CEBC2DE9F0477C
:1015800088B0364C119DD4F8009006460F4614469C
:101590009846002D43D00022314B30463946FEF7A5
:1015A0009FFD80BB0DF11C0E0321109B0393009146
:1015B0003B46CDF80880019432464846CDF810E00D
:1015C00000F092FD079BD8F800109842C1F100018D
:1015D0002ED2491B2B4610F8012B03F8012B079A3A
:1015E000824203EB0106F6D8B44224DDA21B1A4462
:1015F000302103F8011B9A42FBD1002313702846C7
:1016000008B0BDE8F0870022164B30463946FEF799
:1016100085FD0028C6D00DF11C0E0221C5E7D9F8C2
:10162000502004F123039A4207DDD9F85450B2E761
:101630000E462B46D8E71A46DFE704F1240A524645
:10164000D9F854104846FFF7FFFC05460028D6D0CD
:10165000C9F850A0C9F854009DE700BF2899FF1FA2
:101660000000F03F0000F0BF38B5074D074C2C1BC1
:10167000A41005D0013C55F8043D9847002CF9D141
:10168000BDE8384002F0BCBC0000000000000000D3
:10169000F8B5234F0C460646FFF7D2FCBB685D68E1
:1016A00025F00305291B01F6EF7121F47F6121F07C
:1016B0000F01A1F58054B4F5805F07DB00213046AF
:1016C000FFF7B2FEBB682B44984204D03046FFF7C8
:1016D000B9FC0020F8BD61423046FFF7A5FE01309D
:1016E0000DD0104BBA6819682D1B45F00105304626
:1016F000091B55601960FFF7A5FC0120F8BD00210A
:101700003046FFF791FEBA68831A0F2BDEDD064CD8
:101710000449246843F00103001B53600860D5E7C7
:101720002C99FF1F00A2FF1F389DFF1F002945D0E5
:101730002DE9F0410D468046FFF782FC55F8047C08
:101740006A4927F00103A5F10804E2188E68506881
:10175000B24220F0030062D0FE0750600BD455F86F
:10176000087CE41B01F1080EA56875453B446FD069
:10177000E768EF60BD6015186D68ED0742D543F06E
:1017800001026260E350B3F5007F18D2DB085A1CF7
:101790004D6851F83270A76001209B1000FA03F3E6
:1017A00001EBC2001D430838E0604D6041F8324053
:1017B000FC604046BDE8F041FFF744BC70475A0A60
:1017C000042A53D89A0902F139077F0002F138053B
:1017D00001EB870051F827204449083890424DD04A
:1017E000516821F003018B4202D292689042F7D1F6
:1017F000D068E060A2608460D4604046BDE8F041FB
:10180000FFF720BC95683A4FBD4203443FD0D068F3
:10181000E86043F0010285606260E350B3E7FF07D0
:10182000034407D455F8082CA41A1344A068E268AE
:10183000C26090602F4A126843F0010093426060DA
:101840008C60B6D32C4B40461968FFF721FFB0E7F8
:1018500011184968C90744D49168D268CA60034422
:1018600043F0010091606060E350A2E7142A17D8AA
:1018700002F15C077F0002F15B05A9E7AA104B6843
:10188000012505FA02F213434B600246B1E743F02B
:1018900001024C610C61E560A5606260E35088E77D
:1018A000542A06D81A0B02F16F077F0002F16E0569
:1018B0008EE7B2F5AA7F06D8DA0B02F178077F002F
:1018C00002F1770584E740F25450824206D89A0C20
:1018D00002F17D077F0002F17C0579E7FE277E2576
:1018E00076E743F001026260E35062E72C99FF1F44
:1018F0003499FF1F349DFF1FFCA1FF1FC36C70B5FF
:1019000005460C464BB153F8240080B1026843F8F9
:10191000242000230361C36070BD21220421FEF74F
:10192000AFFFE86403460028EDD1002070BD01211F
:1019300001FA04F6721D28469200FEF7A1FF002866
:10194000F3D044608660E4E731B1C36C4A6853F871
:101950002200086043F82210704700BFF0B50C6900
:1019600083B00D46064601F1140E0027DEF8000094
:1019700081B202FB01310B0C000C02FB003389B277
:10198000013701EB0341BC424EF8041B4FEA1343FD
:10199000ECDC3BB1AA68944207DA05EB840201341F
:1019A00053612C61284603B0F0BD69680193013191
:1019B0003046FFF7A3FF2A69023205F10C01074602
:1019C00092000C30FBF7EAF8F26C6968019B52F860
:1019D0002100286042F821503D46DEE7030C1B043D
:1019E000B3B90004102310F07F4F04BF0002083386
:1019F00010F0704F04BF0001043310F0404F04BFDB
:101A000080000233002807DB420003D42020704707
:101A10000023E8E7581C704718467047036813F026
:101A2000070207D0D90720D49A0720D49B08036067
:101A30000220704799B209B91B0C102213F0FF0F56
:101A400004BF1B0A0832190704BF1B090432990797
:101A500004BF9B080232D90704D45B0801D12020BF
:101A600070470132036010467047002070475B08E2
:101A700003600120704700BF10B50C460121FFF73D
:101A80003DFF01224461026110BD00BF2DE9F04F0E
:101A90000D691769BD4283B00C46164604DA2A4622
:101AA00034463D460E461746A368616805EB0708B5
:101AB0009845C8BF0131FFF721FF00F1140C0CEB72
:101AC0008809CC45009005D26346002143F8041BE9
:101AD0009945FBD806F1140202EB870A04F11403BE
:101AE000524503EB850E54D2CDF80490994652F836
:101AF000043B1FFA83FBBBF1000F20D000204F46B0
:101B00006646054600E01E4657F8044B3068A1B211
:101B100083B20BFB0131240C000C4B190BFB0400AE
:101B200000EB134099B2334641EA0041BE454FEA0B
:101B3000104543F8041BE6D8756052F8043C5FEA90
:101B4000134B20D0DCF80030674618464D46002184
:101B500000E037462C88000C0BFB040001449CB2CB
:101B60003E4644EA014346F8043B786855F8044B86
:101B700083B2240C0BFB043404EB1143AE454FEA53
:101B80001341E6D87B6092450CF1040CAFD8DDF828
:101B90000490B8F1000F0BDD59F8043CA9F10409D9
:101BA0001BB105E059F8043D13B9B8F10108F9D1AA
:101BB0000098C0F8108003B0BDE8F08F12F0030366
:101BC0002DE9F041144607462ED10E46A4101CD034
:101BD000BD6C95B3E3074FF0000806D4641014D031
:101BE0002868A8B10546E307F8D52A4631463846A5
:101BF000FFF74CFFB6B17268FB6C641053F822100B
:101C0000316043F822600646EAD13046BDE8F081F3
